:020000040800F2
:10000000F0FF001035C5050831560508CD19020866
:10001000D5C50508D5C50508D5C5050800000000EB
:100020000000000000000000000000003556050838
:1000300039560508000000003D5605082DE001086E
:10004000D5C50508D5C50508D5C50508D5C5050814
:10005000D5C50508D5C5050895C60108B9C6010866
:10006000F1C6010829C7010861C701081DD90008A8
:100070002DD9000841D9000855D9000869D90008D0
:100080007DD9000891D90008D5C50508D5C5050852
:10009000D5C50508D5C50508D5C5050899C7010802
:1000A00015160208751502082516020865150208BE
:1000B0009D150208AD150208BD15020805CD000802
:1000C000C9D100080DCD0008CDD10008D5C505085F
:1000D000D5C505082DDA01081DDB01080DDC010876
:1000E000D1C70108D5C50508C18A0508351602081B
:1000F000ED15020845160208DD150208A5D900080D
:10010000D5C50508CD050108CD150208D5C50508DA
:10011000FDDC0108EDDD0108D5C50508D5C50508DC
:10012000B9D90008CDD90008E1D90008F5D90008EF
:1001300009DA0008D5C50508D5C50508D5C50508DF
:10014000D5C50508D5C50508D5C505084156050816
:100150001DDA000831DA000845DA0008DDDE0108A2
:1001600015CD0008D1D10008D5C50508D5C50508AD
:10017000D5C50508D5C50508D5C50508D5C50508E3
:08018000D5C50508D5C5050829
:0828000000C00F0800001008E1
:1080000082B01E4B002201920193019B1C4A043353
:108010000193019B1968936803F00C03042B06D0AD
:10802000082B08D0174B184A1A6002B07047154B3E
:10803000196002B070475368506813F4800F00F065
:108040003F00536812D1C3F388130F49B1FBF0F11D
:1080500001FB03F30A4A0B495268C2F301420132A1
:108060005200B3FBF2F30B6002B07047C3F3881306
:10807000B1FBF0F101FB03F3ECE700BF5028004037
:1080800000380240081900200024F400B84B00EB2F
:10809000800103EBC10170B54A685268B2F814E080
:1080A0001EF0010F4FEA800C6ED15FFA8EF4A60726
:1080B00042D5BFF35F8F91F82040012CE5B200F06C
:1080C000D180118BBFF35F8F0CEB000103EBC1017B
:1080D00091F82040022C00F0E7800CEB000103EB4C
:1080E000C10191F82040032C07D191F8221021B151
:1080F00093F87D10002940F0E780918889B241F41F
:108100008061918093F97C100CEB000E03EBCE0E96
:108110009EF820E00EF1010E8E450CD1002183F86F
:108120007D1093F87E10002940F0B780604403EB87
:10813000C00300225A7770BD65075DD414F0400477
:1081400000F0CB80148A93F97C508E6AE4B27455A7
:108150005FFA85FE0EF1010464B291F8206083F8A5
:108160007C40E51CAE42214600F025810CEB000569
:1081700003EBC50595F82050AC42C5D10EF10201C4
:1081800049B283F87C10BFE7B2F800E02EF4006E2D
:108190004FEA0E4E4FEA1E4EA2F800E01488A4B239
:1081A00044F48064148091F82240002583F87C50C8
:1081B000002C48D093F87D40002C41D0012183F859
:1081C0007D100CEB000103EBC10191F82010022996
:1081D00004D1118889B241F4006111800CEB0001D7
:1081E00003EBC101897F41F001011182604403EB7F
:1081F000C00393F8203070BD91F82240012583F828
:108200007E50002C70D093F87D40002C71D10CEB87
:10821000000103EBC10191F82110002900F0AA80B0
:10822000118889B241F40071118093F87C100131FA
:108230004CB283F87C401188CE05FCD4214663E71C
:10824000C97FFF29BAD00CEB000103EBC1018C7F81
:1082500004F0FE041482CA7FFF2AC7D0FF2283F8ED
:108260007C20C3E791F8221000293FF42AAF93F84D
:108270007D1000293FF425AF118821F480610904A5
:10828000090C1180BFF35F8F118B118883F87E502A
:1082900089B241F4007111802FE7918821F4407177
:1082A0000904090C918041E791F8221000293FF45C
:1082B00014AF93F87D1000293FF40FAF118821F41B
:1082C00080610904090C1180918821F480610904FE
:1082D000090C918093F97C1016E71FFA8EF52D0694
:1082E0002DD493F97C100FE793F87D1000298ED0E0
:1082F00096E791F82040022C148846D924F4806433
:108300002404240C1480158A8E6A93F97C40EDB203
:1083100035558E6A118889B241F400711180E4B23A
:10832000158A611C49B2EDB275549188023489B244
:1083300064B241F4806183F87C4091807BE793F9DB
:108340007C506E1C3ED04C6A665D16826C1C91F8A7
:10835000205064B2A54283F87C4021467FF4D4AE1D
:10836000948824F480642404240C9480CCE600BF18
:1083700008190020118893F97C4089B241F480717A
:108380001180012183F87D1055E7A4B244F40074F4
:108390001480158A8E6A93F97C40EDB23555E4B2AB
:1083A0008E6A158A611C49B20334EDB264B2755409
:1083B00083F87C403FE7958825F480652D042D0CDB
:1083C0009580D3E683F87C40CC7F148291F82240DC
:1083D00024B991F8201000297FF408AF918821F486
:1083E00080610904090C918000E700BF30B5EAB153
:1083F0008E464FEA014C034600F1C005002419687F
:108400009A6841EA0C0142EA0E029A60C3E900143C
:108410000C33AB42F3D1D0F8C030C0F8C44043EACB
:108420000E03C0F8C030C0F8C84030BD4FEA014E5E
:108430008C46E0E783691969B3F80CC00A6830B468
:108440009C6822F0010224680A60A28992B222EAA2
:108450000C02A281027D04681F2A06D96568203AB1
:1084600008209040284245D0FEE72568082090402B
:108470002842F9D1202000FA02F2A260264A12789E
:10848000002A35D01A7E012A39D0D3F8F4200132DF
:10849000C3F8F420EFF31181502282F31288586858
:1084A0005C6C026822EA04029C6C2243C9B202603E
:1084B00081F31188D3E90C401A6999681D6C096829
:1084C00014605061D3E90E40546090600024B3F80A
:1084D000A800D5604C62C862106801242043106077
:1084E0001C7683F8F1408A899B8913439BB28B8168
:1084F00030BC7047202000FA02F2E260BEE70022A2
:1085000083F8F120D3F8F8000A68013022F0010264
:10851000C3F8F8000A60EBE70400001010B40C4C3C
:108520006368002B11DD002004F1080C0146DCF823
:10853000A03003F1C00259600C339342FBD1636851
:10854000013083420CF5807CF1DC5DF8044B704710
:1085500004000010F0B5494C04EB401C9CF82424A6
:1085600002B9F0BD464B4FF08C0E0EFB003E93F867
:10857000E06493F8E1249EF882708CF80A749642C5
:108580004FF0000C4FEA40158EF882C00ED002EB7F
:10859000420C03EBCC0C57009CF8E4C40CF1FF3EFA
:1085A000BEF1010F5CD9BCF1030F53D06019A0F8E4
:1085B0000814EFF31182902383F3128890F80A34A1
:1085C000B0F8081443EA41030021D2B29BB280F80C
:1085D0000A1482F311881A09217882EA13225A4078
:1085E000D9B1D0F82044D0F80C14D4F8A040D2432C
:1085F0001B019BB202F00F0201208840134304F1DB
:10860000C0015A0013F4004F93B202D162680243D2
:1086100062600C348C42F4D1F0BDD0F82014D0F854
:108620000C04D1F8A0401B0100F110019BB202F034
:108630000F0201208840134304F1C0015A0013F4D3
:10864000004F93B202D16268024362600C34A142CF
:10865000F4D1F0BD02F1010C0CF0030CB445A5D02F
:108660003A4403EBC202131893F8F11400299DD089
:108670006319012283F80A2498E700BF0400001060
:1086800008190020704700BF024B03EB401090F820
:1086900025047047040000104368B0F8502010B45F
:1086A0001A83EFF31182502383F312884168446CDC
:1086B0000B6823EA0403C46C2343D2B20B6082F339
:1086C0001188D0E907418268036912681C6059610A
:1086D000D0E909415C60C46A9960B0F86010DC6060
:1086E0000023D1625DF8044B03767047037D1F2B96
:1086F00030B54FF02002046816D9A3F12005616857
:10870000AA400A420FD00C4A002182F84415416861
:108710000A681F2B22F001020A604FF0200206D9DE
:10872000203B9A40E26030BD21689A40E9E702FAB6
:1087300003F3A360F7E700BF081900202DE9F0411B
:1087400015F0C0FC1F4F204E05464FF000087C6816
:10875000002C2ADD00231A4607EB0321013391F890
:10876000F9109C4242EA0102F6D142EA0804E4B25E
:1087700090467368C3F30803A3B9EFF311838BB971
:1087800017F0CCFC431BB3F5FA6F02DCB8F1000F15
:10879000DDD124B10D4B93F845254F2A09D0204651
:1087A000BDE8F08115F062FCECE744464FF00008AC
:1087B000DFE7B3F84C250132A3F84C252046BDE88D
:1087C000F08100BF0400001000ED00E00819002057
:1087D000074BD0F8E4105B68D0F8F0205B1A9A429F
:1087E000B8BFC0F8F030012380F81C31002070477A
:1087F000001000E04FF40063838170473D4B9FED14
:108800003E4A93F8511593F8500593F8522593F882
:1088100053C5090201EB00410A44090248BF02F1B5
:108820007F4207EE902AB3F96C2593F8540593F82C
:10883000551506EE102AB3F96825F8EEE77A06EE2C
:10884000902A67EE847AB3F96A25B8EEC66AF8EE24
:10885000E66A0002E7EE866A00EB0C40014406EE91
:10886000102AB3F9662505EE102AD3F86025000218
:1088700007EE102AB3F9642548BF01F17F41F8EEF5
:10888000C75A04EE902A07EE101AD3F85C25B8EE0A
:10889000C66AB8EEC55AE6EEA75A012006EE902A3F
:1088A000B8EEC77AA7EE865AB3F95A25B3F9583508
:1088B00027EE047AF8EEE44AB8EEE66A06EE902A6D
:1088C000A7EE246AE5EE075AF8EEE66A05EE103ADE
:1088D00026EE877AB8EEC55AF6EE004AF0EE466A02
:1088E000E7EEA56A054BA5EE247AC3ED066A83ED93
:1088F000077A70470819002008218436601E00207E
:1089000030B10A4BD3ED067AFDEEE77AC0ED007A7E
:1089100051B1064B9FED067AD3ED077A67EE877A61
:10892000FDEEE77AC1ED007A704700BF601E0020BF
:108930000000C842704700BF012070470120704707
:10894000704700BF024B002083F87805704700BFD6
:1089500008190020122301480B807047880100206D
:10896000042301480B8070479C0100202048D0F868
:10897000E837D0F8EC2730B59B184FF01A040C807C
:1089800001D11C4830BD1B4AD0F8EA174FF0000E49
:1089900010467546B3F1204F4FEA137C0CF13004BA
:1089A0000EF1020E2ABF0CF1370C847080F802C061
:1089B000BEF1100FC5704FEA031300F10200E9D1B8
:1089C00000200446B1F1204F4FEA117303F1300C3F
:1089D00000F102002ABF373382F812C093740828CE
:1089E000D4744FEA011102F10202EBD1014830BD0B
:1089F00000F0FF1FA001002038B5074BD3F87C35ED
:108A00001B6A14460D4698474FF4007302682A60AB
:108A10000020236038BD00BF0819002008B5074BAF
:108A2000D3F87C3533B15B69984780F00100404250
:108A300040B208BD4FF0FF3008BD00BF081900204C
:108A4000002070472DE9F04123B3164D16468846A5
:108A50009F18D5F87C450023A4681A464146304645
:108A6000A0470028F5D0D5F87C3533B15B6998472D
:108A700020B9D5F87C35002BF8D1FEE70136B74296
:108A800008F50078E5D1D5F88035C5F884350020A3
:108A9000BDE8F081034DD5F88035C5F88435002058
:108AA000BDE8F081081900202DE9F0415BB31A4CB4
:108AB00016460F4603EB020804E0D4F87C1519B102
:108AC0004B699847D4F87C150D6900231A4639463E
:108AD0003046A8470028F0D1D4F87C3533B15B6923
:108AE000984720B9D4F87C35002BF8D1FEE7013641
:108AF000B04507F50077E5D1D4F88035C4F8843562
:108B00000020BDE8F081044CD4F88035C4F88435E9
:108B10000020BDE8F08100BF081900200020704748
:108B200000207047002070472DE9F04FDFF81C93BC
:108B300099F800A091B0BAF1000F03D1012011B053
:108B4000BDE8F08FBC49D9F80835BC4A0493D1F888
:108B50008035CDF800A0A2FB0323B94A5B09A2FB34
:108B6000032C4FEADC0C0CEB8C0CA3EB4C0C91F8B7
:108B7000E134182202FB031303F2F1430F930B4677
:108B800091F88815029193F845150391B3F94E15A4
:108B90000B91D9F814150191B3F94815B3F94A3579
:108BA00006910022D9F810150D9309F214645FFAAA
:108BB0008CF317460C920891079304EB8C0C09F583
:108BC000816609F20C5B09920E920A920592049B4F
:108BD000BB4240F3DC807368B2694FEA830AD2E992
:108BE0003A310AF1085A0AEB431A01F18060029BFC
:108BF00039380AEB80100AEB8313984240F28781E0
:108C00001A68002A00F06F811A6C002A00F06D814A
:108C1000D3F88020002A00F06A81D3F8C02003F541
:108C20008073002AE9D1039DA3EB0A0A4F2D4FEA76
:108C3000AA12CAF3871A00F03781984240F29B804B
:108C4000891A45294FF0000528BF452103EB811102
:108C500098462846AE460DE01A6C002A40F0C080C7
:108C6000D3F88020002A40F0F380D3F8C02003F529
:108C700080732AB9994206D91A68002AECD0403389
:108C8000994200F2B1807546112D40F25981CEF122
:108C90001503002BC0F25481AAF10A0A5FFA8AF286
:108CA000029206D098400122CEF1140302FA03F397
:108CB00018436449C0F3C4330D4651F8232000F033
:108CC0001F0351F8233043EA0233C0F34412C0F3C8
:108CD000842051F8221043EA011155F8203041EA6E
:108CE000032181EA112383EA131303F00F030F2BEF
:108CF00040F0CC80B1F5803F80F0C880039B4F2BC3
:108D00004FEA111100F0D880019BB1F5606F03F1BB
:108D10000103019300F0DD80ABF80C1094F858309B
:108D20000798834210D0DCF8082023689B1A236040
:108D3000DCF8302063689B1A63600023CCF80830AD
:108D4000CCF8303084F85800236801332360DCF815
:108D500008300133CCF808304FF6FF73994240F0E9
:108D60009280636801336360DCF830300133CCF803
:108D70003030009B05930137082F04F15C040CF19F
:108D80005C0C06F120060BF1140B7FF420AF059B61
:108D90001BB1294B029A83F888250A9B1BB1264BED
:108DA0000B9AA3F84E250E9B1BB1234B0D9AA3F8EB
:108DB0004A25099B1BB1204B069AA3F84825059B21
:108DC00013B1019BC9F814350C9B13B1089BC9F86A
:108DD00010350123012089F8123611B0BDE8F08F5B
:108DE000803399427FF64FAFA3EB08029211551CD6
:108DF000154A82FB0582A2EBE572012AB8BF012267
:108E0000904001259644013A05FA02F210431D46AE
:108E10002A68FAB12A6C002A6BD0D5F88020002A83
:108E200069D0D5F8C02005F58075A2B1A942EFD868
:108E300098462B461EE700BF081900201F85EB51FE
:108E4000CDCCCCCCF8DB05085655555504000010A8
:108E5000C03315E74035A942EAD9EB1A9B115A1CD9
:108E60003A4B83FB0283A3EBE273012BB8BF0123D0
:108E700098409E440122013B02FA03F318432B461B
:108E800098462B46F6E6009B059374E7039B4F2B11
:108E900033D0019B01330193089B01330893009B5E
:108EA0000C934FF6FF7139E70FFA8AF598420B954C
:108EB0003DD900980A90C3E6069B01331BB2069386
:108EC000019B01330193B1F5606F009B09937FF41F
:108ED00023AF0F9BDB5D0D2B7FF41EAF6FF07F0385
:108EE0008BF81E301AE740339DE680339BE6C03393
:108EF00099E68035AFE7C035ADE7069B01331BB27D
:108F00000693019B01330193009B0993C4E7039DE2
:108F1000A3EB0A0A4F2D4FEAAA12CAF3871A7FF46D
:108F20008CAE0FFA8AF30B93009B0A9301E0009B2F
:108F30000A930D9B01331BB20D93009B0E931AE70E
:108F4000039B4F2B7FF417AFF3E700BF56555555E2
:108F500010B5044654F022F981B22046BDE8104015
:108F6000FFF7F8BA2DE9F0411E4B93F8E02493F88F
:108F7000E1349A422FD11C4F7D68002D12DD384616
:108F8000002410F8086BA046013416B1037E012BB3
:108F90001CD002691368AC4243F0010300F58070F5
:108FA0001360F1D115F08EF8D7F8F448002C0BDDE2
:108FB0000E4A02EBC404116893888889083203437F
:108FC0009BB294428B81F6D1BDE8F08180F8F080AD
:108FD000FFF762FBDDE750F08DFB0028CBD1BDE849
:108FE000F08100BF0819002004000010FC080010E8
:108FF00010B57D4C94F8E02494F8E1349A4240F0A6
:1090000099817A4B93F81829002A00F0EC8093F8A4
:109010001C39002B40F0EC80D4F88C15088820F027
:1090200080000004000C0880B4F89005C86208882D
:1090300080B240F0800008804B62B1F80CC0B4F8F8
:10904000A00540EA0C0080B2012A8881A4F8A0356E
:1090500000F0C980D4F8A415088820F0800000042E
:10906000000C0880B4F8A805C862088880B240F0F7
:10907000800008804B62B1F80CC0B4F8B80540EA33
:109080000C0080B2022A8881A4F8B83500F0AB80C9
:10909000D4F8BC15088820F080000004000C08807B
:1090A000B4F8C005C862088880B240F0800008802B
:1090B0004B62B1F80CC0B4F8D00540EA0C0080B2A5
:1090C000032A8881A4F8D03500F08D80D4F8D41517
:1090D000088820F080000004000C0880B4F8D8054F
:1090E000C862088880B240F0800008804B62B1F806
:1090F0000CC0B4F8E80540EA0C0080B2042A88816C
:10910000A4F8E8356FD0D4F8EC15088820F080007A
:109110000004000C0880B4F8F005C862088880B22A
:1091200040F0800008804B62B1F80CC0B4F8000633
:1091300040EA0C0080B2052A8881A4F8003652D09B
:10914000D4F80416088820F080000004000C088081
:10915000B4F80806C862088880B240F08000088031
:109160004B62B1F80CC0B4F8180640EA0C0080B2AB
:10917000062A8881A4F8183635D0D4F81C16088839
:1091800020F080000004000C0880B4F82006C862BB
:10919000088880B240F0800008804B62B1F80CC0B3
:1091A000B4F8300640EA0C0080B2072A8881A4F89F
:1091B000303618D0D4F83426B4F83806118821F0A7
:1091C00080010904090C1180D0621088B4F8481697
:1091D00080B240F08000108053629089014389B2D0
:1091E0009181A4F8483610BD081900200400001031
:1091F000D4F89435B4F8981559601968D4F88C05EA
:1092000041F00101196040F20D33A0F84830818926
:1092100089B241F48071012A8181E4D0D4F8AC157F
:10922000B4F8B0054860086840F001000860D4F860
:10923000A405A0F84830818989B241F48071022ADE
:109240008181D0D0D4F8C415B4F8C8054860086846
:1092500040F001000860D4F8BC05A0F848308189CE
:1092600089B241F48071032A8181BCD0D4F8DC1525
:10927000B4F8E0054860086840F001000860D4F8E0
:10928000D405A0F84830818989B241F48071042A5C
:109290008181A8D0D4F8F415B4F8F80548600868BE
:1092A00040F001000860D4F8EC05A0F8483081894E
:1092B00089B241F48071052A818194D0D4F80C16CA
:1092C000B4F810064860086840F001000860D4F85F
:1092D0000406A0F84830818989B241F48071062AD9
:1092E000818180D0D4F82416B4F828064860086834
:1092F00040F001000860D4F81C06A0F848308189CD
:1093000089B241F48071072A81813FF46CAFD4F8AF
:109310003C16B4F840264A600868D4F8342640F079
:1093200001000860A2F8483093899BB243F480732F
:10933000938110BD50F0DEF900287FF462AE10BDBD
:1093400070B5104ED6F80835002B19DD06F581648E
:10935000002505E0D6F80835AB4204F120040FDD06
:10936000237F0135002BF5D0E0680028F2D0217D65
:1093700013F0EEFBD6F80835AB4204F12004EFDC25
:10938000012070BD04000010F8B5037D85691F2B16
:1093900004464CD90168A3F120024E682020904079
:1093A000064233D010239340C860CB604B68D34053
:1093B000DE077BD4EFF31183502282F312882A6CEC
:1093C0001168C9075AD4516889B271B9D5E90960E1
:1093D000864250D0AF690744D7606CD9301A80B24A
:1093E0005060AE62002185F86410116841F00101FF
:1093F000DBB2116083F3118895F86430002B44D1FF
:10940000237D1F2B27D92168A3F120024C68082057
:109410009040044200D0C8604C68042000FA02F278
:10942000224203D0203B00FA03F3CB60F8BD026870
:10943000202016689840064219460ED01021994007
:10944000906091601168D940C807B3D5012101FA35
:1094500003F39360AEE722681946106808238B4037
:10946000184200D093601068042303FA01F101420E
:10947000DCD09160F8BD012285F86420DBB283F373
:10948000118895F86430002BBAD095F87C30002B09
:10949000B6D195F8710013F0CFFF012385F87C3029
:1094A0000028ADD0202113F053FBA9E7012303FAD4
:1094B00002F2CA607EE72E69301A80B25060A9625B
:1094C00090E700BF2DE9F047037D02681F2B04469B
:1094D00008D95068A3F120052021A940014206D1F6
:1094E000BDE8F0871068202199400142F8D0BB49BF
:1094F000BB4E4968C6F8201996F81C19D4F8189084
:10950000DFF8E482F1B98C2101FB0981D1F88800F0
:10951000D1F8007105683868B1F88CC020F00100FE
:109520003860A98989B221EA0C01A9813178E9B9A9
:109530001F2B40F2B580A3F1200120238B40D36084
:10954000BDE8F0878C2101FB0981D1F888104869BA
:109550000D68016821F001010160A98921F4807181
:109560000904090CA98131780029E1D04FF08C0A57
:109570000AFB098ADAF80071384647F0E5FED6F8AA
:10958000283901228AF8D420002B00F0F5802A889F
:109590008C2303FB098392B242F080022A80B3F845
:1095A000F4204FF0FF31E962002A7FD12A8CB3F812
:1095B000F610B3F8F800B3F8FCC022F00102120470
:1095C000120C2A84B3F8FA202B8B23F0F3031B042C
:1095D00040EA0C101B0C0343288C9BB22B8383B2F4
:1095E00023F00A030B4343F001032B842B8B23F05E
:1095F0000C031B041B0C2B832B8B9BB21A432A835B
:109600008C2303FB09830022D3F8AC00C3F8A42009
:10961000D3F8982039680243D3F8B0000243D3F856
:10962000B4000243D3F8B8000243D3F8BC000243AD
:10963000D3F8C0000243D3F8CC000243D3F8D000E3
:1096400002436848084002433A60D3E9312079690F
:10965000024321F007010A437A61D3F8A8207A6017
:10966000D3F89C20BA60D3F8A020FA60D3F8002188
:1096700016215160116841F001011160D3F8882072
:10968000B3F88C30126891890B439BB25349938194
:109690004B68C6F82439237D22681F2B3FF64BAF59
:1096A000202101FA03F39360BDE8F087042A33D048
:1096B000082A2A8C65D022F48052B3F8FC10B3F843
:1096C000F800B3F8F6C01204120C2A84090341EA28
:1096D0000020A98BB5F820E0B3F8FA2045F6FF7317
:1096E00003EA0E0343EA0C3340F6FF4C0CEA010197
:1096F0009BB2014343F4805389B2A9832B84AB8B83
:1097000023F440631B041B0CAB83AB8B9BB243EA7B
:1097100002239BB2AB8373E7298CB3F8F820B3F82C
:10972000FC00B3F8F6C021F010010904090C2984EB
:109730001202B3F8FA1042EA0032288B2B8C9BB24B
:1097400023F0A00343EA0C1340F6FF4C0CEA0000A0
:109750009BB2024343F0100392B22A832B842B8BDB
:1097600023F440631B041B0C2B832B8B9BB243EA1B
:1097700001239BB22B8343E714F0A4FCC6F828090D
:1097800005E722F480721204120CB3F8F600B3F865
:10979000F810B3F8FCC02A84B3F8FA20AB8B23F09E
:1097A000F3031B0441EA0C111B0C0B4399B22B8CE5
:1097B000A9839BB223F4206343EA00239BB243F4C2
:1097C00080732B84AB8B23F00C031B041B0CAB832B
:1097D000AB8B9BB21A43AA8312E700BF001000E0D4
:1097E000040000103F801CF0081900202DE9F04F04
:1097F000DFF80CB19BF8004087B024B90124204663
:1098000007B0BDE8F08F3B4ED6F8805514F05AFCF7
:109810009BF860390390002B00F0DE82364AA2FBF1
:109820000532364B5209A3FB0213DB0803EB83031B
:10983000A2EB4303DAB204920BF2146202EB83034D
:1098400000930BF20C53019206F1E00402930027FF
:10985000DBF82839039AD31A04D454F8082C93421D
:10986000C0F26A82234A54F858AC256ADAF80060DC
:109870008C2303FB072393F8D430002B40F0968110
:10988000284647F061FD1B4A8C2303FB0723002277
:1098900083F8D4209AF805100C2914D8DFE811F0C9
:1098A000780113001300130071011300130013005B
:1098B0007F011300130013000D00B38B23F400632A
:1098C0001B041B0CB3832246304617F04FFF9AF857
:1098D00005300C2B1ED8DFE813F04B011D001D00D6
:1098E0001D0042011D001D001D0039011D001D004D
:1098F0001D001500081900201F85EB51CDCCCCCCE4
:1099000004000010B38B23F400631B041B0C43F40E
:109910000063B383019B54F8342C54F8101C5C335F
:109920000193009B5C330093029B1433029354F821
:10993000483C43F04003134354F8302C134354F88D
:109940002C2C134354F8282C134354F8242C134381
:1099500054F8202C1343402244F83C2C54F8142C87
:1099600013432A6822F07E6222F45F3222F470727E
:109970000B4313432B6054E907316A690B4322F010
:10998000070213436B6154F8383C6B6054F8443C55
:10999000AB6054F8403CEB602B6843F010032B6045
:1099A0009BF8603901379F4204F18C04FFF650AFF9
:1099B000012200218BF81226CBF82819002B3FF446
:1099C0001DAF9D4890F89010890700F1A081D0F854
:1099D0008810086849798A40018C92B289B221EADC
:1099E00002010184018C89B20A43012B02843FF4F5
:1099F00005AF914991F81C21970700F1A281D1F898
:109A0000142110685479018C012289B2A24092B2CB
:109A100021EA02010184018C89B20A43022B0284EB
:109A20003FF4ECAE844991F8A821960700F1A28199
:109A3000D1F8A02110685479018C012289B2A2408A
:109A400092B221EA02010184018C89B20A43032BFC
:109A500002843FF4D3AE784991F83422950700F19F
:109A60009281D1F82C2210685479018C012289B29C
:109A7000A24092B221EA02010184018C89B20A4318
:109A8000042B02843FF4BAAE6B4991F8C0229407CC
:109A900000F18281D1F8B82210685479018C01223A
:109AA00089B2A24092B221EA02010184018C89B2FA
:109AB0000A43052B02843FF4A1AE5F4991F84C2381
:109AC000900700F17281D1F8442310685479018C19
:109AD000012289B2A24092B221EA02010184018CE2
:109AE00089B20A43062B02843FF488AE524991F8AA
:109AF000D823920700F16281D1F8D02310685479FD
:109B0000018C012289B2A24092B221EA02010184B1
:109B1000018C89B20A43082B02847FF46FAE464A57
:109B200092F864349B0740F15281D2F85C240423FC
:109B3000116850790A8C83409BB292B222EA0302E8
:109B40000A840A8C92B213430B8457E6B38B23F03A
:109B500008031B041B0C43F00803B383DAE6338BC2
:109B600023F400631B041B0C43F400633383D1E62E
:109B7000338B23F008031B041B0C43F008033383CF
:109B8000C8E6338B23F400631B041B0C33839AE673
:109B9000338B23F008031B041B0C338393E6B38B36
:109BA00023F008031B041B0CB3838CE66B6834F8AA
:109BB000542C1FFA83F8B389C8F116089BB223EA24
:109BC0000203B8F1070FB3817FF65AAEDBF8143504
:109BD0000133CBF81435A36A05939E4600225EF844
:109BE00004CB0121914660461DE0DEF800C0B9F1CA
:109BF000140FACEB000321DC13F1080048BF03F1A4
:109C00001700031109EB2019604603F1FF3C0131F5
:109C100002FA03F3012202FA0CF2884542EA030237
:109C20000EF1040E0AD38845DFD8C9F11503DEF81A
:109C300000004FF01509E8E708190020B9F1150FE9
:109C40005CD16848C2F38423C2F3441100EB830360
:109C500000EB8101D3F88030D1F880101B0243EA79
:109C6000011302F01F0100EB8101C2F3C43200EBCB
:109C70008202D1F88010D2F880200B4343EA0233ED
:109C800083EA132282EA121202F00F020F2A35D160
:109C9000C3F30F134FF6FF7293422FD0B3F5606FEB
:109CA00058D0029A93810198049990F858208A42DA
:109CB00010D0009A91680268521A00990260096BEC
:109CC0004268521A0099426000228A600A6304992D
:109CD00080F85810019900980A6801320A60826879
:109CE000013282604FF6FF7293427FF4C9AD4B6838
:109CF00001334B60036B01330363C1E5DBF81035BF
:109D00000133CBF810356FB14FF6FF73CBE7364A0E
:109D1000D2F8882010685479018C0422A24089B2BC
:109D200092B25CE605993148582253F0AFFEDAF85A
:109D300000604FF6FF73B6E70024204607B0BDE889
:109D4000F08F294AD2F8142110685479018C04222A
:109D500089B25BE6244991F8E12402EB420201EB6F
:109D6000C2023A4492F8F1240D2A9AD10299802233
:109D70008A7798E71C4AD2F8A02110685479018CA0
:109D8000042289B25BE6184AD2F82C221068547972
:109D9000018C042289B26BE6134AD2F8B82210680B
:109DA0005479018C042289B27BE60F4AD2F844230D
:109DB00010685479018C042289B28BE60A4AD2F8E1
:109DC000D02310685479018C042289B29BE6064B9B
:109DD000D3F85C240123ABE601228BF81226CBF8E2
:109DE00028390CE5F8DB050808190020BC0500102F
:109DF000F8B590F871301C09013C052C0FD8184EAD
:109E000006EB44020546B2F8000103F00F0340FAE6
:109E100003F2D20703D595F87C70012F01D0012001
:109E2000F8BD07FA03F3013B1840344452F0AEF991
:109E300094F80C210B4C104454F8302004EBC0046F
:109E40001069A3881840EBD0EB6E002285F87C20C7
:109E5000204693F82120022113F05AF83846F8BD25
:109E6000F8DB0508541F00202DE9F04F836893B0FC
:109E7000044613B11A689B885383B64B5B68C3F3DF
:109E80000803002B40F04081EFF31183002B40F0DA
:109E90003B81B14B4FF0E025D3F88015A869D3F88A
:109EA00080258A42F8D1D3F854198842F4D8D3F8DF
:109EB00050694FF47A7505FB06F1091AB1FBF6F10A
:109EC00005FB0211A34E4FF0E0204FF47A754FF0DE
:109ED000100C01277268C2F30802002A40F0C78004
:109EE000EFF31182002A40F0C280D3F88085D0F8C9
:109EF00018E0D3F880259045F7D1D3F8542996453A
:109F0000F3D8D3F8509905FB09F2A2EB0E02B2FB8D
:109F1000F9F205FB0822521AB2F57A7FDAD3A26869
:109F200012B1116892880A838A484FF00A0B1025F3
:109F30004FF0E0214FF47A7C4268C2F30802002A15
:109F400040F0B780EFF31182002A40F0B280D3F8DE
:109F50008025D1F81880D3F88065B242F7D1D3F8C4
:109F60005469B045F3D8D3F850990CFB09FEAEEB19
:109F7000080EBEFBF9FE0CFB02EE4268C2F30802BB
:109F8000002A54D1EFF31182002A50D1D3F8806512
:109F90008F69D3F880259642F8D1D3F85429974297
:109FA000F4D8D3F850A90CFB0AF2D21BB2FBFAF298
:109FB0000CFB0622A2EB0E02B2F57A7FDDD3BBF1D9
:109FC000010BB9D12368ADF804B05A6A2AB19442A2
:109FD00003D0002013B0BDE8F08F1B6A002BF8D12E
:109FE00080200DF103018DF80300029101A80221E8
:109FF000CDE90801002000210122CDE90C0102A9D0
:10A000002046CDE90332CDE906338DF814308DF8C2
:10A0100028200B930E938DF83C20109311F07EFFB7
:10A0200023685A6A002A68D094425AD0FEE7EFF3B8
:10A03000118985F312888F690A69D20303D5012239
:10A04000C3F84C298F69D3F88025D3F84C695FFA9F
:10A0500089F989F3118806EB0208D3F850690CFBE3
:10A0600006F2D21BB2FBF6F20CFB0822A2E7EFF3DA
:10A0700011828CF31288D0F81880D0F810E01EF40A
:10A08000803F03D0C3F84C79D0F81880D3F880957E
:10A09000D3F84CE9D2B282F31188CE44D3F8509968
:10A0A00005FB09F2A2EB0802B2FBF9F205FB0E2256
:10A0B00031E7EFF3118E85F31288D1F818800A6921
:10A0C000D60304D50122C3F84C29D1F81880D3F85F
:10A0D0008095D3F84C295FFA8EFE8EF311884A449E
:10A0E00041E71A6A002AFCD19DF80530242B14BFE1
:10A0F00000200F2013B0BDE8F08F1A6A002AF3D0B9
:10A100001A6A002AF9D1EFE7EFF31181102383F3E4
:10A1100012884FF0E0229069136913F4803F0E4BD0
:10A1200003D00120C3F84C099069D3F88055D3F8C7
:10A130004C29C9B281F31188D3F8506951194FF4F1
:10A140007A7505FB06F2121AB2FBF6F205FB012145
:10A15000B8E600BF00ED00E00819002010B5044685
:10A160000E49D0F8D83094F8D020D0F8E4004968EF
:10A170000344012AC4E9361305D0D4F8D43001339E
:10A18000C4F8D43010BD04F1E801201D11F0C6FE62
:10A19000D4F8D4300133C4F8D43010BD001000E03E
:10A1A00070B5866996F8DC30012B8AB0054629D057
:10A1B000023B012B31D8D6F89C301D4C8C221A70F2
:10A1C0000FCCEC46ACE80F00D6F89C300093D6F8E4
:10A1D000A03001930FCCACE80F0094E80300AB690A
:10A1E0008CE8030003F11000694611F097FEAA699C
:10A1F0001369596A103299B18A4200D0FEE71A6A8F
:10A20000002AFCD1D6F8A030B3F90220EA81B3F9D4
:10A2100004202A82B3F906306B8201200AB070BD97
:10A220001A6A002AEED01A6A002AF9D1EAE700BFBA
:10A230000CDD05082DE9F04190F81E31032B92B09A
:10A24000044650D090F8DC00D4F8A070012800F04B
:10A25000E28016D8D4F89C3000221A605A609A60C6
:10A260009A81D4F8E0300522B3F57A7FC4F8F02063
:10A270002CD801250323284684F8DC3012B0BDE831
:10A28000F0810238012829D8D4F89C30804E9222DF
:10A290001A700FCE02AD0FC50FCE0FC596E80300A2
:10A2A000D4F89C3004F1100885E80300029302A959
:10A2B000D4F8A0300393404611F030FE23695A6A67
:10A2C000002A00F08F80904578D0FEE723691A7B42
:10A2D000002A40F0B980022384F8DC3001252846AA
:10A2E00012B0BDE8F0810023CDE90633CDE9083393
:10A2F00068490B9300F11006674B0291012203930A
:10A3000002A90A2330468DF814208DF828200493E2
:10A3100011F004FE23695A6A002A48D0964200D000
:10A32000FEE71A6A002AFCD15C4AB2F85A39052BBA
:10A330005FDDB2F95C19D2F85C09B2F95E59B2F985
:10A34000602911F5004F77D0C4F8D000A4F8D420CC
:10A350000125063B002BC2D07E238DF80630B023AA
:10A360008DF807300DF106030293002303938DF857
:10A370001430069308930B930E93109301230493C8
:10A3800009938DF828308DF83C300DF10703002239
:10A39000079302A900233046CDE90C2311F0BEFD3E
:10A3A00023695A6A002A2ED0964224D0FEE71A6A00
:10A3B000002AB9D01A6A002AF9D1B5E71A6A002A28
:10A3C000FCD1B7F90230A4F8D030B7F90430A4F8C2
:10A3D000D230B7F90630A4F8D4300125284612B09F
:10A3E000BDE8F0811A6A002AEBD01A6A002AF9D176
:10A3F000E7E70025AEE71A6A002A3FF470AF1A6A51
:10A40000002AF8D16BE71A6A002A3FF468AF1A6A8B
:10A41000002AF8D163E7B7F90830A4F8D030B7F9CB
:10A420000A30A4F8D230B7F90C30A4F8D43005467D
:10A43000284612B0BDE8F08115F5004F84D112F521
:10A44000004F81D1002584E75B69002B3FF443AFC7
:10A4500094F89850002D3FF43EAFD4F89C30C4F8E7
:10A46000A4408C221A70D4F8A020C4F8F8200E2240
:10A4700001230B49C4F8FC20D4F89C20C4F8041133
:10A48000C4F8F42084F8003184F8DC3027E700BFFA
:10A490000CDD0508BC010020602200200819002006
:10A4A000D18700082DE9F04F95B000230122CDE9B6
:10A4B0000532CDE90A328DF81C3008930D931093C4
:10A4C0001293B623054600F110077E2190F81E0175
:10A4D0008DF80F300DF10F0301908DF80E108DF8EF
:10A4E00030208DF844200993002200230DF10E0640
:10A4F00004A93846CDE90E23049611F00FFD2B690F
:10A500005A6A002A00F03B81974200D0FEE71A6A9F
:10A51000002AFCD164239E4CDFF8788207EE907A03
:10A520004FF010094FF0E0224FF47A7C4FF0010B0E
:10A530009A46D8F80430C3F30803002B40F046874E
:10A54000EFF31183002B40F04187D4F880359069F8
:10A55000D4F880158B42F8D1D4F854198842F4D835
:10A56000D4F850190CFB01FEAEEB000EBEFBF1FE61
:10A570000CFB03EED8F80430C3F30803002B40F0C3
:10A580003B86EFF31183002B40F03686D4F88075BC
:10A590009369D4F880158F42F8D1D4F854198B42BE
:10A5A000F4D8D4F850190CFB01F0C31AB3FBF1F343
:10A5B0000CFB0733A3EB0E03B3F57A7FDAD3BAF1C2
:10A5C000010AB6D1AB6917EE907A13B11A689B886D
:10A5D0005383704B5B68C3F30803002B41F02E8458
:10A5E000EFF31183002B41F029844FF0E02ED4F8D3
:10A5F0008025DEF818C0D4F880359A42F7D1D4F817
:10A6000054399C45F3D8A0EB0C03B3FBF1F34FF4A2
:10A610007A7101FB0233DFF87C814FF0E0204FF4C8
:10A620007A7E4FF0100A4FF0010BD8F80420C2F3E5
:10A630000802002A40F06786EFF31182002A40F0FA
:10A640006286D4F88015D0F818C0D4F880259142DD
:10A65000F7D1D4F854299445F3D8D4F850990EFB87
:10A6600009F2A2EB0C02B2FBF9F20EFB0122D21AA4
:10A67000B2F57A7FD9D3AB6913B11A689B8813837B
:10A68000DFF810814FF00A094FF0100A4FF0E02276
:10A690004FF47A7CBB46D8F80430C3F30803002B90
:10A6A00040F0A986EFF31183002B40F0A486D4F884
:10A6B00080359069D4F880158B42F8D1D4F85419BC
:10A6C0008842F4D8D4F850790CFB07F1091AB1FB91
:10A6D000F7F10CFB0311D8F80430C3F30803002B87
:10A6E00040F06885EFF31183002B40F06385D4F8C8
:10A6F00080059769D4F880359842F8D1D4F8543958
:10A700009F42F4D8D4F850E90CFB0EF3DB1BB3FBEB
:10A71000FEF30CFB00335B1AB3F57A7FDBD3B9F1A0
:10A720000109B8D10DF10F03CDE9093901230693D1
:10A730000B938DF830308DF844307C2300228DF857
:10A740000E3004A900235846CDE90E23CDE9046953
:10A750008DF80F908DF81C90CDF82090CDF83490A6
:10A76000CDF84090CDF8489011F0D8FB2B695A6A8B
:10A770005F46002A00F0908093450DD0FEE71A6AEC
:10A78000002A3FF4C7AE1A6A002AF8D1C2E600BF19
:10A790000819002000ED00E01A6A002AFCD1874B5E
:10A7A0005B68C3F30803002B41F02483EFF31183AC
:10A7B000002B41F01F834FF0E020D4F880358169F1
:10A7C000D4F880259342F8D1D4F854299142F4D892
:10A7D000D4F850C94FF47A7000FB0CF2511AB1FB57
:10A7E000FCF100FB0311DFF8D4814FF0E0204FF4BF
:10A7F0007A7E4FF0100A4FF0010BD8F80430C3F303
:10A800000803002B40F06885EFF31183002B40F024
:10A810006385D4F88025D0F818C0D4F880359A42E2
:10A82000F7D1D4F854399C45F3D8D4F850990EFB9D
:10A8300009F3A3EB0C03B3FBF9F30EFB02335B1A32
:10A84000B3F57A7FD9D30DF10F03099300238DF867
:10A850000F3005938DF81C3008930A930D931093D5
:10A860001293012306930B938DF830308DF844300A
:10A87000592300228DF80E3004A900233846CDE973
:10A880000E23049611F04AFB2B695A6A002A00F045
:10A890008C80974208D0FEE71A6A002A3FF47FAF07
:10A8A0001A6A002AF8D17AE71A6A002AFCD1434BC7
:10A8B0005B68C3F30803002B41F07882EFF3118348
:10A8C000002B41F073824FF0E020D4F8803581698D
:10A8D000D4F880259342F8D1D4F854299142F4D881
:10A8E000D4F850C94FF47A7000FB0CF2511AB1FB46
:10A8F000FCF100FB0311DFF8C4804FF0E0204FF4BF
:10A900007A7E4FF0100A4FF0010BD8F80430C3F3F1
:10A910000803002B40F02485EFF31183002B40F057
:10A920001F85D4F88025D0F818C0D4F880359A4215
:10A93000F7D1D4F854399C45F3D8D4F850990EFB8C
:10A9400009F3A3EB0C03B3FBF9F30EFB02335B1A21
:10A95000B3F57A7FD9D3002305938DF81C30089383
:10A960000A930D9310931293012306938DF83030C0
:10A970008DF84430124B09935E238DF80D300DF1A4
:10A980000D0304934FF4A47300220B9304A9002336
:10A990003846CDE90E2311F0C1FA2B695A6A002A14
:10A9A00000F0928097420DD0FEE71A6A002A3FF429
:10A9B0007EAF1A6A002AF8D179E700BF00ED00E007
:10A9C00034DD05081A6A002AFCD1DFF838834FF01D
:10A9D0000A094FF0100A4FF0E0224FF47A7CBB4690
:10A9E000D8F80430C3F30803002B40F0D084EFF311
:10A9F0001183002B40F0CB84D4F880359069D4F8D3
:10AA000080158B42F8D1D4F854198842F4D8D4F880
:10AA100050790CFB07F1091AB1FBF7F10CFB03119C
:10AA2000D8F80430C3F30803002B40F0A283EFF3FF
:10AA30001183002B40F09D83D4F880059769D4F8EA
:10AA400080359842F8D1D4F854399F42F4D8D4F8DC
:10AA500050E90CFB0EF3DB1BB3FBFEF30CFB0033E6
:10AA60005B1AB3F57A7FDBD3B9F10109B8D10DF1E7
:10AA70000F03CDE9093901238DF80F3006930B93AD
:10AA80008DF830308DF84430592300228DF80E3087
:10AA900004A900235846CDE90E23CDE904698DF8B9
:10AAA0001C90CDF82090CDF83490CDF84090CDF8A2
:10AAB000489011F033FA2B695A6A5F46002A00F079
:10AAC0009080934508D0FEE71A6A002A3FF47DAFD4
:10AAD0001A6A002AF8D178E71A6A002AFCD1894B51
:10AAE0005B68C3F30803002B41F03A81EFF3118355
:10AAF000002B41F035814FF0E020D4F8803581699A
:10AB0000D4F880259342F8D1D4F854299142F4D84E
:10AB1000D4F850C94FF47A7000FB0CF2511AB1FB13
:10AB2000FCF100FB0311DFF8DC814FF0E0204FF473
:10AB30007A7E4FF0100A4FF0010BD8F80430C3F3BF
:10AB40000803002B40F08683EFF31183002B40F0C5
:10AB50008183D4F88025D0F818C0D4F880359A4283
:10AB6000F7D1D4F854399C45F3D8D4F850990EFB5A
:10AB700009F3A3EB0C03B3FBF9F30EFB02335B1AEF
:10AB8000B3F57A7FD9D3019B032B01F09F810DF19F
:10AB90000F030993002305938DF81C3008930A9343
:10ABA0000D9310931293012306930B938DF830307D
:10ABB0008DF8443040238DF80E309B2300228DF811
:10ABC0000F3004A900233846CDE90E23049611F076
:10ABD000A5F92B695A6A002A00F08C80974208D0A8
:10ABE000FEE71A6A002A3FF47AAF1A6A002AF8D1FF
:10ABF00075E71A6A002AFCD1424B5B68C3F308036D
:10AC0000002B41F03F81EFF31183002B41F03A819B
:10AC10004FF0E020D4F880358169D4F88025934244
:10AC2000F8D1D4F854299142F4D8D4F850C94FF44B
:10AC30007A7000FB0CF2511AB1FBFCF100FB03111E
:10AC4000DFF8C0804FF0E0204FF47A7E4FF0100A1A
:10AC50004FF0010BD8F80430C3F30803002B40F089
:10AC60002583EFF31183002B40F02083D4F8802557
:10AC7000D0F818C0D4F880359A42F7D1D4F85439B6
:10AC80009C45F3D8D4F850990EFB09F3A3EB0C03C1
:10AC9000B3FBF9F30EFB02335B1AB3F57A7FD9D31A
:10ACA0000DF10F030993002305938DF81C300893D1
:10ACB0000A930D9310931293012306930B938DF82F
:10ACC00030308DF8443041238DF80E3003230022BC
:10ACD0008DF80F3004A900233846CDE90E230496E1
:10ACE00011F01CF92B695A6A002A00F09C809742E7
:10ACF0000AD0FEE71A6A002A3FF47EAF1A6A002AD9
:10AD0000F8D179E700ED00E01A6A002AFCD18E4BF9
:10AD10005B68C3F30803002B41F08181EFF31183DB
:10AD2000002B41F07C814FF0E020D4F88035816920
:10AD3000D4F880259342F8D1D4F854299142F4D81C
:10AD4000D4F850C94FF47A7000FB0CF2511AB1FBE1
:10AD5000FCF100FB0311DFF8F0814FF0E0204FF42D
:10AD60007A7E4FF0100A4FF0010BD8F80430C3F38D
:10AD70000803002B40F08482EFF31183002B40F096
:10AD80007F82D4F88025D0F818C0D4F880359A4254
:10AD9000F7D1D4F854399C45F3D8D4F850990EFB28
:10ADA00009F3A3EB0C03B3FBF9F30EFB02335B1ABD
:10ADB000B3F57A7FD9D394F86539013BDBB2022B26
:10ADC00000F23883614A134493F884321B0163F024
:10ADD0003203DBB28DF80F300DF10F03099300231E
:10ADE00005938DF81C3008930A930D9310931293DA
:10ADF000012306930B938DF830308DF844304223B5
:10AE000000228DF80E3004A900233846CDE90E2328
:10AE1000049611F083F82B695A6A002A00F08C809E
:10AE2000974208D0FEE71A6A002A3FF470AF1A6A08
:10AE3000002AF8D16BE71A6A002AFCD1424B5B6802
:10AE4000C3F30803002B40F06787EFF31183002B57
:10AE500040F062874FF0E020D4F880358169D4F863
:10AE600080259342F8D1D4F854299142F4D8D4F8EB
:10AE700050C94FF47A7000FB0CF2511AB1FBFCF18F
:10AE800000FB0311DFF8C0804FF0E0204FF47A7E22
:10AE90004FF0100A4FF0010BD8F80430C3F3080349
:10AEA000002B40F04782EFF31183002B40F04282E9
:10AEB000D4F88025D0F818C0D4F880359A42F7D15C
:10AEC000D4F854399C45F3D8D4F850990EFB09F3C3
:10AED000A3EB0C03B3FBF9F30EFB02335B1AB3F5E0
:10AEE0007A7FD9D30DF10F030993002305938DF8D1
:10AEF0001C3008930A930D93109312930123069329
:10AF00000B938DF830308DF8443043238DF80E309C
:10AF1000082300228DF80F3004A900233846CDE91C
:10AF20000E23049610F0FAFF2B695A6A002A00F0EB
:10AF3000968097420CD0FEE71A6A002A3FF47EAF53
:10AF40001A6A002AF8D179E700ED00E0F8DB05087D
:10AF50001A6A002AFCD1BE4B5B68C3F30803002BBE
:10AF600040F01886EFF31183002B40F013864FF06A
:10AF7000E020D4F880358169D4F880259342F8D157
:10AF8000D4F854298A42F4D3D4F850C94FF47A70D3
:10AF900000FB0CF2511AB1FBFCF100FB0311DFF8CE
:10AFA000B0824FF0E0204FF47A7E4FF0100A4FF05D
:10AFB000010BD8F80430C3F30803002B40F03181B3
:10AFC000EFF31183002B40F02C81D4F88035D0F8BA
:10AFD00018C0D4F880259A42F7D1D4F85439634583
:10AFE000F3D3D4F850990EFB09F3A3EB0C03B3FB96
:10AFF000F9F30EFB02335B1AB3F57A7FD9D3019BC9
:10B000000496032B0DF10F0309934FF000030593F2
:10B010008DF81C3008930A930D93109312934FF000
:10B02000010306930B938DF830308DF844304FF0C8
:10B0300058038DF80E3000F02485042300228DF88B
:10B040000F3004A900233846CDE90E2310F066FF27
:10B050002B695A6A5AB1974200F03984FEE71A6A9E
:10B06000002A3FF478AF1A6A002AF8D173E71A6A07
:10B07000002AFCD1764B5B68C3F30803002B40F039
:10B080000D84EFF31183002B40F008844FF0E02093
:10B09000D4F880258169D4F880359342F8D1D4F86A
:10B0A00054298A42F4D3D4F850C9DFF8A4E14FF40C
:10B0B0007A7000FB0CF2521A4FF0100AB2FBFCF24D
:10B0C0004FF0010B00FB03224FF0E02C4FF47A709D
:10B0D000DEF80430C3F30803002B40F05184EFF393
:10B0E0001183002B40F04C84D4F88015DCF81880D4
:10B0F000D4F880359942F7D1D4F854399845F3D82B
:10B10000D4F8509900FB09F3A3EB0803B3FBF9F360
:10B1100000FB01339B1AB3F57A7FD9D30DF10F03EE
:10B120000993002305938DF81C3008930A930D931F
:10B1300010931293012306930B938DF830308DF802
:10B14000443053238DF80E300A2300228DF80F303F
:10B1500004A900233846CDE90E23049610F0DEFE44
:10B160002B695A6A002A00F0E881974200F0648156
:10B17000FEE7EFF311878AF31288D2F818E013691B
:10B18000D80304D50123C4F84C39D2F818E0D4F818
:10B190008035D4F84C09FFB287F31188D4F8507980
:10B1A00018440CFB07F3A3EB0E03B3FBF7F30CFB04
:10B1B000003355E4EFF311878AF31288D2F818E0D0
:10B1C0001369D80304D50123C4F84C39D2F818E028
:10B1D000D4F88035D4F84C09FFB287F31188D4F83D
:10B1E000507918440CFB07F3A3EB0E03B3FBF7F302
:10B1F0000CFB0033FFF78FBAEFF3118189F312884C
:10B2000093691069C70344BFC4F84CB99369D4F873
:10B210008005D4F84C79C9B281F311880744FFF74F
:10B22000C0B9EFF311838AF31288D0F818C002690D
:10B23000D20303D5C4F84CB9D0F818C0D4F880258F
:10B24000D4F84C99DBB283F311884A44C9E600BFB5
:10B2500000ED00E0EFF311838AF31288D0F818C0F4
:10B260000269D20303D5C4F84CB9D0F818C0D4F899
:10B270008025D4F84C99DBB283F311884A4474E4F6
:10B28000EFF311838AF31288D0F818C00269D20351
:10B2900003D5C4F84CB9D0F818C0D4F88025D4F838
:10B2A0004C99DBB283F311884A4476E5EFF31183BE
:10B2B0008AF31288D0F818C00269D20303D5C4F803
:10B2C0004CB9D0F818C0D4F88025D4F84C99DBB22A
:10B2D00083F311884A44D5E4EFF311838AF312888B
:10B2E000D0F818C00269D20303D5C4F84CB9D0F81D
:10B2F00018C0D4F88025D4F84C99DBB283F31188B8
:10B300004A44FFF792BAEFF311828AF31288D0F819
:10B3100018C00169C90303D5C4F84CB9D0F818C0E6
:10B32000D4F88015D4F84C99D2B282F311884944EC
:10B33000FFF793B9EFF311838AF31288D0F818C09E
:10B340000269D20303D5C4F84CB9D0F818C0D4F8B8
:10B350008025D4F84C99DBB283F311884A44B3E5D5
:10B36000EFF311838AF31288D0F818C00269D20370
:10B3700003D5C4F84CB9D0F818C0D4F88025D4F857
:10B380004C99DBB283F311884A44FFF7D6BAEFF346
:10B3900011808AF3128897691369DB0303D50123AF
:10B3A000C4F84C399769D4F88035D4F84C19C0B238
:10B3B00080F31188D4F850090B440CFB00F1C91B31
:10B3C000B1FBF0F10CFB0311FFF72ABBEFF3118186
:10B3D00089F3128890691369DB0344BFC4F84CB940
:10B3E0009069D4F88035D4F84C79C9B281F31188CA
:10B3F0003B44FFF7B5B8EFF311808AF312889769E1
:10B400001369DB0303D50123C4F84C399769D4F8D9
:10B410008035D4F84C19C0B280F31188D4F85009A3
:10B420000B440CFB00F1C91BB1FBF0F10CFB031149
:10B43000FFF751B9CD23CDE41A6A002AFCD1874B1E
:10B440005B68C3F30803002B40F0B282EFF3118373
:10B45000002B40F0AD824FF0E020D4F880258169C8
:10B46000D4F880359342F8D1D4F854299142F4D8D5
:10B47000D4F850C94FF47A7000FB0CF2511AB1FBAA
:10B48000FCF100FB0311DFF8D4814FF0E0204FF412
:10B490007A7E4FF0100A4FF0010BD8F80430C3F356
:10B4A0000803002B40F04882EFF31183002B40F09B
:10B4B0004382D4F88025D0F818C0D4F880359A4259
:10B4C000F7D1D4F854399C45F3D8D4F850990EFBF1
:10B4D00009F3A3EB0C03B3FBF9F30EFB02335B1A86
:10B4E000B3F57A7FD9D30DF10F03099300230593A8
:10B4F0008DF81C3008930A930D9310931293012337
:10B5000006930B938DF830308DF844307C238DF802
:10B510000E30022300228DF80F3004A90023384694
:10B52000CDE90E23049610F0F9FC2B695A6A002A23
:10B5300000F08C80974208D0FEE71A6A002A3FF498
:10B540007EAF1A6A002AF8D179E71A6A002AFCD17C
:10B55000424B5B68C3F30803002B40F06F82EFF3AC
:10B560001183002B40F06A824FF0E020D4F8802550
:10B570008169D4F880359342F8D1D4F854299142A6
:10B58000F4D8D4F850C94FF47A7000FB0CF2511A79
:10B59000B1FBFCF100FB0311DFF8C0804FF0E020AD
:10B5A0004FF47A7E4FF0100A4FF0010BD8F80430B8
:10B5B000C3F30803002B40F0A981EFF31183002BA4
:10B5C00040F0A481D4F88025D0F818C0D4F8803594
:10B5D0009A42F7D1D4F854399C45F3D8D4F850990D
:10B5E0000EFB09F3A3EB0C03B3FBF9F30EFB0233E1
:10B5F0005B1AB3F57A7FD9D30DF10F0309930023BA
:10B6000005938DF81C3008930A930D9310931293B1
:10B61000012306930B938DF830308DF844307D2351
:10B620008DF80E300E2300228DF80F3004A9002370
:10B630003846CDE90E23049610F070FC2B695A6A47
:10B64000002A00F0238197420AD0FEE71A6A002AF6
:10B650003FF47EAF1A6A002AF8D179E700ED00E0E6
:10B660001A6A002AFCD1BF4B5B68C3F30803002BA6
:10B6700040F0C181EFF31183002B40F0BC814FF00B
:10B68000E020D4F880358169D4F880259342F8D140
:10B69000D4F854299142F4D8D4F850C94FF47A70B0
:10B6A00000FB0CF2511AB1FBFCF100FB0311DFF8B7
:10B6B000B4824FF0E0204FF47A7E4FF0100A4FF042
:10B6C000010BD8F80430C3F30803002B40F00881C5
:10B6D000EFF31183002B40F00381D4F88035D0F8CC
:10B6E00018C0D4F880259A42F7D1D4F854399C4533
:10B6F000F3D8D4F850990EFB09F3A3EB0C03B3FB7A
:10B70000F9F30EFB02335B1AB3F57A7FD9D3019BB1
:10B71000032B00F0638295F82131002B00F092801A
:10B720001E09013E052E03F00F0300F2E5878E4F40
:10B7300007EB4602B2F8000140FA03F2D20740F1EB
:10B74000DB87012202FA03F3013B18403E4450F02C
:10B750001DFD96F80C81DFF824928449804409EBA2
:10B76000C806B388B3FA83F2202A4FF02603F38089
:10B77000E960C2F11F0165D07B1804EB810193F8E9
:10B78000887205F10C03C1F888394FF00043D340AB
:10B7900005D0774A116821EA030111605361002145
:10B7A000304611F031F859F8383003F13F4303F5D2
:10B7B0007E03C3F38722B388B3FA83F3C3F11F0078
:10B7C00000F0FC0101F1804101F59C3100F0030023
:10B7D000D1F808C080004FF00F0E82400EFA00F042
:10B7E0002CEA00008860886802438A60604A4FF053
:10B7F0000048116828FA03F321EA03011160516837
:10B8000021EA030151605B49D1F8000C1843C1F8EB
:10B81000000C906820EA03009060D06820EA0300E2
:10B82000D060D1F8082C04EB070C1A43C1F8082C9F
:10B830009CF8C829F02A00F24F871BB14C490A68CE
:10B8400013430B6022684C4BB3EB920F80F041879F
:10B85000B3EBD20F80F03A87B3EB121F80F0508722
:10B86000B3EB521F80F04F87B3EB921F80F04E87EF
:10B87000B3EBD21F80F04D87B3EB122F34BF4FF4E0
:10B8800080738023AB8215B0BDE8F08F1A6A002A5E
:10B890003FF4E9AE1A6A002AF8D1E4E6EFF3118228
:10B8A000102383F312884FF0E02399691869C003CD
:10B8B00003D50121C4F84C199969D4F88005D4F84E
:10B8C0004C39D2B282F311880344FFF7ECBB1A6AF9
:10B8D000002A3FF4CFAB1A6A002AF8D1FFF7CABB9F
:10B8E000EFF311838AF31288D0F818C00269D203EB
:10B8F00003D5C4F84CB9D0F818C0D4F88025D4F8D2
:10B900004C99DBB283F311884A44F2E6EFF31183DA
:10B910008AF31288D0F818C00269D20303D5C4F89C
:10B920004CB9D0F818C0D4F88025D4F84C99DBB2C3
:10B9300083F311884A4451E6EFF311838AF31288A6
:10B94000D0F818C00269D20303D5C4F84CB9D0F8B6
:10B9500018C0D4F88025D4F84C99DBB283F3118851
:10B960004A44B2E500ED00E0F8DB05085DA10008FF
:10B97000003C01400030014080969800541F002098
:10B98000EFF311838AF31288DCF81880DCF81010CA
:10B99000C90303D5C4F84CB9DCF81880D4F8801575
:10B9A000D4F84C99DBB283F311884944FFF7A8BB64
:10B9B000EFF31182102383F312884FF0E02398698C
:10B9C0001969C90303D50121C4F84C199869D4F841
:10B9D0008015D4F84C39D2B282F31188D4F850C90A
:10B9E0004FF47A720B4402FB0CF1091AB1FBFCF123
:10B9F00002FB031147E5EFF31182102383F3128852
:10BA00004FF0E02398691969C90303D50121C4F8EF
:10BA10004C199869D4F88015D4F84C39D2B282F315
:10BA20001188D4F850C94FF47A720B4402FB0CF120
:10BA3000091AB1FBFCF102FB031138E6EFF31182A6
:10BA4000102383F312884FF0E02398691969C90322
:10BA500003D50121C4F84C199869D4F88015D4F89D
:10BA60004C39D2B282F31188D4F850C94FF47A72AB
:10BA70000B4402FB0CF1091AB1FBFCF102FB0311B0
:10BA80008AE5022300228DF80F3004A900233846EE
:10BA9000CDE90E2310F042FA2B695A6A002A72D0BF
:10BAA000974200D0FEE71A6A002AFCD1BE4B5B68C1
:10BAB000C3F30803002B40F00785EFF31183002B3D
:10BAC00040F002854FF0E020D4F880358169D4F849
:10BAD00080259342F8D1D4F854298A42F4D3D4F87B
:10BAE00050C9DFF8C4824FF47A7000FB0CF2521A8E
:10BAF000B2FBFCF200FB0322D8F80430C3F30803C6
:10BB00004FF0E0204FF47A7C4FF0100A4FF0010B19
:10BB10001BBBEFF3118303BBD4F88035D0F818E0DA
:10BB2000D4F880159942F7D1D4F854397345F3D33A
:10BB3000D4F850990CFB09F3A3EB0E03B3FBF9F314
:10BB40000CFB01339B1AB3F57A7FBFF4E7AAD8F850
:10BB50000430C3F30803002BDBD0EFF311838AF327
:10BB60001288D0F818E00169C90303D5C4F84CB9AC
:10BB7000D0F818E0D4F88015D4F84C99DBB283F3F0
:10BB800011884944D4E71A6A002A8FD01A6A002A19
:10BB9000F9D18BE7EFF31182102383F312884FF072
:10BBA000E02398691969C90303D50121C4F84C1928
:10BBB0009869D4F88015D4F84C39D2B282F3118840
:10BBC000D4F850C94FF47A720B4402FB0CF1091AF5
:10BBD000B1FBFCF102FB0311FFF7E1B90DF10F031B
:10BBE0000993002305938DF81C3008930A930D9355
:10BBF00010931293012306930B938DF830308DF838
:10BC000044307E238DF80E30B02300228DF80F30A3
:10BC100004A900233846CDE90E23049610F07EF9DE
:10BC20002B695A6A1AB1974200F0AF84FEE71A6A8C
:10BC3000002AFCD15C4B5B68C3F30803002B40F087
:10BC4000F584EFF31183002B40F0F0844FF0E020F7
:10BC5000D4F880358269D4F880158B42F8D1D4F8B5
:10BC600054198A42F4D8D4F850094FF47A7101FB80
:10BC700000F6B61AB6FBF0F601FB0366DFF8288182
:10BC8000D8F80430C3F308034FF0E0214FF47A777B
:10BC90004FF0100E4FF0010C0BBBEFF31183F3B913
:10BCA000D4F880258869D4F880359342F8D1D4F847
:10BCB00054299042F4D8D4F8509907FB09F2121A8B
:10BCC000B2FBF9F207FB03239B1BB3F57A7FBFF4AA
:10BCD00022ADD8F80430C3F30803002BDDD0EFF316
:10BCE00011838EF3128888690A69D20302D5C4F8D9
:10BCF0004CC98869D4F88095D4F84C29DBB283F319
:10BD000011884A44D4F8509907FB09F31B1AB3FB76
:10BD1000F9F307FB0233D7E7EFF31182102383F324
:10BD200012884FF0E02398691969C90303D50121EE
:10BD3000C4F84C199869D4F88015D4F84C39D2B2AB
:10BD400082F31188D4F850C94FF47A720B4402FB85
:10BD50000CF1091AB1FBFCF102FB0311FFF792B8D9
:10BD6000EFF31182102383F312884FF0E0239869D8
:10BD70001969C90303D50121C4F84C199869D4F88D
:10BD80008015D4F84C39D2B282F31188D4F850C956
:10BD90004FF47A720B4402FB0CF1091AB1FBFCF16F
:10BDA00002FB0311FEF7BFBE00ED00E0EFF31182CE
:10BDB000102383F312884FF0E02398691969C903AF
:10BDC00003D50121C4F84C199869D4F88015D4F82A
:10BDD0004C39D2B282F31188D4F850C94FF47A7238
:10BDE0000B4402FB0CF1091AB1FBFCF102FB03113D
:10BDF000FEF781BDEFF31182102383F312884FF019
:10BE0000E02398691969C90303D50121C4F84C19C5
:10BE10009869D4F88015D4F84C39D2B282F31188DD
:10BE2000D4F850C94FF47A720B4402FB0CF1091A92
:10BE3000B1FBFCF102FB0311FEF7D5BCEFF311825D
:10BE4000102383F312884FF0E02399691869C00327
:10BE500003D50121C4F84C199969D4F88005D4F8A8
:10BE60004C39D2B282F31188D4F850C91A184FF461
:10BE70007A7000FB0CF35B1AB3FBFCF300FB02339C
:10BE8000FEF7C9BBEFF31182102383F312884FF042
:10BE9000E02398691969C90303D50121C4F84C1935
:10BEA0009869D4F88015D4F84C39D2B282F311884D
:10BEB000D4F850C94FF47A720B4402FB0CF1091A02
:10BEC000B1FBFCF102FB0311FEF7BABE0DF10F034B
:10BED000099300238DF80F3005938DF81C300893DB
:10BEE0000A930D9310931293012306930B938DF8ED
:10BEF00030308DF84430482300228DF80E3004A9EC
:10BF000000233846CDE90E23049610F007F82B697C
:10BF10005A6A1AB1974200F0D183FEE71A6A002AE2
:10BF2000FCD1A34B5B68C3F30803002B40F03683BE
:10BF3000EFF31183002B40F031834FF0E020D4F871
:10BF400080358269D4F880158B42F8D1D4F8541921
:10BF50008A42F4D8D4F850094FF47A7101FB00FCFE
:10BF6000ACEB020CBCFBF0FC01FB03CCDFF8408225
:10BF70004FF0E0224FF47A7E4FF0100A4FF0010BA1
:10BF8000D8F80430C3F30803002B40F0F480EFF33B
:10BF90001183002B40F0EF80D4F880359169D4F8FC
:10BFA00080058342F8D1D4F854098142F4D8D4F8FA
:10BFB00050990EFB09F0411AB1FBF9F10EFB031386
:10BFC000A3EB0C03B3F57A7FDAD30DF10F030993DA
:10BFD000002305938DF81C3008930A930D9310935A
:10BFE0001293012306930B938DF830308DF8443073
:10BFF00049238DF80E30802300228DF80F3004A9DC
:10C0000000233846CDE90E2304960FF087FF2B69F5
:10C010005A6A002A00F0A780974224D0FEE7EFF387
:10C020001182102383F312884FF0E0239869196975
:10C03000C90303D50121C4F84C199869D4F88015B7
:10C04000D4F84C39D2B282F31188D4F850C94FF4E5
:10C050007A720B4402FB0CF1091AB1FBFCF102FBF2
:10C060000311FEF778BE1A6A002AFCD1504B5B68B8
:10C07000C3F30803002B40F0FD82EFF31183002B84
:10C0800040F0F8824FF0E020D4F880358269D4F88F
:10C0900080158B42F8D1D4F854198A42F4D8D4F8D8
:10C0A00050094FF47A7101FB00FCACEB020CBCFBB5
:10C0B000F0FC01FB03CCDFF8F8804FF0E0224FF4F6
:10C0C0007A7E4FF0100A4FF0010BD8F80430C3F31A
:10C0D0000803002B40F09F81EFF31183002B40F009
:10C0E0009A81D4F880359169D4F880058342F8D1DB
:10C0F000D4F854098142F4D8D4F850990EFB09F0D1
:10C10000411AB1FBF9F10EFB0313A3EB0C03B3F5DA
:10C110007A7FDAD30DF10F03099300238DF80F30E6
:10C1200005938DF81C3008930A930D931093129386
:10C13000012306930B938DF830308DF8443045235E
:10C1400000228DF80E3004A900233846CDE90E23D5
:10C1500004960FF0E3FE2B695A6A002A00F053811F
:10C16000974227D0FEE71A6A002A3FF47FAF1A6A87
:10C17000002AF8D17AE7EFF311838AF312889069E5
:10C180001169C90302D5C4F84CB99069D4F8801577
:10C19000D4F84C99DBB283F311884944D4F8509910
:10C1A0000EFB09F31B1AB3FBF9F30EFB013307E790
:10C1B00000ED00E01A6A002AFCD1C24B5B68C3F3B1
:10C1C0000803002B40F00E82EFF31183002B40F0A8
:10C1D00009824FF0E020D4F880358269D4F88015C8
:10C1E0008B42F8D1D4F854198A42F4D8D4F85009C3
:10C1F0004FF47A7101FB00FCACEB020CBCFBF0FCD1
:10C2000001FB03CCDFF8BC824FF0E0224FF47A7ED2
:10C210004FF0100A4FF0010BD8F80430C3F30803B5
:10C22000002B40F03281EFF31183002B40F02D8181
:10C23000D4F880359169D4F880058342F8D1D4F8D8
:10C2400054098142F4D8D4F850990EFB09F0411AF0
:10C25000B1FBF9F10EFB0313A3EB0C03B3F57A7FEB
:10C26000DAD30622462138460FF04AFF954B5B6829
:10C27000C3F30803002B40F06481EFF31183002B1C
:10C2800040F05F814FF0E020D4F880358269D4F827
:10C2900080158B42F8D1D4F854198A42F4D8D4F8D6
:10C2A00050094FF47A7101FB00FCACEB020CBCFBB3
:10C2B000F0FC01FB03CCDFF80C824FF0E0224FF4DE
:10C2C0007A7E4FF0100A4FF0010BD8F80430C3F318
:10C2D0000803002B40F0BC80EFF31183002B40F0EB
:10C2E000B780D4F880359169D4F880058342F8D1BD
:10C2F000D4F854098142F4D8D4F850990EFB09F0CF
:10C30000411AB1FBF9F10EFB0313A3EB0C03B3F5D8
:10C310007A7FDAD30022472138460FF0F1FE694BCD
:10C320005B68C3F30803002B40F0E780EFF3118351
:10C33000002B40F0E2804FF0E020D4F88035826995
:10C34000D4F880158B42F8D1D4F854198A42F4D825
:10C35000D4F850094FF47A7101FB00FCACEB020CED
:10C36000BCFBF0FC01FB03CCDFF85881D8F80430AB
:10C37000C3F308034FF0E0224FF47A7E4FF0100A27
:10C380004FF0010B13BBEFF31183FBB9D4F88035E9
:10C390009169D4F880058342F8D1D4F854098142D8
:10C3A000F4D8D4F850990EFB09F0411AB1FBF9F119
:10C3B0000EFB0313A3EB0C03B3F57A7FBEF4E7ABDC
:10C3C000D8F80430C3F30803002BDCD0EFF311835B
:10C3D0008AF3128890691169C90302D5C4F84CB96F
:10C3E0009069D4F88015D4F84C99DBB283F31188A6
:10C3F0004944D4F850990EFB09F31B1AB3FBF9F327
:10C400000EFB0133D6E71A6A002A3FF4D6AE1A6A49
:10C41000002AF8D1D1E6EFF311838AF312889069EC
:10C420001169C90302D5C4F84CB99069D4F88015D4
:10C43000D4F84C99DBB283F311884944D4F850996D
:10C440000EFB09F31B1AB3FBF9F30EFB01335CE699
:10C45000EFF311838AF3128890691169C90302D539
:10C46000C4F84CB99069D4F88015D4F84C99DBB273
:10C4700083F311884944D4F850990EFB09F31B1A31
:10C48000B3FBF9F30EFB01333FE7EFF311838AF3BC
:10C49000128890691169C90302D5C4F84CB9906932
:10C4A000D4F88015D4F84C99DBB283F31188494451
:10C4B000D4F850990EFB09F31B1AB3FBF9F30EFBEA
:10C4C0000133C9E600ED00E0EFF31182102383F39E
:10C4D00012884FF0E02399691869C00303D5012140
:10C4E000C4F84C199969D4F88005D4F84C39D2B203
:10C4F00082F311880344FFF7F2BAEFF3118210239D
:10C5000083F312884FF0E02399691869C00303D5BB
:10C510000121C4F84C199969D4F88005D4F84C3934
:10C52000D2B282F311880344D4F850094FF47A72DE
:10C5300002FB00FCACEB010CBCFBF0FC02FB03CCEF
:10C5400012E7EFF31182102383F312884FF0E023F8
:10C5500099691869C00303D50121C4F84C19996978
:10C56000D4F88005D4F84C39D2B282F31188034450
:10C57000D4F850094FF47A7202FB00FCACEB010CCA
:10C58000BCFBF0FC02FB03CC95E61A6A002A3FF4E0
:10C5900051AB1A6A002AF8D1FFF74CBBEFF31182B6
:10C5A000102383F312884FF0E02399691869C003C0
:10C5B00003D50121C4F84C199969D4F88005D4F841
:10C5C0004C39D2B282F311880344D4F850094FF4A5
:10C5D0007A7202FB00FCACEB010CBCFBF0FC02FB32
:10C5E00003CCC3E4EFF31182102383F312884FF0DE
:10C5F000E02399691869C00303D50121C4F84C19D7
:10C600009969D4F88005D4F84C39D2B282F31188F4
:10C610000344D4F850094FF47A7202FB00FCACEBEF
:10C62000010CBCFBF0FC02FB03CCEBE5EFF3118249
:10C63000102383F312884FF0E02399691869C0032F
:10C6400003D50121C4F84C199969D4F88065D4F850
:10C650004C39D2B282F31188D4F850094FF47A726F
:10C66000334402FB00F6761AB6FBF0F602FB0366D3
:10C67000FFF704BBEFF31182102383F312884FF00E
:10C68000E02399691869C00303D50121C4F84C1946
:10C690009969D4F88005D4F84C39D2B282F3118864
:10C6A0000344D4F850094FF47A7202FB00FCACEB5F
:10C6B000010CBCFBF0FC02FB03CCFCE41A6A002A70
:10C6C0003FF42FAC1A6A002AF8D12AE40423FFF7BA
:10C6D000D9B80223FFF7D6B80F4BD85DF0238CF8FA
:10C6E000C839002203214DF0C1FFB388B3FA83F3A8
:10C6F00028FA03F3FFF7A1B8084BEB60FFF7A2B8E5
:10C700000823FFF7BFB81023FFF7BCB82023FFF7BB
:10C71000B9B84023FFF7B6B8084F06085DA1000876
:10C720002DE9F041AB4C94F8CF39012B94B000F0D7
:10C730009D81022B00F03D81002B00F05781A64D1A
:10C7400095F83E305B060DF10E060DF10F0804A9B9
:10C7500004F51D6740F138814FF4F073A5F84030BF
:10C760000023CDE90833CDE90A3305930D93012366
:10C7700085F842308DF81C308DF83030974BC4F876
:10C78000683A03F10213C4F86C3A03F10213C4F8D7
:10C79000703A03F10213C4F8743A03F10213C4F8B7
:10C7A000783A03F102138E48C4F87C3A03F102137D
:10C7B000C4F8803A03F102130490C4F8843A98381C
:10C7C0002023069301910FF0A9FBD4F8D0390199E9
:10C7D0005A6A002A2FD0BA4200D0FEE71A6A002A0D
:10C7E000FCD100238DF80E3005938DF81C30089392
:10C7F0000A930D9310931293012306930B938DF8D4
:10C8000030308DF8443095F83E308DF80F300022EE
:10C81000002374480191CDE90E230496CDF82480BD
:10C820000FF07CFBD4F8D03901995A6A002A37D02E
:10C83000BA4207D0FEE71A6A002AD2D01A6A002A42
:10C84000F9D1CEE71A6A002AFCD1002305938DF8AE
:10C850001C3008930A930D931093129301230693AF
:10C860000B938DF830308DF8443094F8883A8DF879
:10C870000F30022300228DF80E305A480191002318
:10C88000CDE90E230496CDF824800FF047FBD4F8B1
:10C89000D03901995A6A002A37D0BA4207D0FEE748
:10C8A0001A6A002AD1D01A6A002AF9D1CDE71A6A89
:10C8B000002AFCD1002305938DF81C3008930A93BD
:10C8C0000D9310931293012306930B938DF8303040
:10C8D0008DF8443094F8893A8DF80F300323002204
:10C8E0008DF80E303F4801910023CDE90E230496C8
:10C8F000CDF824800FF012FBD4F8D03901995A6A90
:10C90000002A3CD0BA4207D0FEE71A6A002AD1D0EA
:10C910001A6A002AF9D1CDE71A6A002AFCD194F8E4
:10C920008A3A002B53D0012B00F0B380032B14BFA5
:10C93000C723F7238DF80F30002305938DF81C30A3
:10C9400008930A930D9310931293012300228DF8FC
:10C950000E3006930B938DF830308DF8443021481B
:10C9600004960023CDE90E23CDF824800FF0D6FAEB
:10C97000D4F8D0395A6AAAB1BA4207D0FEE71A6A87
:10C98000002ACCD01A6A002AF9D1C8E71A6A002A0C
:10C99000FCD1B5F840201448002114B0BDE8F041A6
:10C9A00051F0D7B81A6A002AF3D01A6A002AF9D1CE
:10C9B000EFE7094D082385F83E300DF10E060DF125
:10C9C0000F0804A904F51D674FF4C373C6E6472397
:10C9D000B0E700BF081900208801002010011101F4
:10C9E00070230020D8220020942300200122A021BF
:10C9F0000DF10E0604F51D67CDE90463CDE908339A
:10CA00008DF80E10069204A98DF81C300B928DF84B
:10CA100030208DF844200D930022109312930DF1D5
:10CA20000F0800233846CDE90E230191CDF8288068
:10CA30000FF074FAD4F8D03901995A6A12B1BA4297
:10CA400020D0FEE71A6A002AFCD19DF80F30144D61
:10CA500003F00602022A03D003F00503012B1AD0CB
:10CA6000082385F83E304FF4C37377E60C4D482316
:10CA700085F83E300DF10E060DF10F0804A904F5FE
:10CA80001D6769E61A6A002ADFD01A6A002AF9D1FE
:10CA9000DBE787234EE7482385F83E305CE600BF9E
:10CAA000880100200A4608B5054920B9054844F028
:10CAB00007FF034808BD044844F002FF004808BDD2
:10CAC00074250020884E0608B04E060810B5044CA8
:10CAD00004480A46214644F0F3FE204610BD00BF3C
:10CAE00074250020D84E060810B5044C04480A46A8
:10CAF000214644F0E5FE204610BD00BF742500200D
:10CB0000EC4E060810B5044C04480A46214644F091
:10CB1000D7FE204610BD00BF74250020F84E060841
:10CB200010B5104CD4F86C2D94F86B3D2AB103F07D
:10CB300001039BB9136892881A834BF05FFD02E0F2
:10CB40005B69984720B9D4F87C35002BF8D1FEE713
:10CB5000D4F88035C4F88435002010BD136892885D
:10CB60005A83EAE708190020BFF34F8F0549064BA7
:10CB7000CA6802F4E0621343CB60BFF34F8F00BF7B
:10CB8000FDE700BF00ED00E00400FA051648174A73
:10CB9000174938B5174C184D121A50F077FFD4F8D2
:10CBA0008820164B164842F47002C4F888201A6890
:10CBB000002142F001021A6099601A6822F0847222
:10CBC00022F480321A6058601A6822F480221A60B7
:10CBD0000C4AD960521B28460B4950F057FFA560FC
:10CBE000BDE83840FBF70CBA00000010040000104C
:10CBF000E3F7060800ED00E00000002000380240E6
:10CC00001030002488010020000000082DE9F041C8
:10CC1000CB781BB900263046BDE8F08100F1100446
:10CC20000D468046897820460FF00AF9064600280E
:10CC3000F0D0E87810F000FCC8F818002B78013329
:10CC4000DBB210B1C3712223837109210FF0DCFD27
:10CC5000D8F818001A4F0FF0EDF8D7F88035632B8D
:10CC6000FBD918480FF0B6F8A8F814002046FDF7D5
:10CC7000FBF80446E0B9E87810F0DEFBD7F8787DE1
:10CC8000002F0646C6DDDFF8408002E00134BC42DA
:10CC9000C0D004EB440518F8050010F0CDFB864227
:10CCA000F4D1214608EB050010F00AFC0026B2E79B
:10CCB000D8F8100088F8D8404EF058FCABE700BF19
:10CCC0000819002040420F008426002043680B4AC8
:10CCD00023F0407323F4807343F4807343608368CC
:10CCE0001A4042F002028260C36A0139CAB223F4D8
:10CCF000700141EA0251C162704700BFFDF7FFC0F9
:10CD0000704700BF0020FBF7C1B900BF0120FBF74F
:10CD1000BDB900BF0220FBF7B9B900BF431C00F04A
:10CD200038812DE9F04FDFF898A300EB80030AEB80
:10CD3000C30287B0D2F80480810005460191DB0070
:10CD4000B8F1000F04D0D468002C4CD0A17911B1F7
:10CD500007B0BDE8F08FD2F81090B9F1000F00F0E5
:10CD6000478199F80620002AF2D118330AF1040607
:10CD7000F018D8F80470F250691CC0E9012215239C
:10CD8000C260C9B2A3711623E17189F8063089F82F
:10CD9000071098F818004CF045FDBB88A28823F4D2
:10CDA00040731B041B0CBB8023681A83D9F8003026
:10CDB000B9F804201A83112120460FF025FD112116
:10CDC00048460FF021FD09264FF0330B24B12268AD
:10CDD000A188106901422DD1BBF1010B00F0D38075
:10CDE0004DF08CFBF2E7D2F81090B9F1000F00F093
:10CDF000E88099F80620002AAAD118330AF1040124
:10CE0000CA18D8F80470CC50C2E901441623D46083
:10CE100089F806306B1C89F8073098F818004CF038
:10CE200001FDBB8823F440731B041B0CBB80BDE7D2
:10CE30002268A18851834DF0BDFB2368A2881A8324
:10CE40004DF0B8FB013EBFD1002C00F0EF8023680D
:10CE5000A2885A834DF0AEFBB9F1000F00F00B81B0
:10CE6000D9F80030B9F804205A834DF0A3FB2368A9
:10CE7000A2881A834DF09EFBD9F80030B9F804203F
:10CE80001A83019B20465C190AEBC404A37D227D12
:10CE9000002B14BF322112210EF0C0FDA37D627D54
:10CEA000002B14BF3221122148460EF0B7FD7E4BF5
:10CEB0009F4200F0CA807D4B9F4200F0D1807C4BA6
:10CEC0009F4200F0E080019B2B440AEBC30A4FF421
:10CED0007A73BAF8184003FB04F4BB8823F4407358
:10CEE0001B041B0CBB803B889BB243F001033B80BF
:10CEF000BD8802A844F0DAF925F03F0504986D4B8F
:10CF00002D04A3FB00232D0C45EA9345BD803A88F0
:10CF100022F001021204120C3A80674A990C9442E2
:10CF20000B4637DC6200B0FBF2F292B20133042A06
:10CF300038BF04223B84BA833B889BB243F0010391
:10CF40003B803B8823F4816323F002031B041B0C0A
:10CF50004FF4804143F480633B8039813B8823F068
:10CF600080031B041B0C00223B8098F81A0011461A
:10CF70004DF07CFB002298F81900114607B0BDE87F
:10CF8000F04F4DF073BB002C7FF452AF4DF012FB0D
:10CF900056E7704704EB4404B0FBF4F082B2C0F3F0
:10CFA0000B0008B942F001024FF4967301FB03F342
:10CFB0004249A1FB03139B09013342F400423B8425
:10CFC000B9E718330AF10401CA18D8F8047041F817
:10CFD0000390C2E90199C2F80C9098F818004CF03F
:10CFE00021FCBB8823F440731B041B0CBB80E2E6CE
:10CFF00018330AF10401CA18D8F8047041F80390F4
:10D00000C2E901991523C2F80C90A3716B1CE3715E
:10D0100098F818004CF006FCBB88A28823F44073F3
:10D020001B041B0CBB8023681A83C4E64DF0C2FAB4
:10D03000B9F1000F32D0D9F80030B9F804205A8382
:10D040004DF0B8FA4DF0B6FA16E703F5F2331A6A66
:10D0500042F400121A621A6A22F400121A6232E7CB
:10D0600003F5F0331A6A42F480021A621A6A22F453
:10D0700080021A6227E74DF09DFA2368A2881A837E
:10D080004DF098FAFDE603F5EE331A6A42F4000219
:10D090001A621A6A22F400021A6214E74DF08AFA40
:10D0A0004DF088FAEDE600BF005400400058004003
:10D0B000005C004083DE1B43A0860100D34D62105C
:10D0C000081900202DE9F843074610F0CFFFDFF8DC
:10D0D0004C8007EB8709044608EBC90542F20F763E
:10D0E00004E010F0C3FF031BB3420ADC6B7F002B8C
:10D0F000F7D108EBC90898F81C0080F00100BDE8E2
:10D10000F883B8F8AC3D013338469BB2A8F8AC3D83
:10D11000FFF704FE0020BDE8F88300BF08190020D7
:10D1200070B5284D00EB800305EBC30384B05A684B
:10D130005468A28A92B20392039A12F4706F1CBFD1
:10D1400001221A77039B13F4E06F4FEA80060CD19B
:10D15000A38A304423F4706305EBC0051B041B0C49
:10D160000022A3826A7704B070BD238BA38823F4C6
:10D1700080631B041B0CA380039B9A05E8D42388BF
:10D180009B05E5D42388D9050FD52388DA05FCD47F
:10D1900023889BB243F40073238023889B05FCD42F
:10D1A0000190FFF7BBFD0198D2E723889BB243F4BF
:10D1B00000732380A38823F440731B041B0CA380FB
:10D1C000C6E700BF081900200020A9E70120A7E753
:10D1D0000220A5E72DE9F84F304F00EB800407EB64
:10D1E000C404D4F80880B8F1000F04D09A46637FD5
:10D1F00003F0FF0923B14FF000094846BDE8F88F5E
:10D200000E469346054610F031FF0A9B7600F6B2B3
:10D21000C4E909330123A67784F81FB084F821906C
:10D2200084F8223084F820A0637784F81C90B8F842
:10D2300004209105064622D4B8F80030DA0512D44D
:10D2400042F20F7404E010F011FF831BA3421ADCBA
:10D25000B8F800309B05F6D4B8F800309BB243F420
:10D260008073A8F80030B8F804309BB24FF0010981
:10D2700043F44073A8F804304846BDE8F88F994657
:10D280004846BDE8F88FB7F8AC3D01339BB228465D
:10D29000A7F8AC3DFFF742FDAFE700BF081900203B
:10D2A00010B503681C78012C82B00AD0022C05D17D
:10D2B0005A6A0AB1904201D11B6A03B3012002B03D
:10D2C00010BD93F904C012490CEB8C0301EBC303AE
:10D2D0005B7F03F0FF0213B1002002B010BDBCF170
:10D2E000FF3FEBD0BCF1020F10DC01F5AA6301791E
:10D2F000009360460623FFF76DFF2046DFE7054AEF
:10D30000062380210EF040FE0120D8E72046D6E714
:10D3100008190020581E0020F8B5774C04EB0016C1
:10D32000D6F8B03D002B00F094800546070196F832
:10D33000B80D4CF077FA96F8B83D590903F01F0282
:10D3400003294FF0010303FA02F300F09880042947
:10D3500000F0858002297DD0E319013593F8B40DE2
:10D3600010F06AF8EDB2064610B112238371C57150
:10D37000E31993F8B50D10F05FF810B11323C571E0
:10D380008371E31993F8B60D10F056F810B1142319
:10D39000C57183713C444A2194F8B72D30460EF094
:10D3A0003DFB94F8B50D10F047F894F8B72D2A21FD
:10D3B0000EF034FB94F8B60D10F03EF894F8B72D4B
:10D3C0000A210EF02BFBD4F8B02D4C4B9A425BD0C7
:10D3D0004B4B9A4248D04B4B9A4260D04A4B9A42B0
:10D3E00068D04A4B9A4270D0494B9A4278D049490A
:10D3F0009088B1F84640B1F84430B1F84E5023431C
:10D40000B1F848402343B1F84A4020F003002343D9
:10D41000B1F84C400004000C2343B1F85040908018
:10D420002B4310882343B1F85240B1F8541000F454
:10D430004150234303439BB21380938B23F4006337
:10D440001B041B0C9383118213889BB243F040038F
:10D450001380F8BD304A516A0B4353627CE72E4A71
:10D4600011690B43136177E703F50033196A41F43F
:10D4700080411962196A21F480411962B7E7264A8E
:10D48000116A0B43136267E703F58433596A41F469
:10D4900080515962596A21F480515962A7E703F516
:10D4A000FE33196A41F400411962196A21F40041FE
:10D4B00019629CE703F58233596A41F400515962BD
:10D4C000596A21F40051596291E703F56843596A9A
:10D4D00041F480115962596A21F48011596286E73A
:10D4E00003F56443596A41F400115962596A21F401
:10D4F000001159627BE700BF08190020003001408D
:10D5000000380040003C0040003401400050014021
:10D5100000540140880100200038024010B4046922
:10D520008269E468416814604024D460446900233F
:10D530000C31C2E90433C2E90633C2E90833C2E957
:10D540000A33C2E90C3393609363516084B1C269BA
:10D55000E0689363C2E90233C2E90433C2E90633E7
:10D56000C2E90833C2E90A33C2E90C33C2E9000157
:10D570005DF8044B704700BF436800221A60037DCA
:10D580001F2B08D9203B2022016802FA03F343F045
:10D590001803CB6070472022016802FA03F343F0BE
:10D5A00018038B60704700BF0268136A11B1D96914
:10D5B00001B3143330B49C681D689169DDB14FF438
:10D5C000806088618D60104640690C6180B1596847
:10D5D000D369C9B10A464FF480619A6099612243C8
:10D5E00012F0010F14BF00224FF400521A621C61A6
:10D5F00030BC704770478D61054D4FF0FF0C05F84A
:10D6000056CF00688D60DFE7024A9A609961E6E7CD
:10D6100088010020E82600200168F8B5D1E904233C
:10D6200004465568002B49D09861107D5E681F281C
:10D6300031D81768202202FA00F040F01800B860D4
:10D640001A7D1F2A32D91868203A202303FA02F2E1
:10D6500042F01802C26000232B603360336889698E
:10D6600043F010033360284643F004FF236830463C
:10D67000D96943F0FFFE2B68226843F001032B6059
:10D680003368526843F00103336093889BB243F0E0
:10D6900003039380F8BD17682038202202FA00F0B7
:10D6A00040F01800F8601A7D1F2ACCD81868202393
:10D6B00003FA02F242F018028260CCE7137D906117
:10D6C0001F2B1CD81068202202FA03F343F0180322
:10D6D000836000232B602B68896943F010032B6063
:10D6E000284643F0C7FE2B68226843F001035268C6
:10D6F0002B6093889BB243F002039380F8BD1068BF
:10D70000203B202202FA03F343F01803C360E0E752
:10D710002DE9F843DFF800927D4F0646356896F80C
:10D7200088806B68B088012285F828201A8822F04A
:10D7300040021204120C1A802A89824223D01988CE
:10D7400021F0380109044B454FEA114100F0BC803B
:10D75000704A934200F0B8800246B2F5807FA8BFBD
:10D760004FF48072022AB8BF0222002A92FAA2F273
:10D77000B2FA82F208BF4FF0FF32013A41EAC20228
:10D7800092B21A802881317BAA7A8A420CD01A88F8
:10D7900022F003021204120C1A801A8892B2002995
:10D7A00000F08F801A80A9721A8892B242F040026B
:10D7B0001A802A6A9168002900F0A0804FF0000CBE
:10D7C0001432E64652F8100C8E4400EA070120B1EC
:10D7D000B1F1805F23D0696909B352F8140C143297
:10D7E00000EA070110B1B1F1805F18D052F80C1CAB
:10D7F0000CF1010C0029E5D12A7B82B1B8F1000FB0
:10D800000DD0BCF1010F6CD8BEF1070F69D80CEB3D
:10D810008C0189002A6A11440A7B002A61D02A6A95
:10D820009268002A52D000220AB1127B22B1B2685B
:10D8300012B1116892884A832A6A14682A6A516868
:10D840002A6A9268501E9AB12CB3224612F801CB74
:10D8500014461A899207FCD5A3F80CC01A89D2077E
:10D86000FCD59A8992B209B101F8012B0138EBD2AB
:10D870002B6A1B7BF3B92B6A1B6993B12B6AD6F811
:10D8800094001B699847012808D0022809D1002379
:10D890002B62BDE8F8834FF0FF0CDAE72B6A143BEC
:10D8A0002B622A6A2B6A14332B622B6A9B686BB13A
:10D8B0006B68B9E7B368002BDDD01A689B881383C7
:10D8C000D9E742F003026DE7420846E72B6A1B687E
:10D8D000DBB12B6AD3E900622A620022C3E900228D
:10D8E0001CE700213046FFF75FFEB36813B11A68EA
:10D8F0009B8853833046BDE8F8438DE62A7B002A97
:10D900008DD0B8F1000F85D189E72B62C1E700BF48
:10D910000000FFFF003C0040003800400248836EDA
:10D920000BB1583018477047880100200348D0F8E1
:10D930008C300BB17C301847704700BF8801002045
:10D940000348D0F8B0300BB1A0301847704700BF83
:10D95000880100200348D0F8D4300BB1C4301847F8
:10D96000704700BF880100200348D0F8F8300BB1A1
:10D97000E8301847704700BF880100200348D0F8FE
:10D980001C3113B100F586701847704788010020DC
:10D990000348D0F8403113B100F59870184770472C
:10D9A000880100200348D0F8643113B100F5AA7053
:10D9B00018477047880100200348D0F8883113B118
:10D9C00000F5BC7018477047880100200348D0F864
:10D9D000AC3113B100F5CE701847704788010020B4
:10D9E0000348D0F8D03113B100F5E0701847704704
:10D9F000880100200348D0F8F43113B100F5F2702B
:10DA000018477047880100200348D0F8183213B136
:10DA100000F5027018477047880100200348D0F8CD
:10DA20003C3213B100F50B70184770478801002095
:10DA30000348D0F8603213B100F5147018477047EE
:10DA4000880100200348D0F8843213B100F51D701E
:10DA50001847704788010020094B0A4A013800EB3B
:10DA6000C00003EB8000116B836D074883420CBF3D
:10DA70004FF400134FF480030B431363704700BF50
:10DA800088010020003802400060024070B5013873
:10DA90003C4C3D4D00EBC00C04EB8C0C9646DCF886
:10DAA00058603A4AAE420CBF4FF400154FF480055F
:10DAB000166B35431563CCF86810CCF870303449D8
:10DAC000DCF85C308B424FEAC0023ED001F5806149
:10DAD0008B423AD0A1F57A718B4246D001F5806134
:10DAE0008B4242D0A1F57A718B4240D001F5806122
:10DAF0008B423CD0A1F57A718B4234D001F5806124
:10DB00008B4230D0A1F57A718B4232D001F5806121
:10DB10008B422ED0A1F57A718B422CD001F5806119
:10DB20008B4228D0A1F57A718B4226D001F5806115
:10DB30008B4222D0A1F57A718B4220D0154D01F590
:10DB400080618B4218BF002500E0134D104404EBA8
:10DB50008003CEF387119D6793F86D00BDE8704098
:10DB600000224CF083BD0D4DF0E70D4DEEE70D4D5D
:10DB7000ECE70D4DEAE70D4DE8E70D4DE6E7054D05
:10DB8000E4E700BF88010020006002400038024046
:10DB900010600240008000282080001000800018E3
:10DBA00000880010008020102080002000880020C5
:10DBB000008020202DE9F04FA24BDFF8A89293F8C7
:10DBC000F63DA14F8DB0CDE90139013BDBB20093A9
:10DBD0009E4B0025A3F5FC66DFF88CB2DFF88CA223
:10DBE0005B46D3469A464FEA9A23A3F58013522BFD
:10DBF0004CD8334493F898320D2B47D8FC56019BF0
:10DC0000012B40F0FE80012C35D14FF00008414639
:10DC1000204613F04DF913F0EBF9037813B1542BB0
:10DC200040F0098108F104081FFA88F8B8F1100FD4
:10DC3000EDD14FF0000E8DB3494600200CE0334487
:10DC400093F898320D2B0ED8FB56A3420ED001301C
:10DC5000A84201F580711EDA8A6813689B0AA3F551
:10DC60008013522BEBD90023A342F0D153799BF8B8
:10DC700005209A42EBD1754B9B454BD05BF820AF0A
:10DC80004FEA9A23A3F58013522BB2D9009B012BA4
:10DC9000F1D90024B9E7BEF1000FECD158460EF0DF
:10DCA000A5FCC3B2022B9BF805C000F23C83431CC9
:10DCB0005BB203EB43034FEA830E654B654903F503
:10DCC000727004E0834200F02E8353F82C1F5145FC
:10DCD000F8D11A796245F5D153F80E40002CF1D0F5
:10DCE0005D4800234268A24203F1010300F08680F0
:10DCF000102B00F12400F5D14FF0FF33574A03EB0E
:10DD0000C30302EB830393F87430002BB3D1029B5F
:10DD1000C3F808B0029B013503F58073042D02930C
:10DD20007FF45AAFDFF848A10AF29C534FF0010884
:10DD300000934B4BD3F8082508F1FF339A425ADD84
:10DD4000DAF80C50002D00F0EA822968AE8801F163
:10DD50003F41B6FA86F601F57E01C6F11F06890A33
:10DD60003F4B5F68002F40F38780002302E00133C0
:10DD7000BB427FD01C0259F804208A42F7D14C44A0
:10DD8000CAF80460CAF818405FFA88F315B1EB715D
:10DD90000323AB71636CE16C72000320904003437A
:10DDA0006364012303FA02F20A43E2642C4A127804
:10DDB00072B3226DB3401A43226515B12A68A9884F
:10DDC0001183D4F8A00099B20122FAF70FFB204684
:10DDD000FAF762FC009A012308F101088AF81C3066
:10DDE0008AF81D305374B8F1090F02F118030AF1D3
:10DDF000200A00939DD10DB0BDE8F08FDBB2013B4E
:10DE00007CE7022B7FF401AF082C3FF4FEAE32E733
:10DE1000226D06F110018B401343236515B12B6869
:10DE2000AA885A830121B140D4F8A00089B2002207
:10DE3000FAF7DCFACBE74FF0010E002D7FF4FCAED1
:10DE400019E700BF08190020104F0608D8E305089D
:10DE5000E4DE050800000140E00100208801002008
:10DE6000040000100C00001000040140D8E2050876
:10DE70000C040010032B61DCA64B03EB07233A02D2
:10DE800018690192002800F0438299600131CAB2FA
:10DE900083F8052102929F4AD0F800B001375760FD
:10DEA000542283F8042144790EF0A0FB9A4AC3B2AD
:10DEB00092F80BCE9AF810200392022B00F23382D4
:10DEC000471C7FB207EB4707944A9549BF000023E0
:10DED00005E00133172B00F0268252F82C1F8B45EA
:10DEE000F7D11179A142F4D1D1590029F1D02C22D6
:10DEF00000EB400002FB03F38A4A03EB8003134468
:10DF00000198D3F8FC22834B0344C3E90612864BE5
:10DF100000221F4618464368994220D00132102A39
:10DF200000F12400F7D1814B93F8502052B95422CC
:10DF300083F85020029A83F8512003E0764A0323A5
:10DF400082F80A3E73487A497A4A7B4BC0F88C19AA
:10DF5000C0F88429C0F894390DB0BDE8F08F531C87
:10DF6000DBB2724A0597013B03EBC30302EB830369
:10DF700093F874200492002AE4D1019F029A83F856
:10DF80007520FA116D4802EB2722542402EB02128D
:10DF900000EB82028C2183F8744069482C683B12A4
:10DFA00001FB03F300EB43005A4B3B44C3E93C0144
:10DFB000C3F8A8203322DC60C3F8AC20614B9B453A
:10DFC00009EB070418D0564B9B4515D003F5804349
:10DFD0009B4511D003F580639B450DD003F580630D
:10DFE0009B4509D04C4B1A68BCF1060F4FEA520210
:10DFF00007D15549554B0EE0474BBCF1060F1A6847
:10E00000F7D0534B53485449BCF1070F08BF19468A
:10E01000524B08BF0346B2FBF3F33E4FB2FBF1F2A3
:10E0200001995846013B07EB010B9BB2013AABF853
:10E03000B020ABF868305431A36500234944A4F8FC
:10E040005C30636543F08CFBDBF810B04449DBF8CF
:10E050000000028892B242F0800202800023ADF8F4
:10E060002030038807914FF48072022123F00103CE
:10E07000CDE90A121B044FF00A0C1B0CCDF824C08A
:10E0800003809BF8051007AA13F070FB9BF80400AF
:10E09000002840F025811F4B019A059F9A18002304
:10E0A0001069D2F818C001680A8892B242F00102E1
:10E0B0000A807A68944503F1010300F00D81102B6A
:10E0C00007F12407F5D14FF0FF33184A254FDFF849
:10E0D0009CC003EBC30302EB8303234A9B6DBB424B
:10E0E0000CBF4FF400134FF48003176B3B431363D3
:10E0F00043790C2B9CBF0B4A02EB4303019A98BF58
:10E10000B3F80078034B134488BF00279F82002395
:10E1100035E000BF0400001008190020E4DE050807
:10E1200000000140F8DB0508E00100208801002024
:10E13000199001081590010821900108142700206A
:10E14000442A002000040140882A1100A0BB0D00D1
:10E150001055220040771B0044950800D0DD0600D2
:10E16000600001000060024000380240FC0800101E
:10E17000914200F0D2800133042B00F0D7805CF88C
:10E180003320002AF4D16B4A1046D2F8F428013229
:10E19000C0F8F42800EBC302DB00C2F8F8186344AF
:10E1A00004989A88644917439F80624A019BD71854
:10E1B00023469022FFF76AFCB8690268002342F008
:10E1C00010020260C4E92533A367C4F88830C4F89C
:10E1D0009C30FA6962664FF400310422C4E92312CC
:10E1E0004FF4806B4021C4F87CB02167D7F8AC10A5
:10E1F0006167F968019B1831A1664FF48051C4F83A
:10E200008010D7F8A820E26603F164014FF4804241
:10E210004944C4F8842043F02DF9B869019BD0F833
:10E2200000E0C4F81CE0D0F814E0C4F820E0D0F816
:10E2300004E0C4F824E003F1AC01D0F808E0C4F82D
:10E2400028E00023D0F80CE0C4F82CE0C4E9373310
:10E25000C4F8B830C4F8C030C4F8D030C4F8E430E2
:10E2600004224FF4403CFB69C4F8AC30C4E935C229
:10E27000C4F8C4B0D7F8F430C4F8BC30FB6810332D
:10E28000C4F8B0304FF40063C4F8C830D7F8F030A9
:10E29000C4F8B4304FF480434944C4F8CC3043F060
:10E2A000E9F8BA6911682163516961635168A16332
:10E2B0009168E163D1682164116841F01001116037
:10E2C000039A8AF810205FFA88F3CAF80460CAF843
:10E2D0000C50CAF818405AE5DBB20493013BF4E64F
:10E2E0000FF0AAF8029038B19BF8082002210EF036
:10E2F0000FFE029B5422DA80DBF80020B2F8443093
:10E300006FEA43436FEA53439BB2A2F84430C2E63C
:10E310000A4A022382F80A3E14E6DB003FE74FF088
:10E32000FF3631461CE500235B68FFDE00239B8837
:10E33000FFDE00BF0400001035840008081900202B
:10E34000084B10B5D3F8A43418440C46007E0FF0E7
:10E3500073F818B1036882880CB11A8310BD5A8310
:10E36000FCE700BF002A00200B4B10B5D3F8A43403
:10E3700003440446187E0FF05FF858B12E228271D4
:10E38000621CC27101210EF03FFA20460021BDE857
:10E390001040D5E710BD00BF002A00202DE9F04F46
:10E3A0008DB00E469DF85840019403930546002811
:10E3B00000F0CF80DFF8CCC1077900230CF595641D
:10E3C00002E0152B00F0C58003EB43010133605CD4
:10E3D000B842F6D161442F6891F9AA8495F805E016
:10E3E0005FFA88F3022B00F2B48008F1010C4FFAB7
:10E3F0008CFC0CEB4C0C5F4B4FEA8C0C002105E0C5
:10E400000131172903F12C0300F0A380186887421B
:10E41000F6D118797045F3D153F80C40002CEFD0A9
:10E420002C2303FB01F108EB4808534BDFF858B1EC
:10E4300001EB88011944D1F8FC3205939BF81C3993
:10E440000093002B40F08A804C4FFB6DA34200F0FC
:10E45000E382D7F880309C4200F0CC84D7F8A43017
:10E46000A34200F0C984D7F8C830A34200F0C684A4
:10E47000D7F8EC309C4200F0C384D7F81031A342A7
:10E4800000F06284D7F83431A34200F0BB84D7F89F
:10E4900058319C4200F0B884D7F87C31A34200F098
:10E4A000B884D7F8A031A34200F0BF84D7F8C431B4
:10E4B0009C4200F0B884D7F8E831A34200F0B7845A
:10E4C000D7F80C329C4200F0BC84D7F83032A3421B
:10E4D00000F0BE84D7F85432A34200F0B784D7F8D6
:10E4E0007832A34208BF0F2300F0978200234FF039
:10E4F000FF3A0693009B002B48D00AEBCA0207EBB9
:10E5000082024FEACA03079392F87430392B00F065
:10E510002783D5F800804FEA9822A2F58012522A6C
:10E5200000F29B8214490A4492F898220D2A00F2C4
:10E5300094821349895CCBB9079A524407EB820253
:10E5400082F87510392182F87410069A72B100931E
:10E5500032E0DFF834B09BF81C393BB1D5E9054314
:10E5600005931CB1012300936EE729B300200DB081
:10E57000BDE8F08FE4DE0508F8DB0508880100201F
:10E58000104F0608002A0020040000100AEBCA03FE
:10E5900007EB83034FEACA01079193F8741000292F
:10E5A000E4D1013283F87520032283F87420069B9E
:10E5B000002BDBD0D5F80080DFF86C939BF818397E
:10E5C00006EB8602C2EBC20231B20B9191000891B8
:10E5D00009F1800101EB82020992ABB3D9F88C25D5
:10E5E000424500F01384012B2ED0D9F8A425904584
:10E5F00000F01684022B27D0D9F8BC25424500F044
:10E600001884032B20D0D9F8D425424500F01B8470
:10E61000042B19D0D9F8EC25424500F01B84052BBA
:10E6200012D0D9F80426424500F01784062B0BD0EF
:10E63000D9F81C26424500F01484072B04D0D9F8E1
:10E640003426424500F0828303EB430209EBC20209
:10E650000293C2F88C855A1CD2B28BF81829134643
:10E66000013B0299AB4A04938C2303FB069301EB15
:10E67000410102EBC10183F89160C3F88850C3F8EF
:10E68000041195F804C04FEA1C13013B052B0CF054
:10E690000F0C00F24F83A0490A9301EB4300B0F83E
:10E6A00000E14EFA0CF010F0010012D0012000FA47
:10E6B0000CFC0CF1FF3C0CEA0E004DF067FD964996
:10E6C0000A9B944A0B44C03293F80C31184402EB75
:10E6D000C000019A9BF8003002F00101013113B132
:10E6E00082F0010301938C2303FB0693490141F05F
:10E6F0000A01C3F894102A7A0DF090F9049B029A4B
:10E70000934200F07182039B063BDBB20A93089AA6
:10E7100082496032531807EE903A8C2306FB03F3CC
:10E7200003F1680C0A468C4409EB030100206033B6
:10E73000A1F8E400C1F8E800CCE901004FF0600C5A
:10E7400042F803C0019B13F00202089200F07881A6
:10E75000DB0003F00803A1F8EE300423A1F8F20077
:10E76000A1F8E4308C2303FB06930021C3F8E810E2
:10E770004FF00A0C68799BF81C19A3F8F6C04FF00B
:10E78000010CC3F8F8C04FF0020CA3F8F400A3F892
:10E79000FCC0002900F0CF81D3F804319C602368CD
:10E7A000CDED017A23F001032360204642F0CCFD39
:10E7B000009BDDED017A002B00F0AC818C2303FB84
:10E7C00006939BF81C090027C3E92677C3E928773D
:10E7D000C3E92A77C3E92C77C3E92E77C3E93077F9
:10E7E000C3E93277C3F8D070002800F06F81039A34
:10E7F0002968082A029A01F14C00494902EBC20E2D
:10E80000D3F8042101EB4E111161AA69C3F89820D5
:10E81000C3E927014FF04001C3F8A4104FF0040EE4
:10E820004FF00301C3E93377C3E931E10CBF06219F
:10E830001221C3F8AC70C3F8BC70C3F8A8104FF431
:10E8400080624FF48051C3E92C214FF48041C3F81A
:10E85000B8104FF400310A9AC3F8C0108C2303FBA0
:10E860000693022AC3F8004100F2E58003990829C3
:10E87000294901EB820108BF5F27D1F88C0829499B
:10E88000B1FBF0F101F12301C3F8D81018BF132731
:10E890008C2101FB06912046D1F80431D1F888A0E3
:10E8A0009F80CDED037A0191DAF8007042F04CFDC3
:10E8B0000199DDED037A002381F8D4309AF8051030
:10E8C0000C2914D8DFE811F0CB001300130013005B
:10E8D000F400130013001300ED00130013001300E5
:10E8E0000D00BB8B23F400631B041B0CBB8317EED2
:10E8F000902A384612F03AFF9AF805300C2B1DD8B2
:10E90000DFE803F0C61C1C1CBD1C1C1CB41C1C1C1A
:10E91000140000BF941E0020F8DB050888190020B1
:10E92000E82E002000D0121308190020BB8B23F41E
:10E9300000631B041B0C43F40063BB83099920682C
:10E940008C2202FB069240234B62D2F8A410D2F82C
:10E9500098300B43D2F8AC100B43D2F8B0100B43F5
:10E96000D2F8B4100B43D2F8B8100B43D2F8BC1055
:10E970000B43D2F8C0100B43D2F8CC100B43D2F8A3
:10E98000D0100B43924901400B439BF81C092360B4
:10E99000D2E9313167690B4327F007073B436361D5
:10E9A000D2F8A8306360D2F89C30A360D2F8A030CF
:10E9B000E360236843F01003236090B3009B83B3AC
:10E9C000B8F800309BB243F00103A8F80030B8F863
:10E9D0002020089B697992B25BB304238B409BB2E1
:10E9E00022EA0302A8F82020B8F8202092B21343AC
:10E9F000A8F82030029A049B934200F0D1809BF843
:10EA00000030002B5BD18C2303FB0696012086F897
:10EA10008F000DB0BDE8F08F0023591C06919A4677
:10EA200068E592F8913006986A499022FFF72EF82F
:10EA3000C6E70123D2E78D21C3F8D810132727E7B3
:10EA40005B0003F00203A1F8EC300123A1F8E230EF
:10EA50004FF48073A1F8F03084E600216BE53B8B26
:10EA600023F008031B041B0C3B8340E7BB8B23F004
:10EA700008031B041B0C43F00803BB835EE73B8BBE
:10EA800023F400631B041B0C43F400633B8355E732
:10EA90003B8B23F008031B041B0C43F008033B8350
:10EAA0004CE7BB8B23F008031B041B0CBB831EE746
:10EAB0003B8B23F400631B041B0C3B8317E72B6881
:10EAC0006A7934334FF6FF7199509CE7059AC3F881
:10EAD00098200B9A4049C3F8D00002EB820702EB62
:10EAE000470701EBC701C3F80811C3F8A010C3E939
:10EAF00032004021C3F8A4100421C3F8C4102968CF
:10EB00006F79C3F8AC0034313944C3F89C10C3F8B2
:10EB1000BC0094E6079B31493148534407EB830717
:10EB2000BB6D83420CBF4FF400134FF48003086B9E
:10EB300003430B6342E60C2800F2FE80294B03EBF3
:10EB40004000B0F80018C84300B28C2303FB0693C2
:10EB5000A3F88C10D3F80431998A084098821EE6F5
:10EB6000D5F8008092F875104FEA9822A2F580122D
:10EB7000522A3FF6FAAC1B4800EB020C9CF898C2F4
:10EB8000BCF10D0F40F2DB804FF0000C61453FF40B
:10EB900013AD024492F898220D2A7FF6CAACE5E440
:10EBA000B8F800309BB243F08003A8F80030B8F802
:10EBB00044306FEA43436FEA53439BB2A8F84430B2
:10EBC000B8F800309BB243F00103A8F8003016E714
:10EBD0003F801CF0C5940008E83700200038024050
:10EBE00000600240F8DB0508AC4B984500F03D8121
:10EBF000B8F1804F00F03D81A3F57C43984500F0CB
:10EC0000368103F58063984500F0378103F5806312
:10EC1000984500F0308103F58063984500F033811A
:10EC200003F58063984500F02C8103F57043984507
:10EC300000F0318103F57053984500F02A8103F507
:10EC40008063984500F0238103F58063984500F0C8
:10EC50001C81A3F5983398457BD003F580639845D4
:10EC600000F00D8103F58063984508BF0D2371D036
:10EC7000B8F8003023F001031B041B0CA8F8003087
:10EC8000D9F800305B0807EE903A039B063BDAB2F6
:10EC9000022AF8EE677A0A9200F29980804BDFED43
:10ECA000816A03EB820303F68C0292ED007AB8EEE0
:10ECB000477A87EE870A30EE260A4EF06FFA039BFA
:10ECC0000138082B82B214BF13215F217348B8F8B2
:10ECD000003080459BB26FD000F5806080456BD0DE
:10ECE000B8F1804F68D0A0F58030804564D000F541
:10ECF0008060804560D000F5806080455CD06A48C7
:10ED0000804570D000F5806080456CD023F440735E
:10ED10009BB2A8F80030614BC8F82C109845A8F8B1
:10ED2000282040F089800023A8F830300123A8F87B
:10ED30001430ECE40020CCE44FF0FF3005E7DFF8BE
:10ED400078E11EF90CC021E7052366E6072202924E
:10ED500086E40B23524A02EBC303012193F82038C7
:10ED600003F01F025B09032B01FA02F253D0042BBC
:10ED700026D14E490B6B13430B63B8F8003023F0D8
:10ED800001031B041B0CA8F80030494B984510D018
:10ED9000A3F5806398450CD003F58043984508D0CF
:10EDA00003F58063984504D003F5806398457FF4AC
:10EDB00067AFD9ED007A68E723F070039BB29EE756
:10EDC000022BDAD139494B6C1A434A64D5E79FEDDF
:10EDD000397A9FED340AA7EE870A4EF0DFF9013841
:10EDE00082B2132172E7A8F80030C8F82C10A8F8F6
:10EDF00028209BE7012310E602230EE603230CE6FE
:10EE000004230AE6062308E6072306E60022029208
:10EE100026E4082301E625490B6C1A430A64ACE793
:10EE2000012202921CE40A23F7E50923F5E50B23EE
:10EE3000F3E50222029213E41D4B98453FF473AFB1
:10EE400074E70C23E9E50322029209E40E23E4E5CA
:10EE50000D23E2E50422029202E405220292FFF76A
:10EE6000FFBB06220292FFF7FBBB002372E70223DF
:10EE700070E701236EE704236CE703236AE70C23A2
:10EE800068E7062366E7052364E70A2362E70923A8
:10EE900060E708235EE707235CE700BF000001404E
:10EEA000F8DB05080AD7233C001000400038024078
:10EEB00000040140FCF4B234104F060838B5424C4F
:10EEC0008C2303FB004393F88F3003B938BD94F8CB
:10EED000E0C494F8E1349C450ED003EB430204EB0C
:10EEE000C20292F8E4E40EF1FF35012D4FEA43022D
:10EEF00046D9BEF1030F3ED08C2202FB0042A2F89D
:10EF00008010EFF31181902383F31288B2F88050C0
:10EF100092F8823043EA45030025C9B29BB282F8D9
:10EF2000825081F3118829491A090D7882EA132247
:10EF30005A4005B1D2431B019BB202F00F021A43A3
:10EF400091F81C395BBB8C2303FB0044D1F8643A75
:10EF5000D4F8080101219847D4F80411B4F88C5072
:10EF60008A8AD4F800312A438A8258601A6842F0AB
:10EF700001021A6038BD5D1C05F003056545BBD074
:10EF8000134404EBC303034493F8F1140029B3D0F2
:10EF90008C2303FB0043012283F88220ACE78C23FF
:10EFA00003FB0044D1F8645AD4F88830D4F8041133
:10EFB0005B79086903F0FC0318440421A847D4F8DE
:10EFC00004318000988138BD081900200400001029
:10EFD00030B50446006EA268838923F400531B04F5
:10EFE0001B0C8381637995B013F0040F4FF000017F
:10EFF000019214BF4FF480520A46ADF808201A035C
:10F000001B0203F48063ADF80C302379ADF80E10C9
:10F0100002F40052ADF80A20DA0744BF0422ADF82A
:10F020000E209B07ADF8101005D5BDF80E3043F04B
:10F030000803ADF80E3001A942F0E0FB6279236EBF
:10F04000D50700F18B8012F0080F9A8A48D092B24F
:10F0500042F008029A829A8992B242F400529A814E
:10F060002279D00732D5E06B002800F08980002398
:10F07000E26D0893CDE90C33CDE91033CDE91233BD
:10F080004FF480750A936369E1680E9506920793C1
:10F09000626C05924FF480634FF480350B930991B5
:10F0A0000F9542F051F905A9E06B42F0E3F9E26BEC
:10F0B000216E136843F0010313608B8A9BB243F007
:10F0C00040038B82536822799BB2636591070DD40C
:10F0D000226E93899BB243F40053938115B030BDE7
:10F0E00022F008021204120C9A82B4E7206C002865
:10F0F00052D02369A26D0993A36CCDE90532402358
:10F1000000254FF4803108934FF480630B930F91E7
:10F11000CDE90C55CDE91055CDE9125507950A9565
:10F120000E9542F011F9206C05A942F0A3F9236C69
:10F13000226E586940F080005861186840F016004F
:10F1400018605D60938A9BB243F0800302F10C016A
:10F1500093820B6843F040030B60BAE71E498B4271
:10F1600024D0A1F54C418B421ED001F580618B4229
:10F170001ED102200121FFF7E3F86279236E62E7D6
:10F180004FF6DF711980D96841F02001D960D96844
:10F1900041F01001D96099E7226ED36843F08003F3
:10F1A00002F10C01D360D4E70120E3E70020E1E79E
:10F1B00001F580618B420AD001F580618B4208D055
:10F1C00001F544418B427FF43EAF0520D2E7032096
:10F1D000D0E70420CEE700BF001001402DE9F84F32
:10F1E000484C04EB8004D4F8684A002C00F081807D
:10F1F000E56E002D79D01F46EB6A6361AB6AA361AF
:10F200006B8EE3602B8E23616B6823663E4B23601D
:10F210003E4BA160A3660646204691460EF050FA8A
:10F2200094F871000EF008F9804695F8200094F8E3
:10F2300070B0A246002855D102233A0784F87C30EA
:10F240003BD419F0020F15D0B8F1000F12D00B23E8
:10F2500088F80630731C88F80730FB074BD494F805
:10F2600071000EF0E9F8012384F87C3010B1202100
:10F270000DF06EFC19F0010F04D1E26B9AB150460B
:10F28000BDE8F88F58460EF0D7F80028F5D00C22CC
:10F290000136C671827195F8212022210CF0BEFB47
:10F2A000E26B002AEBD195F8241095F82200890929
:10F2B0004BF0DCF95046BDE8F88F0136F6B2B8F1F4
:10F2C000000F04D00B2388F8076088F8063017F089
:10F2D000500F95F82120404614BF022112210CF056
:10F2E0009DFBCAE74AF09EFAA6E7AA465046BDE84B
:10F2F000F88FA246C3E795F82120404622210CF062
:10F300008DFBB7E70400001090E40508F19D0008AC
:10F3100008B572B6FDF728FC00B583B00D49002290
:10F3200000920091009B0C330093009B1B68012B03
:10F3300002D003B05DF804FB01920191019B0649E4
:10F340000C330193019B1A600B6883F308884B68A8
:10F350009847FEE7502800400000FF1F30B501200D
:10F3600085B042F009F9794A936823F0030393606A
:10F37000936813F00C0FFBD113687449002857D120
:10F3800043F00103136041F288330A68950770D493
:10F39000013BFAD16E4C6D4B6E4AE2606E4A596F7A
:10F3A000A2605A6B6D4D22F080025A63586F6C4A0E
:10F3B00040F080705867186B40F4CE001863596BAA
:10F3C0005963996B9963196C29431964596C0A4301
:10F3D0005A64684641F06AFFD4F8FC10614B6248F9
:10F3E000009A41F080710025C4F8FC10C3F8B00FFA
:10F3F0005D6019685D4841F00101196003685C496E
:10F40000A1FB03135B499B09013BA1FB0212920C78
:10F41000B3F1807FC0F8502908D24FF0E022F021EC
:10F420005361072384F823109561136105B030BD43
:10F4300043F4803313600A68940341F2883304D4A0
:10F44000013BA7D00A689403FAD54B4C4B4A4C4B6E
:10F45000B0FBF3F3B0FBF2F0B3EB400F18BF18466C
:10F460004FF48002B3FBF0F344F83C2C44E914035E
:10F4700007E0414C0822022344E91423002144F808
:10F480003C1C022042F078F803280FD83D4B54F87A
:10F490004C1C03EBC0008588C288438844F8445C58
:10F4A000B3FBF1F344F8402C44F8483C274B364971
:10F4B0001A6C42F080521A640A6842F440420A60B0
:10F4C0009A689A609A6842F400429A609A6842F494
:10F4D000A0529A6054F83C0C54F8502C54F8481C34
:10F4E000024342EA811254E91110490842EA0062DB
:10F4F000013942EA01425A601A6842F080721A6089
:10F500001A689201FCD5214A40F205711160996890
:10F5100021F003019960996841F00201A2F580622F
:10F520009960936803F00C03082BFAD154F84C0C43
:10F530001749D823B3FBF0F39B0143F0005301209C
:10F54000C2F884308866F8F75BFD23E70038024094
:10F5500000ED00E00005FA0500000020FFC9FE36BE
:10F56000335F0700001000E055CEACC5081900203D
:10F57000D34D621083DE1B43F83A002080841E00C6
:10F5800040420F00C0E4050800700040003C02400B
:10F59000000047421D4B1E48196C1E4A10B441F032
:10F5A00080510124196404625321FF24CA2054624B
:10F5B000506251625B6FDB0085B017D4164804239C
:10F5C000002102910290029A1A440292029A043394
:10F5D0001C2B1160F5D103910390039B0393039BB4
:10F5E0000E4A1A6005B05DF8044B70470A4B0022C2
:10F5F00001920193019B0193019A084B12689A4270
:10F60000DCD105B05DF8044B704700BF0038024004
:10F6100000000E420028004050280040316665423C
:10F620004B1C10B408BF4FF0800C4D4C18BF4FF06E
:10F63000450C4FF4003300E003B3626B12EA0C0F89
:10F6400003F1FF33F8D0002923DD626B52071CD48D
:10F6500003291ED0424A536B13F0010320D1022923
:10F6600008D01369DBB283421ED1012953692BD024
:10F6700006291BD000205DF8044B7047002904DDEB
:10F68000636B5C0701D40329E4D103205DF8044BCC
:10F690007047002B14BF002003205DF8044B704717
:10F6A00001205DF8044B70471020EFE713F4604F22
:10F6B00004BF2C4A42F8383C990431D45A04F3D49C
:10F6C0001B04D7D50F20E1E7274818400028DDD0DC
:10F6D000002B29DB5C0025D4980029D4D90025D43F
:10F6E0001A0129D45C0125D4D8012FD41902E9D4F8
:10F6F0005A02D9D49C0227D4D8022FD419030FD48C
:10F700005A0329D49C0325D4D80321D4190419D42D
:10F710005A0415D49C0411D41807ABD51A20B5E7A8
:10F720001320B3E70920B1E71C20AFE70B20ADE7BA
:10F730000A20ABE70D20A9E70C20A7E71920A5E7D1
:10F740001820A3E71720A1E711209FE70E209DE7CF
:10F7500016209BE7152099E7142097E7122095E7DC
:10F76000002C0140F83A002008E0FFFDF8B5164DE6
:10F7700055F80C3CA3B155F8041C0129044615D0DA
:10F78000124BDA6A22F00802DA6240F2FF510022DC
:10F79000996345F80C2C236823F001032360F8BD1E
:10F7A0000A4AD36B43F48073D363F8BD074E40F22B
:10F7B000FF570023B763B36040F24C43F3600C2063
:10F7C000FFF72EFFB763DBE7F83A0020002C01407B
:10F7D0002F4B1A68910102D59A6D52074BD42C4BCE
:10F7E0001A68500202D5DA6E11063CD4284B1A680A
:10F7F000D20102D59A6D90072DD4254B1A6851017C
:10F8000002D59A6D120717D4214B1A68120112D52E
:10F810009A6DD0060FD59A6D510334D49A6DD205E6
:10F8200003D49A6D22F010029A65194B19484FF0D3
:10F8300000629A609AE770479A6D500307D49A6DF8
:10F84000D10503D49A6D22F008029A65104B4FF04F
:10F8500080629A60D8E79A6D4FF0807122F00202C0
:10F860009A659960C9E7DA6E4FF4800122F0800250
:10F87000DA669960BAE79A6D4FF0007122F00402DF
:10F880009A659960ABE74FF000629A60704700BFDD
:10F890000064024058640240384B5A68110303D593
:10F8A000D3F8A02052075BD4344B5A68D00303D559
:10F8B000D3F8B420110649D4304B5A68520303D50B
:10F8C000D3F8A020900737D42C4B5A68D10203D527
:10F8D000D3F8A02012071CD4284B5A68920217D5DF
:10F8E000D3F8A020D00613D5D3F8A020510341D4DB
:10F8F000D3F8A020D20505D4D3F8A02022F010021E
:10F90000C3F8A0201D4B1E484FF40012DA602DE70B
:10F910007047D3F8A02050030AD4D3F8A020D10513
:10F9200005D4D3F8A02022F00802C3F8A020134B7E
:10F930004FF48012DA60CFE7D3F8A0204FF4802193
:10F9400022F00202C3F8A020D960BDE7D3F8B420AA
:10F950004FF4803122F08002C3F8B420D960ABE7C5
:10F96000D3F8A0204FF4002122F00402C3F8A02015
:10F97000D96099E74FF40012DA60704700640240E2
:10F98000A064024070B52A4E327882B00023022A69
:10F99000CDE9003346D8274D6B699B0102D50E2077
:10F9A00002B070BD0446684649F03EFE0028F7D11B
:10F9B000B4F5006F019B0CBF4FF480224FF48032EE
:10F9C0001A4232D056F8382C40F2774340F2FF56B4
:10F9D000AE630121AA603720EB60FFF721FEAE6322
:10F9E0000028DDD1B4F5006F08BF022040F2464385
:10F9F000AE630121A860EB600620FFF711FEAE6345
:10FA00000028CDD16B6803F400639C42C8D00A4A39
:10FA10006B68134023436B606B6803F40063A3427D
:10FA2000F6D1BDE7282002B070BD2620B8E700BFA0
:10FA3000F83A0020002C01400081FFFF70B5174DFF
:10FA4000174C55F8382C40F2FF5640F24D43A66350
:10FA50000121A2600D20E360FFF7E2FDA66320B95B
:10FA60006369C3F34323042B02D04FF0FF3070BD12
:10FA7000A86D0028FBD002688388116995F855208D
:10FA80000B402AB1002B0CBF00204FF0FF3070BD9F
:10FA9000002B14BF00204FF0FF3070BDF83A00205B
:10FAA000002C014070B51B4EB46D10463CB125686A
:10FAB000A2882C69224096F855402CB332BB0A46E6
:10FAC000002149F047FD08BB56F80C3C002BFBD148
:10FAD000114C40F2FF5556F8382CA56340F24D43C7
:10FAE000A26001210D20E360FFF79AFDA5630028C5
:10FAF000F1D16369C3F34323042BECD1074BD3F853
:10FB00008025C3F8842570BD002AD8D14FF0FF307E
:10FB100070BD00BFF83A0020002C014008190020F9
:10FB200070B51B4EB46D10463CB12568A2882C6997
:10FB3000224096F855402CB332BB0A46002149F0CA
:10FB4000ADFC08BB56F8083C002BFBD1114C40F231
:10FB5000FF5556F8382CA56340F24D43A2600121B1
:10FB60000D20E360FFF75CFDA5630028F1D1636918
:10FB7000C3F34323042BECD1074BD3F88025C3F800
:10FB8000842570BD002AD8D14FF0FF3070BD00BF72
:10FB9000F83A0020002C014008190020C64B53E918
:10FBA0000D1270B58C0F83F8F840C1F3836483F8AD
:10FBB000F940C1F3016483F8FA40100EC1F3074421
:10FBC00083F8FB400001C1F30724C9B283F8FC406D
:10FBD00083F8FD10A3F8FE00B3F8FE10C2F3035043
:10FBE00089B20143C2F30344A3F8FE10C2F3C0304C
:10FBF00083F80041C2F34031C2F3803483F801013D
:10FC000083F8024183F80311C2F3003183F8041131
:10FC1000197800200129C2F3072C83F8050140F26E
:10FC2000F380022900F0C58053F82C1C2A204FEAEB
:10FC30004C0C0CF07E0C83F8114183F812C193F840
:10FC40001241C1F3C012144353F8282C83F8124117
:10FC500001F07F01D40F83F8131183F81441910D43
:10FC6000C2F3417483F8154101F00C01C2F38264C0
:10FC700083F8164183F8171193F81711C2F38154D2
:10FC80002143C2F3405583F8171183F8185100251A
:10FC900083F81951C2F3004583F81A51C2F3C035F5
:10FCA00083F81B51C2F3803583F81C51C2F34035F1
:10FCB00083F81D5153F8244CC2F3003583F81E51CC
:10FCC000C2F3812583F81F51C4F30741C2F3012514
:10FCD000C2F3460283F820514FF0010C83F8212132
:10FCE0000902220E83F822C183F82421A3F82611E9
:10FCF000B3F82611C4F3072289B211432406A3F8EE
:10FD0000261153F8201CC3F82841D3F828210C0EE3
:10FD100042EA0442C3F82821D3F828410A0A02F42F
:10FD20007F422243C3F82821D3F8285153F81C2CD2
:10FD3000C1F307242C43C9B2C3F8284183F82C111E
:10FD4000110E83F82D11110C0906C3F83011D3F8E8
:10FD50003041110201F47F012143C3F83011D3F87F
:10FD60003011120292B20A43C3F83021D3F8301195
:10FD700053F8182C41EA1261C3F8301193F834118A
:10FD8000C2F30354214383F83411110A01F4706162
:10FD9000A3F83611B3F83611C2F3072489B2214310
:10FDA000C2F34602A3F8361183F8382183F839C12B
:10FDB00070BD120402F47C12C3F8082153F82C1C05
:10FDC000D3F808210C0E42EA0422C3F80821D3F824
:10FDD0000841C1F307422243C3F80821D3F80821A0
:10FDE000013240F10004A40244EA92549202C3F8A2
:10FDF00040214FF40072C3F84441C1F3072CC3F80B
:10FE00004821C1F3803412E74FEA8C2C0CF4406196
:10FE1000C3F80811D3F80811920002F47F720A4364
:10FE2000C3F80821D3F8084153F82C1C44EA917414
:10FE3000C3F80841C1F3C265C1F3026483F80C51F1
:10FE4000CA0B83F80D41C1F3425483F80E4102F00E
:10FE50000602C1F3824483F80F4183F8102193F81E
:10FE60001021C1F3C034224383F81021D3F8084194
:10FE700093F8102193F800E1961C012202FA0EF586
:10FE8000B240D617A2FB052E05FB06EE04FB0EEED4
:10FE90000134A2FB0424A644520A42EACE52C3F81B
:10FEA00040214FEA5E22C1F3072CC3F84851C3F842
:10FEB0004421C1F38034BAE6F83A002070B50E4E02
:10FEC000B36D0D4614463BB11A689B881269134006
:10FED00096F8552052B15BB9FFF760FED6F8402185
:10FEE0002A604FF400730020236070BD002BF3D113
:10FEF0004FF0FF3070BD00BFF83A00202DE9F84FF9
:10FF0000734F744BD7F850410546002259688C4214
:10FF100003F1240302F1010200F09580102AF5D1CB
:10FF200000246D4B9D4205D048339D4202D00020F5
:10FF3000BDE8F88F661EDFF8D09106EBC60309EB2B
:10FF400083034FEAC60A93F87420002AEFD14FF0DA
:10FF5000170BA3F874B0002CE9D0DFF89081D8F823
:10FF6000243043F40063C8F82430012010F0A0FAD4
:10FF7000D8F8243023F40063C8F82430012010F0AE
:10FF800097FAD8F8443043F40063C8F84430D8F8FE
:10FF9000303043F48003C8F83030D8F8303043F0C4
:10FFA0000C03C8F8303097F85631DFF86081A8F8B4
:10FFB00092B7002B49D1A8F8B2B7A8F8E2B708F277
:10FFC0008C700C220E210BF029FD44480C220E21CE
:10FFD0000BF024FD42480C220E210BF01FFD414B7B
:10FFE000414ADB68414BC7F8505100214FF40030C3
:10FFF00082F8311350601A6B42F480021A63364A59
:020000040801F1
:10000000296056443A49A960954209EB86093FD0D8
:10001000D9F85810374A384E38484FF47417F760FB
:10002000914228604FF00700686146D01A6B42F495
:1000300080021A633249204600230122FDF726FD83
:100040000120BDE8F88FD4B26BE708F28C70A8F8F5
:100050009AB7A8F8A2B7A8F8AAB7A8F8B2B7A8F8AC
:10006000E2B70C220E210BF0D9FC08F294700C229E
:100070000E210BF0D3FC08F29C700C220E210BF029
:10008000CDFC08F2A4700C220E210BF0C7FC9CE7FB
:100090004FF07466D9F85800164942F8506C583A37
:1000A000164D956588424FF00705D5660AD01A6B44
:1000B00042F480021A631349BDE71A6B42F400123E
:1000C0001A63B7E71A6B42F400121A63F3E700BF32
:1000D000F83A0020E001002058640240B4200020DB
:1000E000E420002000ED00E000E100E000380240E4
:1000F000802C014000600240006402406054A3086C
:1001000099F80008D1F7000888010020081900209C
:1001100038B50E4B0E4C53F8382C40F2FF5540F2D8
:100120004D43A5630121A2600D20E360FFF778FA3B
:10013000A56340B96069C0F34320A0F10400B0FAA0
:1001400080F0400938BD002038BD00BFF83A0020DB
:10015000002C01402DE9F043B24C636823F4FD43C9
:1001600023F07F0343F0760363606368032223F484
:10017000807363600220226093B010F099F9636885
:1001800040F2FF5043F4807300214FF480626360BB
:10019000A0634FF40033A160E26002E0002B00F0A6
:1001A000BE80626B120603F1FF33F7D5002B00F01F
:1001B000B68040F2FF554FF4D5724FF48963A563C2
:1001C0000721A5630820A260E360FFF729FAA56371
:1001D000002800F09E800026DFF8488240F2FF5998
:1001E000002240F27743C8F838900121C8F808206F
:1001F0003720C8F80C30FFF713FAC8F838900446D7
:10020000002840F0828046F000460546074646F446
:10021000801602E0954200F0FD8040F27743C8F876
:1002200038900121C8F808703720C8F80C30FFF763
:10023000F7F9044640F26943032129200135C8F843
:100240003890002C61D1C8F83890C8F80860C8F818
:100250000C30FFF7E5F94FF6FF72C8F83890044606
:10026000002852D1D8F81430002BD3DA4FF6FF72A1
:10027000954200F0CF805F005AD4D8F800309C0738
:100280005DD0694D287804285ED1FFF787FC0446CD
:1002900000283AD1634E55F8382C40F2474340F2DB
:1002A000FF57B7630121B2600720F360FFF7B8F989
:1002B000B763736823F4FD4323F07F037360044640
:1002C00018BB95F85631002B00F09E804FF400606B
:1002D000FFF758FB0446C4B995F85431ABB1514D02
:1002E00002943C22214603A84DF033FCCDE90044A2
:1002F0006846EC6249F098F9002840F0E380019BE1
:1003000013F0407F40F092800024204613B0BDE8F7
:10031000F083454B01221A704FF080465CE7414B59
:10032000032440F2FF5220469A6313B0BDE8F083E5
:100330003D4D02202870D8F800309E0704D12624B5
:10034000204613B0BDE8F0833649002340F2FF5247
:100350008A638B6040F2C243CB604FF4003301E00C
:10036000013B03D04A6B12F0450FF9D02D4B5A6B6D
:10037000520751D45A6B12F0010F40F2FF529A63A8
:1003800046D15A6945F8242C9A6945F8202CDA6937
:1003900045F81C2C1B6A45F8183C01282FD8214E23
:1003A00040F2FF57002240F24343B7630621B26098
:1003B0000320F360FFF734F9B76304460028A4D1A3
:1003C000184E55F8382C40F2FF5740F2C943B76336
:1003D0000221B2600920F360FFF722F9B7630446F7
:1003E000002892D1736945F8343CB36945F8303C34
:1003F000F36945F82C3C336A45F8283C45E700F0A2
:10040000FB000228CBD0DBE7FFF7BCFA044662E72B
:1004100001247AE71B2478E740F2FF529A63032411
:1004200073E700BF002C0140F83A002040F2FF566D
:100430004FF48A634027AE630121AF601020EB6068
:10044000FFF7EEF8AE6300283CD1284B6B62AF6239
:10045000EB6A274A43F06303EB6240F24643AE6324
:100460000121AA600620EB60FFF7DAF8AE6348BB13
:1004700009AB40F22A41A3F11C0202E0686B0004C0
:100480002AD4686B0842F9D06B6B19071AD46B6BCE
:100490009B0717D46B6B9F0614D46B6B9E020CD515
:1004A000144B1549134401E0934206D0D1F8800063
:1004B00042F8040B486B8002F6D49DF815309D0776
:1004C0003FF522AF0C4B5A6842F480625A605A687A
:1004D00042F400525A6018E7A3F12002D5F88000D8
:1004E00042F8040F9342F9D12033C4E700E1F50547
:1004F00001FFFF800084D717002C014038B52F4C36
:1005000094F85D010CF098FF08B11F23C3802C4DB7
:1005100020210CF079F995F86B3DD5F86C2D03F09E
:1005200001031AB10BBB136892881A8394F95721FF
:10053000D3B2012B17D8234B4FF00C0C082003F536
:1005400013711CFB020C8B420DD013F81C2F032AD5
:10055000F9D15A78002AF6D153F80C000028F2D0CD
:10056000FFF7CCFC28B9012038BD136892885A8364
:10057000DCE7A36D43B11A689B881269134094F8B5
:10058000552072B9002BEED094F8613163B10E4B57
:1005900093F898020028E6D1D5F88035C5F884355F
:1005A00038BD002BDFD1EFE7012384F86131FFF77D
:1005B000D1FD054B83F89802ECE700BFF83A002024
:1005C00008190020E0E405088801002070B5314CCE
:1005D000636BD90521D54FF4807340F2FF56A363B6
:1005E000A663E36B2C4D23F4414323F03A03E3630A
:1005F00055F8043C9A0723D40122002345F8142C13
:1006000045F8103C234A40F2FF539363D36B23F425
:10061000414323F03A03D36370BD636B980704D55D
:100620001D4B022243F8102CECE7636B190723D40F
:10063000636B9A0625D5184B062243F8102CE1E788
:10064000D5F85021136823F001031360E36A0022F8
:1006500023F00803E36245F8082C55F8043CDB0757
:10066000CAD540F24C43A6630121A2600C20E3608E
:10067000FEF7D6FFA663BFE7074B042243F8102C12
:10068000C0E7636BDB06BDD5034B052243F8102C96
:10069000B8E700BF002C0140F83A002070B5444D87
:1006A000C1F1030195F8422041EA8001CBB29A42A0
:1006B0008AB073D03F4C85F84230102184F8681A14
:1006C000122184F86C1A132184F86E1A142184F80C
:1006D000701A152184F8721A162184F8741A1721D9
:1006E00084F8761A182184F8781A192184F87A1A6D
:1006F0001A2184F87C1A1B2184F87E1A1C2184F8A4
:10070000801A1D2184F8821A1E21112084F8841A6F
:100710001F2184F86A0A84F8693A84F86B3A84F8ED
:100720006D3A84F86F3A84F8713A84F8733A84F831
:10073000753A84F8773A84F8793A84F87B3A84F801
:100740007D3A84F87F3A84F8813A84F8833A84F8D1
:10075000853A84F8861A04F51D6684F8873A04F60B
:100760006823002201250093694620233046CDE905
:100770000123CDE90422CDE9062209928DF80C501F
:100780008DF820500BF0CAFBD4F8D0395A6A12B158
:10079000B24205D0FEE71A6A002AFCD10AB070BD49
:1007A0001A6A002AFAD01A6A002AF9D1F6E700BFBD
:1007B00088010020081900200A4BB3F8401071B1DD
:1007C000094B0A4A01EB030C01E0634507D013F81B
:1007D000010B12F8011B8842F7D00020704701205E
:1007E000704700BF880100205C3C0020942300205B
:1007F0002DE9F041964D974ED5F8804594B028B933
:10080000D6F89C3203F57A73A34254D2924FC6F8BD
:100810009C4200230122FF21CDE90532CDE90833B6
:10082000CDE90A338DF80C100D9304A903AB3846BB
:100830008DF81C208DF83020049301910BF06EFB95
:10084000D5F8D03901995A6A002A3BD0BA4200D073
:10085000FEE71A6A002AFCD10023CDE9083305938C
:100860008DF81C300D9310931293012306930B9374
:100870008DF830308DF8443080238DF80E300DF136
:100880000E0304930DF10F0300220A937248002314
:10089000CDE90E230BF042FBD5F8D0395A6AC2B12C
:1008A000BA421DD11A6A002AFCD19DF80F3096F881
:1008B0003E209A423ED195F8CF0990B1002014B065
:1008C000BDE8F0811A6A002AC6D01A6A002AF9D156
:1008D000C2E71A6A002AE8D01A6A002AF9D1E4E7C6
:1008E000FEE7DFF87881D8F82435E31AB3F57A7F8C
:1008F000E5D90123584F06938DF81C308DF8303020
:10090000FF2304A9CDE90800CDE90A0005900D9068
:100910008DF80D3038460DF10D03049301910BF065
:10092000FDFAD5F8D03901995A6A002A32D0BA4274
:1009300006D0FEE7FBF7F4FE012014B0BDE8F0811D
:100940001A6A002AFCD10023CDE9083305938DF8FB
:100950001C300D9310931293012306930B938DF883
:1009600030308DF84430A0238DF80E300DF10E0399
:1009700004930DF10F0300220A9337480023CDE9B9
:100980000E230BF0CBFAD5F8D0395A6A6AB3BA42C3
:1009900007D0FEE71A6A002AD5D01A6A002AF9D1D0
:1009A000D1E71A6A002AFCD195F845259DF80F3049
:1009B000172A0FD196F83E2002F04002002AA5F82F
:1009C000482503F00702A5F84A2514BF10220D227E
:1009D000A5F84E2559070FD50023C8F82835002063
:1009E000C8F8244514B0BDE8F0811A6A002ADBD0AB
:1009F0001A6A002AF9D1D7E703F00503012B1CD0AE
:100A0000002BECD196F83E305B06E8D5D8F82835B7
:100A1000C3B1D5F88025D31A642BE0D9FBF780FE4B
:100A200095F84535172BDAD1B8F82C3501339BB240
:100A3000A8F82C35A5F84C35D1E796F83E305A0683
:100A4000E4D5CCE7D5F88035C8F82835C7E700BF2E
:100A50000819002088010020D8220020F83A002040
:100A60002DE9F04FDFF8E4B19BF82E3585B03BB1AE
:100A7000BBF83005003818BF012005B0BDE8F08F85
:100A8000DFF8CCA1DAF8D039197B61B90A22082144
:100A9000CDE90021596A91B1684881420FD0012007
:100AA00005B0BDE8F08F9AF8581A002914BFF62255
:100AB0000822019214BF14220A220092EAE71E6A59
:100AC000002EECD19BF82F155D4BDFF88881BBF829
:100AD0003075C1EB011103EB411903F574730393F6
:100AE000B8F8403007EB53070DF0ECFABBF830359F
:100AF000029001253446BB4257DA0DF0E3FA029B1F
:100B0000C01A009B834250DDBBF830350AEB03006E
:100B100009EB030E90F88CCA19F80300844567D0DE
:100B2000FF285FD005B92EBB0AEB03019EF80160D8
:100B300091F88D1A8E4265D09BF82E160BEB0406A9
:100B400041F0010186F83515042186F83415023488
:100B500001260BEB04014FF0050C81F834C54FEA78
:100B6000132C81F835C54FF0060C043481F8373565
:100B700081F836C5611C0AEB030E0BEB040C5944DB
:100B80008EF88C0A4FF0070E8CF834E5023481F8A9
:100B900034050025B8F8400001339BB29842ABF809
:100BA000303547D9019A9442A5DB002E38D025482C
:100BB000002D3AD0631C0BEB04015B449BF82E56CE
:100BC000042681F83465023483F83455C8F8A0024D
:100BD00001231D491948C8F8A8428AF878350BF056
:100BE0009DF945E74FF0200209F80320202099E7FE
:100BF000002DCFD196B1039A4FF6077111533546A8
:100C00000234C7E70BEB04019BF82E6681F83565CB
:100C1000042681F83465023400269AE70125B9E7F5
:100C2000002C3FF425AF0748D0E74FF60773035376
:100C30000234BFE70023ABF83035B6E7D8220020F6
:100C40005C3C00202C40002028040020F83A0020C2
:100C5000081900208801002008B50120FFF7C8FD11
:100C6000FFF7FEFE0028FBD108BD00BF00B5114B09
:100C700003F5B27C93F82F35C1EB011E1178C3EB5D
:100C800003130CEB431C91B11D2810D84FEA4E0EF4
:100C9000431E73440CF11D006344704401E0834221
:100CA00005D003F8011F12F8011F0029F7D15DF8E4
:100CB00004FB00BFF83A00202DE9F04FA84CD4F80F
:100CC000D0392DED028B5A6A93B081460F46002A27
:100CD00034D004F51D68424500D0FEE71A6A002AA8
:100CE000FCD100239F4A8DF806308DF8073003931E
:100CF0008DF81430069308930B930E9310930123F1
:100D000082F82E350493002209938DF828308DF84F
:100D10003C30954800230DF106050DF1070602A9A8
:100D2000CDE90C23029507960BF0F8F8D4F8D039EA
:100D30005A6A002A32D0424506D0FEE71A6A002AD3
:100D4000FCD1DFF82482CCE71A6A002AFCD1002308
:100D500003938DF81430069308930B930E9310931E
:100D60000123049309938DF828308DF83C30092332
:100D700000228DF806307C488DF80790002302A9E8
:100D8000CDE90C23029507960BF0C8F8D4F8D039BA
:100D90005A6A002A39D0424507D0FEE71A6A002A6B
:100DA000D5D01A6A002AF9D1D1E71A6A002AFCD1F3
:100DB0009FED698BDFF8B0A1013F4FF0000B4FF0C2
:100DC0000A090023012202A95046CDE90832CDE9E3
:100DD0000253CDE9063604928DF814308DF82820A0
:100DE0000B930E938DF83C2010938DED0C8B8DF8AA
:100DF00006908DF807B00BF091F8D4F8D0395A6A04
:100E0000002A33D0424507D0FEE71A6A002ACFD025
:100E10001A6A002AF9D1CBE71A6A002AFCD10B23FF
:100E20008DF80630002317F8012F8DF81430CDE926
:100E30000253CDE9063608930B930E93109302A943
:100E4000012350468DF80720049309938DF828302C
:100E50008DF83C308DED0C8B0BF060F8D4F8D03968
:100E60005A6A002A43D0424507D0FEE71A6A002A90
:100E7000D5D01A6A002AF9D1D1E71A6A002AFCD122
:100E8000D4F86C3D33B19A881B6859690A4214BF83
:100E90005A831A830BF1010BBBF1360F91D100235A
:100EA00003938DF81430069308930B930E931093CD
:100EB0000123049309938DF828308DF83C300823E2
:100EC0008DF80630A02300228DF8073026480295C1
:100ED000002302A9CDE90C2307960BF01FF8D4F8E4
:100EE000D0395A6A002A41D0424507D0FEE71A6A33
:100EF000002AC5D01A6A002AF9D1C1E71A6A002A65
:100F0000FCD1DFF86490A0274FF0000A4FF0000BEF
:100F10000023012202A94846CDE90253CDE9063358
:100F2000CDE9086204928DF814308DF828200B93D7
:100F30000E938DF83C201093CDE90CAB8DF8067024
:100F40000AF0ECFFD4F8D0395A6A1AB3424514D0EB
:100F5000FEE700BFAFF300800000000000000000CB
:100F600008190020F83A0020D82200201A6A002A26
:100F7000C7D01A6A002AF9D1C3E71A6A002AFCD13D
:100F80009DF807309B06C3D4012013B0BDEC028B43
:100F9000BDE8F08F1A6A002AF2D01A6A002AF9D145
:100FA000EEE700BF08B5002103203EF00DFA72B64F
:100FB000FBF7DAFD08B52E4CD4F8302694F8360647
:100FC00052B11168938809690B40002845D1003B54
:100FD00018BF0123002BF3D114200FF069FA254923
:100FE000002000BFD4F8303663B11A689B881569B9
:100FF00094F836262B4062BB003B18BF01230BB18F
:10100000FFF7D0FFD1F88025D1F88435D31A322BE1
:1010100011D8D4F838369342E3D2D1F86C3D33B1CD
:101020001D689B886E69334214BF6B832B833232F9
:10103000C4F83826D5E791F86B3DD1F86C2D03F054
:1010400001031AB17BB9136892881A83C4F8380671
:10105000C7E7B3FA83F35B09D1E7B3FA83F35B091C
:10106000002BADD1B8E7136892885A83EEE700BF32
:10107000F83A00200819002008B544F03DFE1B2076
:101080000CF0DAF908B12923C3801C200CF0D4F944
:1010900008B12923C3800F4B93F84126022A01D0BF
:1010A000012008BD93F86021012A0ED0022AF7D151
:1010B000094AC3F84426094901F12C0047F0DCFA3B
:1010C000074B002083F8230008BD064AC3F84426D6
:1010D000F1E700BFF83A00205004002090040020FF
:1010E00000ED00E07004002000234FF6FF720121A4
:1010F000017243818381C38102828274704700BF81
:10110000154BFF22F0B54FF0000C4FF0FF3EC270C0
:101110000271027242724273827303F10C077646C7
:1011200065466446624602EB820281189F428454FF
:101130004D7081F802C0CE7081F804E00BD093F9B5
:101140000620DC791D7A93F809C093F90A6093F9B7
:101150000BE00633E7E7F0BD4CE705080023022269
:10116000037043708370C3700271704700230122C3
:10117000027043708370C370704700BF4FF4F07209
:1011800002804FF4FA6240F22E4C0921028440F2B0
:1011900026220023A0F81EC081704FF47A7C0E2115
:1011A00082830222A0F822C0437140F2012C8360A6
:1011B000C36080F82410427440F2034140F205629B
:1011C00043820723A0F814C0C1820283837670474C
:1011D0008388C3F30B039342A8BF134670B51A4626
:1011E0001D460C46064680684CF050FC621994423D
:1011F000B569074B08D0074814F8011B00FB03F33F
:10120000A24283EA0103F7D12B60012070BD00BF29
:10121000C59D1C81930100010023037043708370FE
:10122000C37070470023037043708370C3707047AE
:10123000002306214FF47A72C0E901230170037381
:10124000704700BF00234370C37003700371837045
:10125000704700BF10B50023411CFF2200F8132087
:1012600001F813200133082BF8D10B4B4FF0FF315D
:1012700003F10F0400228C4605E093F904C093F9B2
:10128000051013F8032F00F812C000EB420E9C4229
:101290008EF80110F1D110BD60E70508704700BF5E
:1012A0000A44914219D000B501F1FF3C02F1FF3E22
:1012B00041F221011CF8012F082380EA022010F4DA
:1012C000004F81EA40020ABF400090B280B2013B69
:1012D000F5D1E645EED15DF804FB7047704700BFDD
:1012E000D0ED007AD0ED016A30EE677AE6EE877ACB
:1012F000B0EE670AC0ED007A704700BFD0ED017A0A
:10130000D0ED026A30EE677A90ED000AE6EE877A59
:1013100037EEC07AC0ED017AA6EE870A80ED000AAA
:10132000704700BF90ED017AD0ED036AD0ED027AEC
:1013300030EE470AA6EE807A90ED000A80ED017A41
:1013400037EE676AE6EE867A37EEC07AC0ED027A4B
:10135000A6EE870A80ED000A704700BFD0ED056A4F
:10136000D0ED017A90ED007A90ED066AD0ED025A48
:1013700090ED035A80ED050A66EEA77AC0ED066A85
:10138000E7EE007A90ED077AE5EE867A90ED086A4E
:10139000D0ED045A80ED087AE5EE477AE5EEC67A9C
:1013A000B0EE670AC0ED077A704700BFD0ED057A4E
:1013B00090ED006A90ED067AD0ED035AE6EE007AE1
:1013C00090ED016AF0EE406AA6EE267AB0EE670A6A
:1013D000D0ED047A90ED026A67EEC07AA5EEC07A8D
:1013E000E6EE267A80ED057AC0ED067A704700BFFA
:1013F0002DE9F047089F3C460E4614F8011B002BD0
:10140000054614BF4FF030094FF0200941B3002AC0
:101410002CDD234600E0B2B113F8010B9046013AEF
:101420000028F8D1A8F102086AB1C2464946284608
:10143000B0475346002B0AF1FF3AF7DC397828EA27
:10144000E872013249B1D71B2846B047E01914F8B9
:10145000011B0029F8D1BDE8F0871046BDE8F087F0
:10146000002A02F1FF38E0DC0846F4E70022EAE750
:1014700003685A1C02601970704700BF024B18685D
:1014800003681B68184700BFF8470020884210B562
:101490004FF001043ED301FB04F4B0FBF4FC8C4597
:1014A000F9D2CCB122BB08E0A14203F801EBB4FBB6
:1014B000F1F211D8B0FBF2FC1446BCF1090F0CF1AB
:1014C000570E0CF1300204FB1C00EDDCA14203F8C6
:1014D000012BB4FBF1F2EDD900221A7010BDA1422C
:1014E00003F801EBB4FBF1F2F6D8B0FBF2FC1446C2
:1014F000BCF1090F0CF1370E0CF1300204FB1C009B
:10150000EDDCA14203F8012BB4FBF1F2EDD900228E
:101510001A7010BD8446002AEAD1CEE7002870B5C3
:1015200003DA2D2301F8013B4042092886464FF09B
:10153000010307DD03EB83035B00B0FBF3F2092A31
:10154000F8D8EBB1104CBEFBF3FCA4FB0320C008A1
:10155000BCF1090F0CF130060CF15705024607D813
:10156000092B01F8016B03FB1CEE09D90346EAE7DE
:10157000092B01F8015B03FB1CEE01D91346E2E7DE
:1015800000230B7070BD00BFCDCCCCCC0378202BDA
:10159000024600F10100F9D0092BF7D02D2B28D0FD
:1015A0002B2B03BF5378B7EE000A0246B7EE000AB2
:1015B000A3F13001C8B209289FED567A10D8F2EE97
:1015C000046A07EE901AF8EEE77A12F8013FE7EEA8
:1015D000267AA3F13001C8B20928B0EE677AF0D9B3
:1015E0002E2B5ED003F0DF03452B07D020EE070A39
:1015F00070475378BFEE000A0246D9E710B451781D
:101600002D2978D02B296AD0A1F13003092B02F1C2
:1016100001026BD80024002303EB830301EB430397
:1016200012F8011FA1F130000928A3F13003F3D90A
:10163000B3F59A7F1A4628BF4FF49A72072B66D9E2
:10164000DFED356A1346F7EE007A083B072B67EEAD
:10165000A67AFAD802F00702DAB1F2EE046A012A99
:1016600067EEA67A15D0022A67EEA67A11D0032A71
:1016700067EEA67A0DD0042A67EEA67A09D0053A5D
:1016800067EEA67A05D067EEA67A012A18BF67EE44
:10169000A67A6CB387EE277A5DF8044B20EE070A32
:1016A00070475378A3F13001C8B2092802F1010252
:1016B00098D8F2EE046AF0EE665A07EE901AF8EE49
:1016C000E77A12F8013F87EEA66AA3F13001C8B2AB
:1016D000092866EEA56A37EE067AEED982E7917898
:1016E000A1F13003092B02F1020293D9F7EE007A3F
:1016F00027EE277AD0E79178A1F13003092B02F188
:10170000020288BFF7EE007AC4D8012483E7F7EE1F
:10171000007AA1E70000000020BCBE4CF8B5164DD1
:101720006B78BE2B25D1022229464FF6FF70FFF7BA
:10173000B7FD124FAC1C22884AB1A618BE4218D27F
:10174000052A16D92146FFF7ABFD3446F3E72146BB
:101750000222FFF7A5FD0222A118FFF7A1FD063422
:10176000074B641B9C8041F60F53C31A58425841E3
:10177000F8BD0020FCE700BF004000080080000822
:10178000F8470020F0B5067906F0E003402B03D1BE
:1017900044794FF0FF3506E0602B4FF00104F8D19B
:1017A000457904FA05F50023012006F00706A34257
:1017B00000D1F0BD042E0FD8DFE806F00308101D9D
:1017C000240048B1C85CD75C78400FE020B1C8560F
:1017D000D756C71B784278410133E8E70028FBD091
:1017E00031F8130032F81370784080B228420CBFF1
:1017F00001200020F0E70028EED031F9130032F983
:101800001370E6E70028E7D051F8230052F8237060
:10181000DAE7037903F01803102B1CD004D82BB19E
:10182000082B06D000207047182BFBD1B0F80B0016
:1018300070470F4BB0F80B0093F90030591C06BFEE
:101840000C4B1B7ADBB203EB8303C3EB031300EBFC
:10185000430080B27047064BB0F80B0093F901309B
:101860005A1C06BF034B5B7ADBB200EB4310F0E778
:101870003C050020F8470020114B002130B50160E5
:10188000818003F10C054FF448748E460A4602EB42
:10189000420200EB420C00F812E08CF80110DA78FA
:1018A0008CF80220AB42ACF8044007D093F9062034
:1018B00093F807E0197A5C890633E8E730BD00BF8A
:1018C00074E7050801394B0003F00802930001F0AA
:1018D0000301A3EB9203C1EB0111C3EB0313C1EBB3
:1018E000011100229B0089000260818043807047C3
:1018F00000B589B000220DF1100C0492ADF814204F
:1019000003469CE803004FF40070ADF81C101880EB
:10191000BDF81C0098814FF4807E014640F2012002
:101920005A80A3F806E09A60D8811A82A3F814E0DE
:10193000C3F81620598309B05DF804FB144B154910
:1019400010B5044618681B79206284F824301522EB
:1019500004F125004CF03DF90F4B1A7E4FF0010EBB
:1019600084F83AE012B984F83B2010BD03F11C0C56
:10197000BCE80F0020606160A260E360BCE80F007B
:1019800084F83BE020616161A261E36110BD00BFAA
:10199000204F0608284F0608F847002010B5002100
:1019A000382204464CF0D5F80B490C4A0C48C4E9DF
:1019B00004120C490C4AA262C4E90601012341F653
:1019C0001E6CA373A4F826C084F821302146074872
:1019D000BDE810402FF008BE6400DC051A046C0757
:1019E0000019750343080E001E7D0101384F0608DB
:1019F000B5EEC00ADFED347AF1EE10FACCBF30EE6E
:101A0000270A30EE670ADFED317A20EE270A70B53B
:101A1000FDEEC07A86B017EE904A054684EAE4707F
:101A2000002303A9A0EBE470CDE90033029344F056
:101A300059FE002CACBF20232D2303A88DF80030C5
:101A400049F0F6FE01286E4628D0022832D003283D
:101A50001CD003A930464CF084F8304649F0E8FE2B
:101A60000338C4B22246314628464CF00FF8002312
:101A70002B55284649F0DCFE2E232B54013031191A
:101A800028444CF08AF8284606B070BD302303A9DC
:101A900030468DF801304CF064F8DEE743F2300256
:101AA000302303A93046ADF801208DF803304CF007
:101AB00058F8D2E743F2300303A93046ADF80130BD
:101AC0004CF04FF8C9E700BF6F12033A00007A44A8
:101AD0000AF060B913B568B14C1E14F8011F21B9A2
:101AE00002B0BDE810400AF069B901900AF052F95D
:101AF0000198F2E702B010BD08B520214CF040F883
:101B0000034620B11A78202A00F10100F8D01846C7
:101B100008BDF8B5D0B1104B0138C70003EBC000C9
:101B2000CA4390F8406090F8415002F0010282EA06
:101B30000604A5420AD0C06B28B105688088B2426D
:101B400014BF288368833B4483F84140CB0701D40A
:101B5000FDF7DEFBF8BD00BFF84700202DE9F3419B
:101B6000124D134F002305F85C3F044600EB81063D
:101B7000B44203D10F4802B0BDE8F081394628468F
:101B80004BF0EFFF214668464CF007F84FF0000895
:101B9000202168464BF0F4FF28B9694628464BF0EF
:101BA000E0FF0434E4E780F80080F1E7F847002024
:101BB000C190060854480020024BD3F8800038F04A
:101BC00059BA00BFF84700202DE9FF471E46C368F9
:101BD000BDF83070DDF8348004468946924643B340
:101BE000CBB20D2B9ABF1A4AD5560025BAF1FF3F4A
:101BF00021D02368174A3146CDE9005A3846C047FC
:101C0000524620795FFA89F10AF05CF9024600B188
:101C10000288D3B20393C2F30323120BCDE900521F
:101C200002930D4A236831463846C04704B0BDE8E8
:101C3000F0874D1CDAE77B06F8D42368074A0C9539
:101C400031463846C44604B0BDE8F047604700BF9F
:101C5000104F0608AC8F0608B98F0608DD8F0608FE
:101C60002DE9F041154686B06A1C8846BDF8306003
:101C70000D9F194623D0030900F00F044033CDE92E
:101C80000045164A05933046B847A8B198F80510A4
:101C9000D8F800002A460AF03DFC68B102880178B5
:101CA0000391C2F30321120BCDE900420291059B7F
:101CB0000B4A00213046B84706B0BDE8F0817306F4
:101CC000FAD40309074A00F00F000C904033304665
:101CD000BC4606B0BDE8F041604700BFEC8F060887
:101CE000FE8F0608279006082DE9F04188B01E46B1
:101CF00003090E9F9046403300F00F0451B3079341
:101D00000FF078F8027A079BCDE900420546164AA3
:101D100041463046B847D0B128680FF057F9E97905
:101D20006A79DFF854C02D7A079B009411F0020FF6
:101D30004FEA92020D4902F1010208BF6146CDE966
:101D40000102CDE903150A4A00213046B84708B020
:101D5000BDE8F081074A0E9441463046BC4608B0C3
:101D6000BDE8F041604700BF3B900608219206089D
:101D70004D9006086F9006080E9B0608084B09490F
:101D80008B4202460AD2184602E01C30884205D235
:101D90000388C3F30B039A42F7D1704700207047C2
:101DA00064D6060898DE0608F8B50546B0F80900BE
:101DB000084EFFF7E3FF96F8847004462846FFF7C5
:101DC00028FD2FB196F8853013B9E3681844F8BDA3
:101DD000A368FBE7F847002038B505460C46FFF737
:101DE000E3FF2B7903F0E002602A03F0070329D117
:101DF000022BDAB20ED0042A18D03AB96A7901233C
:101E00009340DBB2027814B11343037038BD22EA69
:101E10000303FAE76A79012393409BB2028814B165
:101E200013430380F2E722EA0303FAE76A79012306
:101E300003FA02F2036814B113430360E6E723EAEE
:101E40000203FAE7042BE1D8DFE803F003030505FA
:101E500007000470DAE70480D8E70460D6E700BF23
:101E600070B585880B460446C5F30B052A4600214C
:101E700018464BF06EFE6169084A9142034602D350
:101E8000074A914205D319B1BDE87040184608478A
:101E900070BD2A46BDE870404BF0F8BD98DE0608DC
:101EA00063E0060838B5064C064DAC4206D2A16880
:101EB00020461C34FFF7D4FFAC42F8D338BD00BF36
:101EC00064D6060898DE06084840082310F0800F04
:101ED00082EA40010ABF4000C8B2C0B2013BF5D15E
:101EE000704700BF30B505688D4219D901F1FF3E3A
:101EF0006C1E00231EF801CF082183EA0C0313F0A7
:101F0000800F82EA430C0ABF5B005FFA8CF3DBB2FE
:101F10000139F4D17445EDD16A1C02602B7030BDDB
:101F200000236A1C02602B7030BD00BF07EE901AC0
:101F3000B8EE677ADFED7C7A27EE000A60EE277A4A
:101F4000BDEEE77A17EE103A2033402B00F2DB802B
:101F50009FED767AB4EEC70AF1EE10FAB0EE677A2A
:101F60000CDDDFED735A9FED736AF0EE476AF4EE15
:101F7000C66AF1EE10FA37EE657AF6DCDFED6E6ACE
:101F8000B4EEE67AF1EE10FA0CD5DFED695A9FED6A
:101F90006B6AF0EE476AF4EEC66AF1EE10FA37EEBD
:101FA000257AF6D4DFED666AB4EEE67AF1EE10FA41
:101FB00000F39D80DFED636AB4EEE67AF1EE10FA8D
:101FC00044BFDFED5D6A36EEC77A27EE075ADFEDD4
:101FD0005E5A9FED5E6ADFED5E6ADFED5E4AA5EE5A
:101FE000256A27EE054AE5EE066AF7EE005AA4EEEA
:101FF000267AF0EE656AE7EE646AE7EE245A86EE2A
:10200000A54A9FED4F7A77EE877ABDEEE77A17EE15
:10201000103A2033402B6FD89FED4F7AB4EEC70AA9
:10202000F1EE10FA0CDD9FED426ADFED426AB0EE90
:10203000677AB4EEE67AF1EE10FA77EEC67AF6DC5D
:102040009FED3D7AF4EEC77AF1EE10FA0CD59FEDD4
:10205000386ADFED3A6AB0EE677AB4EEE67AF1EE0E
:1020600010FA77EE867AF6D49FED357AF4EEC77AD9
:10207000F1EE10FA4CDD9FED397A77EE677A67EE74
:10208000A74A9FED317A9FED315ADFED316AA4EE18
:10209000875A67EEA43AE4EE856AB7EE006AE3EE8B
:1020A000A67AB6EE007A36EE676AB8EE005A67EEA8
:1020B000857A26EE077AB7EE005AC5EE256A002328
:1020C000836143610362C36180ED044A26EE877A2F
:1020D00026EE866A66EEA77A80ED095A80ED007AD0
:1020E00080ED016A80ED027AC0ED037A7047DFED82
:1020F0001B6A36EEC77A68E7DFED197AB6EE007A2A
:10210000B7EE006AD7E7B7EE004AF0EE445A78E738
:102110009FED0C7AF4EEC77AF1EE10FA44BF9FED12
:10212000067A77EE677AAAE727D4D2360024F448F5
:10213000DB0FC940E4CB1641DB0F49C0E4CB16C12D
:10214000DB0FC93FDB0FC9BF92E741B99730083CAD
:1021500015A82ABEF304353F00247448DB0F49401C
:1021600000000000DFED277AB4EEE70AF1EE10FA86
:102170000CDDDFED256A9FED257AF0EE407AF4EE76
:10218000C77AF1EE10FA30EE660AF6DCDFED207A5F
:10219000B4EEE70AF1EE10FA0CD5DFED1B6A9FED05
:1021A0001D7AF0EE407AF4EEC77AF1EE10FA30EED6
:1021B000260AF6D4DFED187AB4EEE70AF1EE10FA4B
:1021C00014DDDFED107A37EEC00A60EE006A9FED95
:1021D000136A9FED137ADFED137AA6EE867A20EE6E
:1021E000266AE6EE877AA6EE270A7047DFED0E7ABA
:1021F000B4EEE70AF1EE10FA44BFDFED057A37EEF0
:10220000C00AE2E7DB0F4940DB0FC940E4CB1641CF
:10221000DB0F49C0E4CB16C1DB0FC93F92E741B9E0
:102220009730083C15A82ABEDB0FC9BFF0EEC07A74
:10223000B0EEE07AB4EEE77AF1EE10FAB4BFB0EEA9
:10224000676AB0EE476AB5EE406AF1EE10FA46D022
:10225000B4EEE77AF1EE10FA8CBFF0EE675AF0EECA
:10226000475AC5EE866ADFED1F2ADFED1F3ADFED24
:102270001F4A9FED1F5A9FED1F3A9FED1F4ADFED4A
:102280001F5AE6EEE23AA6EE834AE6EEA34AB7EE1E
:10229000006AA6EEA45AA6EE846AE6EE855AC5EE5A
:1022A000866AB4EEE77AF1EE10FA48BFDFED147AF1
:1022B000F5EEC00A48BF77EEE66AF1EE10FA48BFC5
:1022C000DFED107AB5EEC00A48BF77EEE66AF1EEB0
:1022D00010FA48BFF1EE666AB0EE660A7047DFEDAD
:1022E000076ADEE739094E3DE3B59E3E88FA163EA1
:1022F00045FE7F3F99FB243F69A2163EA7DFA83425
:10230000DB0FC93FDB0F494090ED005A9FED4C0AAF
:1023100035EE000A08B5FDEEC07A17EE903A20338C
:10232000402B7BD8FFF71EFFF0EE403AFDEEC57A5A
:1023300017EE903A2033402B7FD8B0EE450AFFF7D6
:1023400011FFB0EE405AD0ED014A9FED3D0A34EE48
:10235000800AFDEEC07A17EE903A2033402B69D800
:10236000FFF700FFF0EE405AFDEEE47A17EE903AE8
:102370002033402B5BD8B0EE640AFFF7F3FEF0EE9B
:10238000404A90ED023A9FED2E0A33EE000AFDEE30
:10239000C07A17EE903A2033402B45D8FFF7E2FE83
:1023A000B0EE404AFDEEC37A17EE903A2033402B50
:1023B00037D8B0EE430AFFF7D5FEF0EE407A24EEB0
:1023C000233A27EEA36A24EE057A67EE856AB0EE1B
:1023D000462AF0EE432AA7EE242AE6EEE42AA6EEE9
:1023E000247AE3EE646A24EE254A65EEE77A25EE68
:1023F000655A65EEA35A81ED004AC1ED017AC1ED3F
:10240000024A81ED032AC1ED042A81ED055AC1ED8E
:10241000066A81ED077AC1ED085A08BDDFED093A79
:1024200084E7DFED087ACAE79FED064ABAE7DFEDF9
:10243000054AA6E7DFED035A96E79FED025A82E7C9
:10244000DB0FC93F000000002DE9F04389B0541CA8
:1024500003941478002C00F0078100250746884675
:102460001E46A94609E021463846C047039A013571
:10247000531C03931478002C3DD0252CF3D1931CCE
:10248000CDE903395078302800F09480A0F1300372
:10249000DBB2092B4FF0000440F297806C2838D053
:1024A000782822D857282AD9A0F15803202B1CD8E5
:1024B000DFE803F0B41B1B1B1B1B1B1B1B1B1B950B
:1024C0009D1B1B1B1B1B1B1B1B1BAF1B1B1B1B1150
:1024D0001BA71B1BB40056F8043B049A009300236F
:1024E00041463846FEF784FF0544039A531C039384
:1024F0001478002CC1D1284609B0BDE8F08300282B
:10250000F9D02528F1D125213846C0470135039A55
:10251000AEE7039B5A1C039219787829A8D857294B
:1025200058D9A1F15803202BA2D801A050F823F0CC
:10253000352601087124010871240108712401085D
:102540007124010871240108712401087124010813
:10255000712401087124010871240108DF25010894
:102560004D26010871240108712401087124010815
:1025700071240108712401087124010871240108E3
:10258000712401087124010815260108712401082D
:10259000712401087124010871240108D72401085D
:1025A00071240108592601087124010871240108C9
:1025B00035260108D31C03939078A0F13003DBB2D9
:1025C000092B4FF001043FF669AF04AA03A944F0B8
:1025D0003FFA63E700298ED0252994D048E756F8C2
:1025E000041B3846C9B2C0470135039A40E756F884
:1025F000040B05A9FEF792FF05AB0093049A23464E
:102600006EE756F8040B05AB00220A21FEF73EFFE9
:10261000F2E7039A56F8043B1D6029E7A0F158023F
:10262000B2FA82F256F8040B520905AB1021FEF7FC
:102630002DFFE1E7A1F15802B2FA82F256F8040B3D
:10264000520905AB1021FEF721FFD5E756F8040B20
:1026500005A9FEF763FFCFE756F8040B05AB002290
:102660000A21FEF713FFC7E7254644E773B5144C6C
:1026700001920646D4F888000D46C0B11149FFF713
:1026800029FAD4F888003146FFF724FA0E49D4F825
:102690008800FFF71FFA0D49019BD4F888002A46ED
:1026A000FFF7D2FE0A49D4F88800FFF713FA94F82E
:1026B0008C3013B1012384F88D3002B070BD00BF9F
:1026C000F847002081900608A2970608D11A010851
:1026D000F59906080EB400B584B005AB019053F827
:1026E000042B0649039301A8FFF7AEFE019B0022CD
:1026F0001A7004B05DF804EB03B070477114010860
:102700002DE9F043002483B006460480214630467C
:10271000013436F035FF082CF8D10023DFF868804B
:1027200086F8EA30C6F8EC30C6F8F030C6F8F43077
:10273000C6F8F8301F46FC3699463A46414601A88D
:10274000FFF7C8FF3546032401AA12F8013B6BB11D
:10275000013C05F8013BF8D10137082F85F80090BE
:1027600006F10406E9D103B0BDE8F083284622460D
:102770002021254401374BF0ECF9082F85F8009013
:1027800006F10406D9D1EEE7444F0608F7B5114E1D
:1027900007463046002300F88E3F0C460E4B0F498B
:1027A000002F08BF194615464BF0DBF90C4F04EB20
:1027B00045058E36AC4202D10A4803B0F0BD394619
:1027C00034F8022B6846FFF785FF694630464BF028
:1027D000C8F9EFE7F8470020979006088E900608A2
:1027E000A090060886480020F7B50C4E0C4F002339
:1027F00006F8BF3F044600EB4105AC4202D1094850
:1028000003B0F0BD394634F8022B6846FFF762FF8B
:10281000694630464BF0A5F9EFE700BFF8470020C6
:10282000CB910608B7480020F8B5084F4E1E054664
:1028300001F11F0416F8012F28463946FFF74AFF19
:10284000A64205F10205F5D1F8BD00BFA590060826
:102850000246531C084605D1034B1A681B790A60CF
:102860000B717047014935E7E78F0608CC910608E0
:1028700010B5013114460EF0BDFA28B9054B1A689F
:102880001B792260237110BD027A03492046BDE8FE
:1028900010401FE7E78F06084890060803685A1C97
:1028A000026019700368090A5A1C026019707047A7
:1028B00002681146531C036011F802CB0160D31C5F
:1028C0005178036093781B0443EA0123111D0160D2
:1028D000D07843EA0C0343EA00607047A0F130036C
:1028E000092B07D920F02000413819288CBF00207F
:1028F0000120704701207047303809288CBF002024
:1029000001207047413819288CBF002001207047F2
:10291000613819288CBF002001207047202805D07D
:10292000093804288CBF002001207047012070471F
:10293000A0F14103192B98BF20307047A0F161032B
:10294000192B98BF2038704710B500F1004402469B
:10295000013C04E0B3EB0E0015D1A24214D012F8F2
:10296000013BA3F14100192811F8010BA0F1410C22
:1029700098BF2033BCF1190F00F1200EEAD91B1AC1
:1029800004D10028E9D110BD002010BD184610BDAB
:1029900002B310B58446841804E0B3EB0E0014D1E2
:1029A000A44513D01CF8013B11F8010BA3F141021F
:1029B000192AA0F1410298BF2033192A00F1200EF4
:1029C000EBD91B1A04D10028EAD110BD002010BD9C
:1029D000184610BD1046704770B5044608460D46AF
:1029E00048F026FF064602E014F8013F43B12046B6
:1029F00032462946FFF7CCFF0028F5D1204670BDAE
:102A00001C46204670BD38B507490546FFF7E4FF70
:102A10000649041E284618BF0124FFF7DDFF08B150
:102A200044F00204204638BDAA900608E0A5060836
:102A30002DE9F041044686469EF800C0BCF1200F07
:102A40007046ACF109050EF1010EF5D0042DF3D955
:102A5000BCF12B0F5BD0BCF12D0F3BD1102A4FF0F6
:102A6000010600F1010E58D19EF800C0BCF1300FF4
:102A70005FD04FF010086FF070450F2742460EF1FF
:102A8000010E00200DE0ACF1300C5FFA8CFC944597
:102A90000FDA854274462DD32AD008FB00C01EF8F9
:102AA00001CBBCF1390FEED94CF0200CBCF1600F1A
:102AB0000BD801B10C600EB323B1B0F1004F28BFA9
:102AC0004FF000404042BDE8F081ACF1570C5FFA96
:102AD0008CFCDCE7102A864649D04FF0FF35B5FB69
:102AE000F2F502FB05F7FF43FFB290460026C6E76A
:102AF0006745D2D21E404FF0FF30D0E7002BE2D026
:102B00006FF00043984228BF1846BDE8F081102AB4
:102B10004FF0000600F1010EA6D04FF0FF35B5FBD7
:102B2000F2F502FB05F7FF4390F801C0FFB29046B3
:102B3000A5E79EF801C0ACF1410019280EF101048F
:102B4000624601D80CF12002782A4FF0100805D017
:102B5000A6466FF070450F27424690E79EF802C0E8
:102B60006FF070450EF1020E0F27424687E70026F0
:102B70007AE700BF01230A22002159E770B50D460C
:102B80001446FEF7B9FF0646A0B1FFF7F3FF40F683
:102B900034039842A8BF1846B0F5617FB8BF4FF420
:102BA0006170A0F561731920B3FBF0F32B702378EB
:102BB000013323703046FEF79FFF0646A0B1FFF7B2
:102BC000D9FF40F634039842A8BF1846B0F5617F9C
:102BD000B8BF4FF46170A0F561731920B3FBF0F337
:102BE0006B70237801332370304670BD10B40288B7
:102BF000C378174CA2F5FA6202F0030140F2B55C0B
:102C00009208013B0CFB0233827801EB4101013A4F
:102C100002EB810204EB420102798C8F417923445B
:102C200003EB430302EBC30384790A4A0089C3EB35
:102C3000031301EB8303C3EB0313224402EB830270
:102C400000214FF47A73C2FB03015DF8044B704717
:102C50004CE7050880436D382DE9F04117461E46C4
:102C600005464FF47A7200233846314649F03EFA61
:102C70004349444A014482FB0143C8170B44C0EB5B
:102C8000631382FB03021A44D8173F4CC0EB621255
:102C900084FB02044FEAE27C3C48CCEBA40C80FBB2
:102CA0000C404FEAEC74C4EBE010C3EB0314A1EB4F
:102CB0008401A971C2EB0211A3EB81036B710CEBD0
:102CC0004C03A2EBC30240F2B55303FB10CCBCF59E
:102CD000896F2A714FEA800044DA40F2DA239C457A
:102CE00047DCBCF5B77FB4BF00220122284B02EBC2
:102CF000420103EBC1034FEA4208B3F8523091B2EC
:102D0000244C08EB020E04EBCE0416344FF00B0EED
:102D100001E034F8023D63451FDDBEF1010EF8D13C
:102D20001B4B424403EBC2024FF0010E938F85F818
:102D300002E000F5FA600CF1010C0844ACEB030C66
:102D4000288085F803C04FF47A7200233846314654
:102D500049F0CCF92A81BDE8F0810EF1010E5FFA4D
:102D60008EFEE4E7032140F296530A464FF0060830
:102D7000C6E7022140F229430A464FF00408BFE7A4
:102D800080BC92C789888888ABAAAA2A73B06D16BE
:102D90004CE7050888E7050808B50C4BD3E93A234A
:102DA00052EA030C09D1002340F2011242808380D1
:102DB000837103800381184608BD054909688A1894
:102DC00043F10003FFF748FF012008BDF84700204A
:102DD000881E002090422DE9F0410B46044615461E
:102DE0000AD2B0FBF5F6134A05FB16441846135DEC
:102DF00000F8013BBDE8F081B0FBF2F69642B6FB6D
:102E0000F2F706D20B4A05FB1767D15D03F8011BE9
:102E1000EAE7BA42B7FBF2F807D9064A05FB187889
:102E200012F8081003F8011BEDE74046FFF7D2FF48
:102E30000346F2E74C4F0608774B9A88B3F808C070
:102E400058899989B2F57A7F88BF4FF47A7210B5A4
:102E500088BF9A80DA88B2F57A7F84BF4FF47A729D
:102E6000DA80BCF57A7F84BF4FF47A7CA3F808C07F
:102E7000B0F57A7F88BF0020DA8988BF5881B1F524
:102E80007A7F84BF4FF47A719981B2F57A7F84BFDB
:102E90000022DA8184459CBF00201881914298BFAE
:102EA0000022598B98BF9A819A8B914284BF00224D
:102EB0005A835A4B1A8882B0002A63D0584CA179A1
:102EC000A378002977D1062B97BF56489FED560A65
:102ED00000EB830090ED270A207900284ED1534B58
:102EE00093F8C80307EE902A07EE100AF8EEE77A87
:102EF000F8EEC76A86EEA77A002972D1B4EEC70A47
:102F0000F1EE10FA3FDD67EE807ABCEEE77A8DEDE8
:102F1000017A9DF8041007EE101AB8EEC77AF4EEA5
:102F2000C77AF1EE10FAC4BF0131C9B2002970D0DE
:102F30001029A8BF1021C9B20A4681423C4938BFB6
:102F4000024683F8C8234A79012A20D100224A7117
:102F50005A7A032A2BD8374901EB42111A7AC3F85F
:102F6000D013032A1CD8344902EB8202C2EB0212AE
:102F700001EB4202C3F8D42302B010BD042B38D8B1
:102F8000002B39D1294B2A494A79012ADED0022A5D
:102F9000DED12A4A1279002ADAD100224A71D7E713
:102FA000254AC3F8D4230021197202B010BD0022B3
:102FB00020495A72D2E7072B85D123790621A170C7
:102FC000002BDFD1194B9FED1E0A93F8C80307EEC3
:102FD000902A07EE100AF8EEE77AF8EEC76A86EE56
:102FE000A77A30EE000AB4EEC70AF1EE10FACADD95
:102FF00089E7053B032BC5D9F7EE007A87EE800AF7
:103000004AF0CCF82288094B904228BF1046208015
:10301000B9E701218FE700BF6C220020840A00106D
:10302000EC2600204CE705086F120338F847002013
:1030300034410020E848002068490020543C00202A
:1030400017B7D1382DE9F04F9B4E85B096F8D8339D
:10305000A3F11702022A00AF00F29582974BBB60E2
:10306000DFF8608296F8E813DFF870B2944D08F14B
:103070006C0944464FF0000A2FE00AF1010A5FFA9A
:103080008AFA4308820802F0333203F0773313449C
:10309000C20802F01132C31A9B1A03EB131303F098
:1030A0000F33ABFB03E2D209C2EB02229A1A83036D
:1030B00001D5012A19D0012A0BD9082A15D8BCF14B
:1030C000000F01D0284204D1F96047F0AFFFF96842
:1030D00058B10C344C4500F04F82206810F0010CC0
:1030E000CBD194F90430142BCBD176480FF074FB7C
:1030F0000024022086F8884411F0F0FE96F88C3403
:10310000022B00F0D482002800F028836E4B96F842
:1031100015A503F5167B4FF47A7E4FF0000C5A8804
:10312000B2F57A7FB3F8462088BFA3F802E0B2F583
:103130007A7F9A8888BFA3F846E0B2F57A7FDA886A
:1031400088BFA3F804E09988B2F57A7F84BF002293
:10315000A3F806C09142B3F85A10B3F85C2098BFA8
:10316000A3F804C0914293F86B2088BFA3F85AC01B
:10317000013A632A84BF642283F86B2093F86C20A1
:103180000132D2B2092A88BF83F86CC003F166000D
:10319000194600228D7A10F8014B0132A54238BF42
:1031A00000F801CC032A01F10601F3D1BAF1010FB5
:1031B00018BF83F884C096335B45B0D1434B9B78EE
:1031C000042B00F0A8823BB9404A1388B3F5F07F86
:1031D00084BF4FF4F0731380FFF72EFE96F82F157F
:1031E000092902D0002940F0E48196F83D1509290B
:1031F00002D0002940F0D981B6F84A25B6F8483502
:103200001343B6F84C2513431BB213B10123A6F8A0
:103210004E35D6F804352E4A1A40002A00F0B48202
:10322000DA0700F12B825D0440F1C7812949D6F805
:1032300008250B400A40C6F80435C6F8082513F4E3
:10324000004200F0FE81002286F8EF2386F8FF237B
:10325000D90440F1008296F85B35DFF87CB0022B90
:1032600004BF012386F85B350BF178045B4602E06E
:103270000633A3420CD01A78072AF9D19978DA7864
:10328000914202D35A79002AF2D0072024F056FE48
:1032900000234FF4806086F8883411F01FFE002868
:1032A00000F04F820C4DAA469AF8051019B39AF80F
:1032B0000000F0B15B4616E0F84700204CE7050837
:1032C000BC020200104C002068490020EC260020BF
:1032D00009600002F6DFFFFD584D002081808080EC
:1032E0000633A34207D01A788A42F9D15A79002AC4
:1032F000F6D024F023FE0AF1060AA245D4D1BA4B37
:1033000093F802B0BBF1080F00F0C681D6F804357F
:10331000B649D6F808250B40C6F8043596F8153599
:10332000A3F10103B3FA83F35B0986F8D83596F865
:103330001635A3F10103B3FA83F35B0986F8DC3594
:10334000B6F8F0351140C2F3C032C6F8081586F859
:10335000DA25002B40F0C981D6F8F43513F07F4F01
:103360001CBF0023C6F8F435D6F8FC3523F40073EF
:1033700023F0020313B10023C6F8FC3596F8F835A4
:10338000013B042B84BF012386F8F835ABF1050B14
:10339000974BBBF1030F93F8901540F2498111B39D
:1033A0000023FB60904B7C606FF00702A2EB030AE6
:1033B000544603F1080B8A4604E004EB0B03534523
:1033C00080F0FF801BF8010B0028F6D00DF03AFDCD
:1033D0000028F2D0C3799B07EFD5FA687C680123F7
:1033E000002A40F0F480804B9B7913B17E4A002381
:1033F0009371B6F8063613F00C0F03D1C3F3031321
:10340000022B03D94FF42063A6F80636B6F8083627
:1034100013F00C0F03D1C3F30313022B03D940F6AF
:103420000123A6F8083696F8813696F875269A4252
:1034300096F8743605D9002286F8752653B1A6F899
:10344000782696F880269A4204D2002386F87436AD
:10345000A6F8783696F86A3796F876266548FC60BE
:103460009A4288BF0023BC6888BF86F8763600F190
:10347000800B10F8043C03EB4303234493F890A122
:1034800093F891E193F892C1C31E1A785245A8BFF0
:10349000524603F8012B59799A787145A8BF7146B5
:1034A0006245A8BF6246984259719A70EDD12030AA
:1034B0005845DED1D6F81024FC68002A00F01F81A0
:1034C0004FF0000C012002E00635A54211D02B7808
:1034D000282BF9D16B7800FA03F11142F4D00433B0
:1034E000063500FA03F3A54222EA03024FF0010C6D
:1034F000EDD1BCF1000F01D0C6F810243E4C04F110
:103500000805234613F8012B072A00F283809D4209
:10351000F8D1EA4688B0EB462022FF2158464AF00F
:1035200018FB354A12F8013B5BF82310013178D1C2
:1035300095424BF82330F5D1B6F80E25B6F80C3588
:103540009A42D54602D32D4BC6F80C35FF232C49A1
:1035500086F89C3798F90430142B05D0D8F8002051
:1035600031EA020200F0D18008F10C08C845F1D11F
:103570001437BD46BDE8F08F0AF1FF3ABAF1020FE9
:103580007FF6B6ADB1E51F4ABA6002EBC30393F80C
:10359000B820002A3FF464ADD3F8BC30002B7FF490
:1035A0005FAD172386F8D8335AE51748FEF78AF936
:1035B00022E61648FEF786F917E61C0767D5144978
:1035C00035E6FA687C680023002A3FF40CAF064910
:1035D0004A7C002A7FF40DAF4A79012A3FF403AFF9
:1035E000002B7FF400AF04E7EC260020DEDFCDFDEA
:1035F000840A0010EE480020FF260020AE014A0198
:10360000010002004CE70508364D0020284D00203F
:10361000FE9FFFFDEA4688B02022FF2168464AF05F
:1036200098FA002304F8013B0133082BFAD183E711
:103630005B4A00231371002900F09D800123FB6089
:10364000B0E696F8EF1300293FF402AED90486F8ED
:10365000FF233FF500AE1A067FF5FDAD96F8D813AF
:10366000182906D84F4B01228A401340002B7FF4C3
:10367000F2ADDFF840B10BF1780409E64A49D6F81B
:1036800008250B400A40C6F80435C6F808259804FA
:103690007FF5D5AD4549CAE51A469B79002B3FF425
:1036A00035AE537C012B04BF022353742EE6002851
:1036B0003FF42CAD3E4B96F8951490F904504FF022
:1036C000FF0C03F16C0093F90820AA4204D10139E0
:1036D00083F808C0C9B201240C338342F3D1002C13
:1036E0003FF414AD86F8951410E596F8EC050DF04E
:1036F000A9FB00287FF430AEA6F8F0052CE62820C0
:1037000024F01CFCD6F81024DAE6143786F89C372F
:10371000BD46BDE8F08FD6F80435214A23F4805326
:10372000C6F80435D6F8083523F48053C6F80835B2
:10373000538CB3F57A7FBFF44FAD4FF47A73538453
:103740004AE5D6F8043523F00063C6F80435D6F808
:10375000083523F00063C6F80835A3E5D6F804253C
:10376000D6F8083522F0800223F08003C6F804253D
:10377000C6F80835CAE4537C002B7FF43AAE53797F
:10378000012B7FF436AE2EE6D6F8082543F0080369
:1037900042F00802C6F80435C6F8082540E500BF27
:1037A000EC26002000410001F79FFFFDF6BFFFFD62
:1037B000904C0020584D00202DE9F04F754F764B6E
:1037C000D7F8AC2702F2DC52C7F8AC27734A934211
:1037D00083B080F0DB8003F11C059B46704B714E7B
:1037E0004FF0010A03F102086D4B5A88002A00F0DD
:1037F000B68008EB0203B34280F0B180444608E093
:103800001A881C461344002A00F0A980B34280F0B5
:10381000A680052A40F2A38035F81C2C6188C2F3EB
:103820000B029142ECD162799207E9D1238855F8D5
:10383000141C94F8049001935846FEF711FB35F8D8
:103840001C2CB9EB123F00F092804FF0000A35F8C3
:10385000181C55F8140CC1F30B0144F073F955F81A
:10386000043C18604D4B0BF11C0B9B4505F11C05EE
:10387000BAD3D7F80435C7F80835FFF7E3FB3B7A2E
:10388000494D797A494C03EB8303C3EB0313A5F14C
:10389000800202EB411205EB4303C7E9F42323F056
:1038A000E7FD4FF0FF33D7F8D40363602DF0DEF867
:1038B00024F098FB05F57C7305F58D6102E0063375
:1038C0008B425ED01A78002AF9D19D78D87885424B
:1038D00002D358790028F2D097F85835227203EBBA
:1038E000830303EB83039B00C72BD8BFC823C7F810
:1038F000A437B7F85C352E49642202FB03F3C72BCB
:10390000D8BFC8230022C7F8A837C7F8C037294B4B
:10391000C7F8AC27C7F8B027C7F8B427C7F8B82747
:10392000C7F8BC27A7F8C42787F8C627C1F804370B
:103930002DF0F8FEB7F8C80797F8CA1726F0AEFAC8
:1039400036F026FC17F0B4FF1B4A1268C7F8AC2704
:103950000123504687F8C53703B0BDE8F08F55F80E
:10396000141C5846FEF77CFA4FF0000A6FE7019BE3
:10397000A11D9A1F5846FDF72BFC00287FF467AF66
:1039800063E7FA7D003A18BF0122A5E74FF0010A6C
:103990006FE700BFF847002064D6060898DE0608E7
:1039A0000040000800800008684900203C05002015
:1039B000840A0010404D0020881E00201C4B01226C
:1039C000032870B51B4D83F80C2706461ED9711CC1
:1039D000C9B249004029184A28BF402100230224C7
:1039E0004FF0140ED454023302EB030C99420CF83E
:1039F00001ECF7D8FF2E08BF02212944FF2381F8EC
:103A0000CC37BDE870400E2016F0D0BA00EB800035
:103A100005F5B873C0EB001003EB4000C5F8D40304
:103A20002E722DF023F826F01DFD26F0F1FDCEE7D5
:103A3000840A0010F8470020C44F0020054BD3F83B
:103A40001028012142F4001283F80D18C3F8102841
:103A5000704700BFF8470020F8B50468C4F30D04B0
:103A600006460F460CB335683F683DF031FD092826
:103A700040F08780444C236923F440732361236919
:103A800043F400732361236943F0010323612F6032
:103A90003DF01EFD2369092823F00103236170D145
:103AA000336804333360002034E0384B384A9342A3
:103AB0002AD302F58042934225D302F580429342F5
:103AC00029D3344A934228D902F58032934226D929
:103AD00002F50032934224D902F50032934222D9F2
:103AE00002F50032934220D902F5003293421ED9EA
:103AF00002F5802293421CD9B3F1016F1BD346F02B
:103B000049FA47F08DFE08243DF0E2FC092814D064
:103B10004FF0FF30F8BD1024F6E71824F4E7202416
:103B2000F2E72824F0E73024EEE73824ECE74024DD
:103B3000EAE74824E8E75824E6E7134D2B6923F425
:103B400040732B612B6943F400732B612B6923F0C5
:103B5000F8032B612B691C4344F002042C612B6990
:103B600043F480332B613DF0B3FC2B6923F0020357
:103B70002B612B69092823F0F8032B613FF473AF05
:103B8000C6E76FF00100C5E7003C024000400008B6
:103B900000400008FFFF00082DE9F041574F3B7837
:103BA000AF2B8AB06FD1FDF7B9FD80F00104E4B20C
:103BB000534B544DB3F89F31534EADF8003004F0E1
:103BC0000104B54261D3002C00F096801022002140
:103BD00006A849F0BEFF4D4B0497DB1B05934C4BE9
:103BE0001A69002A04DA4B4A5A6002F188325A6094
:103BF00001228DF82420F322DA606946022204A80B
:103C00000025089547F0C6FC022269464FF6FF7072
:103C1000FDF746FB3B4F0446B74243D3022201A9BE
:103C200004A80025ADF8045047F0B4FC022201A915
:103C30002046FDF735FB40BAC043ADF8080002222C
:103C400004A802A947F0A6FC079868B106ABC0F12A
:103C500004022946184449F07CFF089818B906A9BF
:103C600004A8FFF7F9FE08909DF82430089823B1C6
:103C7000274A136943F000431361B0FA80F040090A
:103C80000AB0BDE8F081012492E7A988A868C1F3D1
:103C90000B0143F057FFAB691B681C35834218BF0B
:103CA00001248EE7B7F804808DF80D50C8F30B0897
:103CB00008F10603ADF808303B88C3F30B02ADF8FA
:103CC0000A201B0B062202A904A88DF80C3047F02D
:103CD00061FC062202A92046FDF7E2FAB968044613
:103CE000424604A847F056FCB96820464246FDF714
:103CF000D7FA1C3704468FE70120C1E700400008CF
:103D00004CE7050864D6060898DE0608008000081F
:103D1000003C02402301674510B5194CFFF792F9AA
:103D2000D4F8AC37012203F2DC53C4F8AC3784F882
:103D30001428FFF731FF10B9FFF72EFF50B1114BD8
:103D40001B78AF2B02D1FDF7E9FC58B946F022F9F8
:103D500047F066FDFFF720FF0028F0D146F01AF982
:103D600047F05EFD084A0023116884F814380122E8
:103D7000C4F8AC1784F8C52784F8153810BD00BF07
:103D8000F847002000400008881E002010B50B4AAC
:103D90000B4C02230121A37582F80C17FFF7BCFF1F
:103DA000FFF70AFD41F20242FF23A4F8CC2784F872
:103DB000CE370E20BDE8104016F0F8B8840A001087
:103DC000F847002090F88630DFED6A5A03EE903A0B
:103DD00090F88A3006EE103A90F8883004EE103AE7
:103DE00090F88930F8EEE33A04EE903A90F88C308F
:103DF00063EEA57AB8EEC66A03EE903A26EE256A1F
:103E0000B8EEC44AF8EEE44AF8EEE33A26EE276A42
:103E100024EE254A64EEA54A63EEA53AF0B5564D68
:103E200024EE064A64EEA74A63EEA73A002106266E
:103E3000F7EE002AA5F10C0C00F1660E06FB01F26C
:103E4000B7EE005AAC1890F885700244F0EE456A5F
:103E500015E0012904F1060402F10602EED190F802
:103E6000873007EE903A90F88F3006EE903AF8EEF1
:103E7000E77AF8EEE66A27EEA55A66EEA56A237899
:103E800007EE103A66EE867AB8EEC77A27EE277A02
:103E9000FDEEC77A17EE903AFA2BA8BFFA2323EA71
:103EA000E3731372637807EE103A66EE847AB8EE25
:103EB000C77A27EE277AFDEEC77A17EE903AFA2BEB
:103EC000A8BFFA2323EAE37353725CF8213007EEAC
:103ED000903A002BF8EEE77A49DDA37807EE103A26
:103EE000B8EE477A90F88B3037EE677A03EE103AE7
:103EF00087EE272AB8EEC33AB0EE627A23EE253A6F
:103F0000A2EE037A64EEA77A66EEA36A67EE857A7C
:103F100027EE877AFDEEE77ABDEEC77A17EE103A04
:103F2000FA2BA8BFFA2323EAE373937217EE903AB1
:103F3000FA2BA8BFFA2323EAE3730EF80130A38813
:103F400007EE903AF8EEE77A013167EEA67AFDEED9
:103F5000E77A17EE903AB3F57A7FA8BF4FF47A73F9
:103F600023EAE3738F429381BFF673AFF0BDB7EEE0
:103F7000007AC7E70AD7233C28EB050890F88D3074
:103F80006BB3B0F85A308BB190F88E2002EB8203FD
:103F90006421C3EB0313B3FBF1F3A0F85A3096236B
:103FA00012FB03F3B3FBF1F3A0F85C3043884BB191
:103FB00090F88E3003EB8303C3EB03136422B3FB4F
:103FC000F2F34380B0F846304BB190F88E30962231
:103FD00013FB02F36422B3FBF2F3A0F84630704700
:103FE00090F821304BB3438B83B190F82230FA2202
:103FF00013FB02F203EB8303B3F57A7FA8BF4FF400
:104000007A7364218383B2FBF1F24283838843B1E4
:1040100090F82230FA2213FB02F36422B3FBF2F38E
:104020008380C3884BB190F8223003EB8303B3F550
:104030007A7FA8BF4FF47A73C3807047034BD3F8DD
:10404000180D08B107F0BABE704700BFF84700204E
:1040500008B50B4605490246D1F8180D28B10449A8
:10406000FEF7F2F9BDE80840E8E708BDF847002090
:10407000D11A0108024B0146D3F8180DFDF72ABDED
:10408000F847002008B504460848FFF7F3FFFFF79C
:10409000D5FF074BD3F8800015F006FF0CF0F4F9BC
:1040A000012C01D147F0BCFBFBF732F9B2900608B6
:1040B000F84700200048DDE70C9B06080CB4C30657
:1040C00007B500D561B9049805A90191FFF7C0FFB4
:1040D000FFF7F0FF012003B05DF804EB02B070477A
:1040E0000020F8E708B5FFF7C5FFBDE80840E1E7A5
:1040F00010B504460348FFF7BDFF2046BDE8104059
:10410000F0E700BFBE90060808B50948FFF7F0FFCA
:10411000FFF794FF074B002483F81C4DC3F81C4E97
:1041200083F8204E26F014FB2046FFF7ABFF00BFBC
:10413000C3900608F8470020034B0146D3F8180D3A
:1041400008B107F027BE7047F84700200CB407B548
:1041500010F020000BD079B92320FFF7EDFF049871
:1041600005A90191FFF774FFFFF7A4FF012003B039
:104170005DF804EB02B070470020F8E70FB407B514
:1041800004A951F8040B0191FFF762FF03B05DF839
:1041900004EB04B0704730B52B4885B0FFF76AFFD9
:1041A0002A4B1B7923B92A4805B0BDE8304099E76E
:1041B0003FF0CCFE08B92748F6E73FF0DDFE08B92E
:1041C0002548F1E7254B1B68DB6998470028F7D0A5
:1041D0003FF0DAFE0268037D81790446407C02905C
:1041E000207C0190608A009052081D48FFF7C6FFAE
:1041F000E51D0C3415F8010BFFF79EFFA542F9D120
:10420000184C1948FFF736FF6378022B06D007D900
:10421000032B10D11548FFF72DFF0CE01448FAE7E7
:1042200004F580541348FFF725FF94F8E437022B78
:1042300005D0032B05D005B0BDE830403AE70E4865
:10424000E9E70E48E7E700BFEA900608543C002083
:10425000F49006080391060811910608841E0020B8
:1042600020910608148D00204E9106085E910608E4
:1042700064910608719106087791060890910608E6
:104280000FB407B504A951F8040B0191FFF7E0FE44
:10429000FFF710FF03B05DF804EB04B070472DE9A1
:1042A000F041037903F0E002402A4AD004D85AB121
:1042B000202A23D0BDE8F081602A45D0802AF9D198
:1042C0008279417922480BE003F00703022B02D0E8
:1042D000042B08D06BB9B0F80720B0F805101D48C2
:1042E000BDE8F041CCE7D0F805101B48BDE8F0412F
:1042F000C6E7B0F90720B0F90510F0E74679174D89
:10430000174805EBC605FFF7B5FE95F8F4730024D2
:104310000123A74202D8BDE8F041CBE6D5F8F0630F
:1043200056F824204FEA84084AB113B90D48FFF724
:10433000A1FE56F808100C48FFF720FF00230134B7
:10434000E7E741790948D1E7BDE8F041084897E738
:10435000F4910608B8910608A29106084CE70508F2
:10436000CF910608E091060869A60608E3910608C1
:104370000B9206080249034801F521610EC97FE747
:104380000070FF1F2392060810B5752104462DF01A
:104390006FFC01460948FFF773FF1A2120462DF0F4
:1043A00067FC01460648FFF76BFF1B2120462DF0F6
:1043B0005FFCBDE810400146024861E737920608FD
:1043C0004A9206085D92060838B50B4DE87810F061
:1043D000FD0405D10948FFF753FF2046FFF7D4FF3E
:1043E000EB78013B012B06D80548FFF749FFBDE8F4
:1043F00038400120C8E738BD6C22002070920608C2
:104400007B9206082DE9F04FBD4BBE491A68BE4BA2
:10441000B2FBF3F299B08046BC48FFF7AFFEBC4B4D
:10442000DFF89CC30FCBDCF808700CAD85E80F00FB
:10443000B84B0793BC08B84B089314F00204C7F3B9
:10444000810718AB18BFDCF8046003EB870318BFC3
:10445000C6F3805653F8301C002C00F0BF8018AB18
:1044600003EB860353F8442CAC4CAD48AD4FAE4E35
:10447000DFF85093DFF8D8A2FFF780FEB4F8222EC1
:104480004FF47A73B2FBF3F103FB11220A20B4F963
:10449000243E92B2B2FBF0F2A448FFF7F1FEA44A28
:1044A000A449A548FFF76AFEFFF704FEA17DA34AD1
:1044B000A34BA44807EB8101D31AD1F8B815A28801
:1044C000FFF7DEFEA048FFF7D5FD94F8261E9F48B3
:1044D000FFF754FE9E48FFF7CDFD94F8271E9D4838
:1044E000FFF74CFEFFF7E6FD9B48FFF7C3FD0021F9
:1044F0000A46F37F0B4113F0010F01F1010508D0CB
:1045000012B15046FFF7B6FD29464846FFF736FE82
:104510000122072D2946ECD1904D95F86A1505F535
:10452000EC7305F13C02012918BF134693F8DC3007
:10453000032B02D08A48FFF721FE8A4B95F86A15B3
:10454000A3F5CE72012918BF134693F8DC30012B76
:1045500002D18548FFF712FE824B95F86A15A3F544
:10456000CE72012918BF13461B695B7B012B02D950
:104570007E48FFF703FEDFF85092FFF79BFDD4F86B
:10458000283E0393002609F1200A59F8041B39B389
:10459000012303FA06FB039B1BEA030F1CD01BF04D
:1045A0001F0F19D0724B5AF82620985D52F8202020
:1045B00036B17048CDE90412FFF75CFDDDE9041265
:1045C0006D48FFF7DBFDBBF1020F05D195F8311AFD
:1045D00011B16A48FFF7D2FD0136D6E7684A43E7D2
:1045E000FFF768FD94F8761CD4F8782C6548137AA8
:1045F000527A07EB8101D1F8F815FFF741FE6249C5
:104600006248FFF7BBFD62496248FFF7B7FDFFF75D
:1046100051FD614B614819684FF47A73B1FBF3F1B6
:10462000FFF7ACFD09A8FEF7B7FB38B109A910A840
:1046300047F0ACF85A4810A9FFF7A0FDFFF73AFD84
:10464000D4F8B42E002A00F0C38007EE902ADFEDE4
:10465000556AB8EEE77AC6EE877AFDEEE77A17EE8E
:10466000903ADFF86891B9F8740458B107EE900AEF
:10467000DFED4C6AF8EEE77A86EEA77AFDEEC77AB0
:1046800017EE900AD4F8346E5EB107EE906ADFED53
:10469000456AF8EEE77A86EEA77AFDEEC77A17EE5E
:1046A000906AB5F86C1A6429A8BF6421CDE90006A8
:1046B0003D483E4EFFF7E4FD99F8763499F87724AB
:1046C000B9F878143A4807EB83030125D3F80C3680
:1046D000FFF7D6FD374B3848198889B2FFF7D0FD70
:1046E00027494046FFF757FD3448FFF7C3FCD4F88D
:1046F0001048002C6ED1FFF7DDFC19B0BDE8F08F3B
:10470000081900208692060840420F008B92060886
:10471000F4EC0508A8920608AD920608F8470020B8
:10472000B29206084CE705086C220020BA920608EF
:10473000F0FF001000080000DB920608008000086F
:1047400000400008FF9206082E93060840930608D2
:10475000489306084A93060852930608840A0010F4
:104760006B9306085C0C0010739306087893060898
:1047700080050020E09106088093060886930608CD
:104780000E9B06088A9306089C930608BD930608AC
:10479000CB930608D1930608881E0020D7930608FD
:1047A000F19306080024744904940608E897060863
:1047B0004A940608B42600207194060880940608DE
:1047C000003802406293060810ED0508F0580020FA
:1047D000134646E794FAA4F3B3FA83F305FA03F217
:1047E00007EB83033046D3F8201624EA0204FFF7D0
:1047F000C5FC7EE72DE9F04FDFF8788198F80B30A3
:1048000099B0002B00F098805148524EDFF868B103
:10481000DFF86891DFF868A1FFF764FC00252F46F8
:104820000BA9E8B217F08EFA9DF83430002B53D064
:10483000139C54B107EE904A9FED470AF8EE677A51
:1048400080EE270A48F0AAFC04460B9A29465846EF
:10485000FFF794FC109A002A70D002FB04F04FF48A
:104860007A73B0FBF3F30993DDF848C0BCF1000F95
:1048700066D00CFB04F142F21073B1FBF3F198F82F
:104880000B30082D18BF7F18002B5BD017980790AE
:1048900015980690169805900A2311984FF47A7E81
:1048A000B0FBFEFE0998CDF810E0B1FBF3FE03FB70
:1048B0001E11CDE902E10999B1FBF3F103FB1100EF
:1048C000CDE90010BCFBF3F321465046FFF7D8FCBE
:1048D0000023C6E90D33B36201351D2D06F14006F4
:1048E0009ED198F80B3023B31C4C1D48D4F8842477
:1048F000D4F88014D2084FF47A73B1FBF3F3D4F8F0
:104900008814FFF7BDFC0A221648B7FBF2F102FB40
:104910001172FFF7B5FC144B1B78432B06D1D4F86A
:104920008C24D4F890141148FFF7AAFC0023C4F893
:10493000883419B0BDE8F08F0D4866E7099293E717
:1049400061469CE721464846FFF79AFCC0E700BF56
:1049500096940608245600208096184BF0580020A4
:104960003D9506085D9506084D1E002081950608B8
:10497000F4940608F8470020FE940608C7A7060826
:104980000D95060838B52A48FFF774FB294B93F8B4
:104990000134002B49D0284C2848FFF7A3FB94F89A
:1049A000D43A2BB194F8DA3A13B194F8D53A43B922
:1049B000B4F8E05A2248FFF75DFB2DBB2148FFF712
:1049C00091FBB4F8D61A2048FFF7D8FB94F8D43AF4
:1049D0002BB31E48FFF786FBB4F8DC1A1C48FFF720
:1049E000CDFB94F8DA3AE3B11848FFF77BFBB4F853
:1049F000D81A1848FFF7C2FB94F8D53A9BB1134870
:104A0000BDE83840FFF76EBB4FF47A72B5FBF2F1A8
:104A100002FB1152104892B2FFF732FCD1E70F4867
:104A2000D8E70E48E1E70D48EAE70D48E8E700BFA0
:104A3000AB950608F8470020840A0010C1950608C7
:104A4000C8950608E3950608F79506081796060820
:104A50002796060841960608ED9506082096060852
:104A600094D306080EB403B503AA52F8041B0192AE
:104A7000FDF7FCFD064BD3F8182D22B90549D3F8F4
:104A80008800FDF727F802B05DF804EB03B070472B
:104A9000F84700200C9B06082DE9F04715460A79D7
:104AA00002F0E004402C81460F4698462DD1DFF8F5
:104AB00078815C4EDFF89491002415E03B7903F097
:104AC0000703013B032B03D8DFE803F01315181B82
:104AD000295D3046FFF752FB7B79013BA34202DDA3
:104AE0004846FFF7C7FA01347B79A342E6DCBDE80C
:104AF000F0872957EDE735F81410EAE735F9141077
:104B0000E7E755F824104046E4E702F00702042ADC
:104B10003ED8DFE802F0030C141619002E78602C42
:104B200044D02BD8002C4CD0202C61D0DFE795F955
:104B30000060602C3AD021D8002CF5D12EE02E88D0
:104B4000EDE7B5F90060F4E7D5F800A0202C564653
:104B50004ED011D8002CCAD151463348FFF70EFB76
:104B6000D7F805108A4553D8B8F1000FBFD02F48A9
:104B7000BDE8F047FFF702BB602C17D0802CB6D100
:104B800029782B4B2B48002914BF29461946EFE7FB
:104B9000202C2CD007D8002CA9D12646B7F90540E7
:104BA000B7F9075011E0602CE8D100267B7946FA6E
:104BB00003F3DB07BDE8F0474CBF1F481F48FFF772
:104BC000DDBAB7F80540B7F8075016483146FFF789
:104BD000D5FAB4421CDCB5421ADBB8F1000F86D01E
:104BE0002A4621461648BDE8F047FFF7C7BA002617
:104BF0007A79144B03EBC20393F8F423B24207DD36
:104C0000D3F8F03353F82600BDE8F047FFF732BA87
:104C1000FFF750FA3A680C4933464846BDE8F0477A
:104C200020E700BFCC910608B591060861960608FA
:104C300018CC060869A606082092060894D3060830
:104C4000B28F06084CE705086796060848930608E1
:104C500013B50446084601920091FDF7A5F8DDE979
:104C600000130246204602B0BDE8104014E70EB41F
:104C700003B503AA52F8041B0192FDF7F7FC054B9C
:104C80000549D3F88800FCF725FF02B05DF804EB76
:104C900003B07047F84700200C9B06080149024604
:104CA000E5E700BF819606082DE9F041144BD3F8E3
:104CB000603988B00446F3B11A6804A9D56A184669
:104CC0006A46A847064688B1DFF8408004AC6D46C6
:104CD000002735F8022B34F8021B40460137FFF756
:104CE000CFFABE42F5DC08B0BDE8F08105492046A8
:104CF000FFF7BDFFF7E7044908B0BDE8F041B6E7AC
:104D0000F8470020B2960608CA9606089896060844
:104D100013B504460846019146F08AFD024670B17B
:104D20000F2804D10199094848F03FFF38B1074BDB
:104D3000074A0849204602B0BDE8104097E70349FA
:104D4000054802B0BDE81040FFF79ABA284F0608A0
:104D5000D1960608DC9606080697060813B50446A1
:104D60000846019146F064FD0199024668B10428A5
:104D700003D1094848F019FF38B1074B074A0849E1
:104D8000204602B0BDE8104071E70349054802B073
:104D9000BDE81040FFF774BA204F060814970608C4
:104DA000DC960608249706082DE9F04306469BB0DA
:104DB00008460C4646F03CFD002705461C223946B5
:104DC00002A8019748F0C5FE25B3402D07D0394908
:104DD00040232A4630461BB0BDE8F04347E70DF1BB
:104DE000040804F1400902222146684648F0F1FE19
:104DF0000023102209A968468DF80270FDF718FEFD
:104E0000099B0DF10202934222D10234A14508F818
:104E1000010BE8D100213D220AA8099148F099FE32
:104E2000002D3AD0244C257ED5B1202204F11C015E
:104E300001A848F064FE98B104F11C0109A8FDF72F
:104E4000F3FC1E4A1E4909AB3046FFF710FF04E091
:104E50001A781C493046FFF70AFF1BB0BDE8F08303
:104E600094F88430CBB9C5B901AD0FCD164C0FC441
:104E700095E80F0084E80F00144B012209A8A4F163
:104E8000100183F89424FDF7CFFC1148FFF730F9A7
:104E9000104809A9FFF7F4F9DFE70C4B93F89434B5
:104EA0001BB9054B1B7E002BF2D0074909A8FDF763
:104EB000BBFCEDE737970608F84700207597060812
:104EC000DC9606085997060814480020F058002080
:104ED0007F9706088E9706082DE9F74F8346084608
:104EE0000D4646F0A5FC374F0446D7F80495B8B9EF
:104EF0003548364D364FFFF7BDF8012655F8041BEF
:104F000049B106FA04F313EA090F02D03846FFF755
:104F100035F90134F2E703B0BDE8F04FFFF7CAB846
:104F200002462C492846FDF733FD78B92A48274C1C
:104F30002A4DFFF79FF854F8041B0029EBD00B789B
:104F4000002BF8D02846FFF719F9F4E72B782D2B22
:104F50001E4B03BF013504F1FF344FF0010A4FF03F
:104F6000000A002653F8048BB8F1000F06D11C4943
:104F70002A46584603B0BDE8F04F78E6224641463F
:104F800028460193FDF704FD019BC0B90123B340FE
:104F9000BAF1000F0DD029EA03031248C7F804350F
:104FA000FFF768F80D48414603B0BDE8F04FFFF742
:104FB00067B949EA03030C48C7F80435F0E701363E
:104FC000D0E700BFF84700209B970608D4ED0508FE
:104FD000A5970608F9940608A9970608E897060811
:104FE000B4970608C5970608CE9706082DE9F74F2F
:104FF000814608460E461746984646F019FC044678
:10500000E8B93F483F4DFFF7B9F820460FF068FD7B
:105010003B68184206D020460FF074FD0146284632
:10502000FFF7ACF80134182CEFD13B6813B93648C0
:10503000FFF720F803B0BDE8F04FFFF73BB802469A
:1050400032493046FDF7A4FC0546A8B93048FFF7C1
:1050500011F82C462F4D20460FF042FD10EA080FA4
:1050600006D020460FF04EFD01462846FFF786F891
:105070000134192CEFD1DDE733782D2B48F0807304
:1050800003BF013604F1FF34012500254FF0000A6B
:10509000019350460FF036FD2246834601463046C6
:1050A000FDF776FC00BB50460FF01AFD019B034252
:1050B0001AD08DB1BAF1180F1CBF3B6840EA030843
:1050C0001548C7F80080FEF7D5FF1248594603B0CF
:1050D000BDE8F04FFFF7D4B8BAF1180F1CBF3D6818
:1050E00085433D600D48EEE70AF1010ABAF1190F58
:1050F000CFD10B493246484603B0BDE8F04FB6E584
:10510000D6970608E7970608E0970608F994060878
:10511000A9970608E8970608C5970608CE970608D7
:10512000B4970608014A40F202235FE7F44D0020DD
:10513000014A6FF07F4359E7EC4D002070B50546FA
:1051400008461646FDF716FD0D4B93F89025904244
:10515000044605D201460B48FFF792F8204670BD81
:105160002EB1FF2803D10848FFF78AF8F6E7074970
:10517000013A2846FFF77BFD4FF0FF34EEE700BF12
:10518000840A0010EC970608FD9706081098060898
:105190002DE9F04F074691B08248834D0E46FFF748
:1051A0006FF88249C5F898D4002385F89C3406220C
:1051B000012391F890153046402485F89D440BF06A
:1051C0002DF80A200BF074F995F89C340C2BDAB208
:1051D00040F2E4809DF80C50FE2D30D0FF2D0BBF27
:1051E00015240F2401260026944240F0D780611E2A
:1051F000C9B268463AF0F8F804F140030DEB030435
:1052000014F8413C834240F0C48006F1FF385FFA55
:1052100088F8B8F1010F9DF80D3012D903F01F077F
:1052200061375C096248FEF725FF022E6AD0013C17
:10523000042C65D8DFE804F00B5E6064620002268F
:10524000D2E79DF80E709DF80F401D46EAE75948D9
:10525000DFF8BC91DFF8BCB1FEF744FF5648FEF71B
:1052600009FF6C464FF0000A14F8011B48460AF18A
:10527000010AFEF783FFBAF10C0F49D1FEF71AFFBE
:10528000022E4FD06422B5FBF2F102FB11524B48C3
:105290003B46D2B2C9B2FEF7F3FFB8F1010F71D8A5
:1052A000474A484B9DF810104748484D002914BF05
:1052B00011461946FEF7E4FF9DF81110444B45488E
:1052C000002914BF19462946FEF7DAFF022E59D1EC
:1052D0009DF812404048FEF7CDFE4CB3FF2C37D06E
:1052E0000A22B4FBF2F102FB11423C48D2B2FEF7B3
:1052F000C7FF20E03A48ABE73A48A9E73A48A7E7B2
:105300003A48A5E700238DF83F300DF11F009FE7D5
:10531000374B03FB0AF2B2F1553FA5D85846FEF7CA
:10532000A9FEA1E733483A462946FEF7A9FFB7E7A9
:105330002846FEF7D7FE9DF813402F48FEF79AFE49
:1053400044B1FF2C21D02D482146FEF799FF04E0FF
:105350002B48EEE71D48FEF7C5FE1C4E284FDFF830
:1053600070800DF11305002415F8013F7BB1FF2B70
:105370000CBF3A464246214622480134FEF780FFE0
:10538000042CF1D111B0BDE8F08F1D48E3E732469F
:10539000F1E71D493846FFF76AFCF3E71B48FEF7C3
:1053A000A1FEEFE756980608F0580020840A001086
:1053B0006798060872980608A0980608B29806082A
:1053C000369806083F980608E998060846980608A1
:1053D000B3A5060800990608079906081B99060850
:1053E000799806088198060889980608989806080A
:1053F000ABAAAAAACE98060823990608CC9106085B
:105400004A980608339906083E9906084E990608F8
:10541000A590060818CC06082DE9F84FDFF8A880FB
:10542000DFF88890DFF8A4A007460C46204646F037
:10543000FFF9064660B91D4B1D4893F8D8231D4B54
:1054400003EB8203D3F80017BDE8F84FFEF718BF4F
:10545000024641462046FDF79BFA60B1DFF860B096
:1054600000255BF8041BB1B9224638461249BDE855
:10547000F84FFFF7FCBB1148114C124DFEF7FAFD37
:1054800054F8041B19B12846FEF778FEF8E7BDE88A
:10549000F84FFEF70FBE32462046FDF779FA013588
:1054A0000028DED189F8D8535446BFE7F8470020DA
:1054B000579906084CE70508B4970608A997060807
:1054C00050EE0508E8970608F99406080E9B0608B2
:1054D00038B50D4604461A4905222846FDF758FA04
:1054E00068B9184B93F88C2022B9012183F88C10ED
:1054F00083F88D20BDE838401348FEF7F3BD13490B
:1055000003222846FDF744FAA0B90E4D95F88C30D9
:1055100063B195F88D304BB10D492046FFF7A7FBDD
:10552000002385F88C3085F88D3038BD0948FEF7AA
:10553000D9FDF5E720460849BDE83840FFF797BB9D
:10554000FCA40608F8470020619906085CA6060836
:1055500077990608AE990608C299060808B5034669
:1055600010462AB1DB0600D511B1FEF7C1FD0020BF
:1055700008BDF8B50D4E96F88430054693B9F8BDD0
:1055800025B12388C3F30B039D4204D0D4E9020163
:10559000A28848F07BFA1C34BC42F1D3002386F881
:1055A0008430ECE7024C034FF6E700BFF8470020D9
:1055B00064D6060898DE06080A4B93F8843010B5C6
:1055C00004460BB905F07CFFFCF76CFC44B10120EC
:1055D00005F012FF20B9BDE810400348FEF782BD78
:1055E00010BD00BFF8470020D19906082DE9F04F03
:1055F00085B0164601911A46824600213046FFF7D3
:10560000ADFF324C06F0100305464FF0000902933F
:10561000FEF714FD2379019A03F01803934203D097
:10562000002A48D1182B46D1284B4FF00D0B0BFB0D
:105630000933B3F80900FCF7A1FB80462046FCF7CC
:10564000E8F8D8E902210746024401442046FCF765
:1056500099F880F001012A460390C9B23046FFF75D
:105660007DFFDDE90223054602B123BB174A0BFB90
:1056700009FB52F80BB0B2060FD573B91448039367
:105680005946FEF77BFDD8F80820039B3A44214693
:105690005046FFF701FAFEF70DFD0E485946FEF79A
:1056A0006DFDD8F80C2000233A4421465046FFF700
:1056B000F3F9FEF7FFFC09F1010940F23E23994599
:1056C00004F10D04A4D105B0BDE8F08F8CFD0508F0
:1056D000F9990608FA9906080149FFF7C8BA00BF08
:1056E000049A06082DE9F043064687B008460C46A2
:1056F00046F09EF8082843D1671E03AD07342946BB
:105700003A46A84612F8010FFDF718F9A24201F82F
:10571000010BF7D10023DFF87C908DF8143017F8D7
:10572000010FFDF70BF9C1B205F8010B48460191D5
:1057300048F026FA20B10199284648F021FA28B10C
:105740003046FFF7C9FF07B0BDE8F083A742E6D1B6
:105750000F4940462BF048FF0D480E49082310F82A
:10576000012B11F8014B18326A44013B02F80C4C32
:10577000F5D109488DF8143003A9FEF781FDE2E761
:105780000028E9D0304607B0BDE8F043FFF786BAFD
:10579000D84B002008610608139A060807B5009345
:1057A00013460A460249FFF762FA03B05DF804FBAC
:1057B0001A9A060820B10078B0FA80F040097047C4
:1057C000012070472DE9F34106460846FFF7F2FF36
:1057D0000D46074670B1002401A9204640F082FF23
:1057E000013401463046FFF7EDFF122CF4D102B030
:1057F000BDE8F0810846FDF7BDF9C4B2112C71D89F
:10580000681CFCF779F93B4D8046E8B93A4B03EB4D
:10581000440393F8A0148A1E51425141364B03EBC6
:10582000440393F8A024AA5C002954D093F8A1342F
:10583000192040F2EE2100FB03133048214602B04C
:10584000BDE8F041FEF71CBD0178284648F098F904
:1058500070B1032C94BF00220122294902EB4202BD
:10586000431B0A4452FA83F393F87077032F04D151
:10587000304602B0BDE8F0412EE74046FCF73CF967
:1058800008B3022FF4D1FDF775F940F6CA0280B2D1
:105890009042194BA8BF104640F2EE22904203EB13
:1058A0004403B8BF1046A0F2EE201922B0FBF2F07C
:1058B00083F8A104BB1E594259410F4B03EB44032B
:1058C00083F8A074AAE7022FF4D1304602B0BDE8F5
:1058D000F041FFF7E3B90B48214602B0BDE8F041C3
:1058E000FEF7CEBC084911233A46304602B0BDE867
:1058F000F04153E7BC620608F0580020339A0608CE
:105900004CE70508439A0608509A06082DE9F04F1F
:10591000024691B00846FFF74DFF0B46044628B1FA
:10592000104611B0BDE8F04FFFF7B8B94FF0FF32A5
:10593000CDE90820A74ADFF8E482D2F88020DFF81A
:10594000E09292F83810DFF8DCA2CDE90C10CDE936
:105950000E02CDE90A00A04907AA184648F0CCF883
:1059600027460546049426464DB9089A0C9FBA422C
:1059700062D19A48FEF784FC11B0BDE8F08F062F83
:1059800012D8DFE807F0041E2328454C5100514689
:105990002846FDF721F878B14FF480600FF0C0FA87
:1059A00090F90430089301248B4907AA002048F09D
:1059B000A3F801370546D7E72846FDF7DBF808903E
:1059C000F2E72846FDF7D6F80990EDE72846FDF7FF
:1059D0001AF80A90E8E7284645F02AFF41460246B1
:1059E00005902846FCF7D4FF18B3059A4946284687
:1059F000FCF7CEFF06460028D6D02846FDF7BAF8B9
:105A000004280646D0D901467548FEF739FCB3E7AD
:105A10002846FDF7AFF800230C900F93C4E7284603
:105A2000FDF7A8F80D90BFE72846FCF7ECFF0E90B5
:105A3000BAE701230493B7E7DFF8EC8151B243469C
:105A400013F9010B884208D00135092DF8D1002146
:105A500064480131FEF714FC8EE763480121FEF72C
:105A60000FFC7AB2002318F9011B8A4200F00D8165
:105A70000133092BF7D13A460121E9E7A7F11402D6
:105A800053425341059308AD002303F10108EB682D
:105A9000A3BB95F900B058460FF00AFAD5F804A058
:105AA00020B1D0F80090B9F1000F5ED1BAF1000F2B
:105AB00019D14FF461436B604FF0010AAB680BB929
:105AC0000323AB600023D5F8049002932A7A194689
:105AD000CDE9009258461A4614F04CF9E86028B90E
:105AE0004248414691E74FF0000AE7E74A464146FF
:105AF000BAF1000F37D03E48FEF740FBB8F1020F75
:105B000005F110054FF00103BFD1059BDDF83C8086
:105B10000B9D53B13748FEF7E5FAD8F800301B6A01
:105B20001BB135492A4640469847049B002B4ED06E
:105B30003249334B142F18BF19463248FEF7A0FBE9
:105B4000142F09D1049B03B936B12B68DB691BB153
:105B50002D49324628469847002C67D100224146FD
:105B6000284640F073FD2948C6E7C5F80C90BAF105
:105B7000000F25D0264841465246FEF7FFFA51460F
:105B8000484603F059FAD5F808A0BAF1000F0FD033
:105B900099F8042092450BD01E4853464146FEF723
:105BA000EDFAD9F800305FFA8AF19B6948469847C8
:105BB000D9F82C30002BA1D00023C9F82C309DE758
:105BC000D9F8082014484146FEF7D8FADBE70C491B
:105BD000B3E700BFF8470020C19006088E9A060878
:105BE000769A0608D29B0608A79A0608B39A060872
:105BF000CF9A0608869B060839900108589A06082D
:105C00000E9B0608AF9B0608131B0108F39A0608B3
:105C10000F9B0608619B06083C9B0608709A0608C5
:105C2000E2970608659A060828EA050807F0ACFC22
:105C300005200AF03DFC1A4FDFF86C9000264FF06B
:105C4000030A99F89035B34288D917F801BBBBF124
:105C5000000F15D058460BF0F5F8044680B15846B1
:105C600007F0EAFB08B1A0F806A00121049006F0B5
:105C7000CBFDE379049813F0010F03D006F0D4F8BC
:105C80000136DEE706F0D6F8FAE706483A46022182
:105C9000FEF7F6FA099B002B3FF4F0AE0023F1E685
:105CA000F4260020A79A0608840A001010B50446BE
:105CB00008460B46FFF77EFD28B90949032218461E
:105CC000FCF766FE28B90748FEF712FA0120FEF736
:105CD000D9F920460449BDE81040FEF7C8BF00BF0F
:105CE000E49B0608E89B0608C29906082DE9F74FD1
:105CF00005460846FFF75EFD0B46044618B9334AD1
:105D000092F8C47427B9284603B0BDE8F04FE3E425
:105D10002F49DFF8C880DFF8C890DFF8C8A001AAD3
:105D2000184647F0E9FE264610B907F03BFC08E0AC
:105D300056B9012201462846FFF700FA421C0446E4
:105D40001BD103B0BDE8F08FFCF714FF2F2883466A
:105D500036D80FB107F018FCBBF1060F14D01D495F
:105D6000012391F890155FFA8BF2E0B20AF056FA2F
:105D700059464846FEF784FA0027154901AA002033
:105D8000013647F0B9FECFE7DAF808351B0113D525
:105D9000FF2C0FD0E1B22846FFF7FAF9E8E72846D2
:105DA000FFF7F6F901370B4B93F89025F9B28A42C9
:105DB000F5D8DDE70027F6E70748FEF793F9D7E7C0
:105DC0002F2241462846FEF752FFD6E7F058002022
:105DD000C1900608840A00100A9C06082A9C06083E
:105DE000199C0608F84700202DE9F04F064685B0BB
:105DF0000846FFF7DFFC0B46044628B1304605B0E5
:105E0000BDE8F04FFEF74ABF3149DFF8D490DFF824
:105E1000D4A0DFF8D4B003AA184647F06DFE274699
:105E20000546A04665B92B4B3A46D3F88000A1B28F
:105E300042F088F968BB28493046FEF718FF28E091
:105E4000B8F1000F06D0B8F1010F25D03046FEF7AB
:105E500025FF1EE0284645F0EBFC4946024601902E
:105E60002846FCF795FD50B3019A51462846FCF7A9
:105E70008FFD30B3019A59462846FCF789FD10B3CF
:105E8000019A16492846FCF783FDF0B13046FFF72A
:105E900023FC05B0BDE8F08FBB1E5A425A4129468B
:105EA0003046FFF74BF9421C0446F2D0084903AADA
:105EB000002047F021FE08F101080546B2E74746F9
:105EC000F4E70127F2E70227F0E70327EEE700BF38
:105ED000C1900608F8470020569C0608539C060807
:105EE0004A9C06084D9C0608509C06082DE9F7437D
:105EF00080460846FFF75EFC0B46054628B1404643
:105F0000FEF7CCFE03B0BDE8F0832E49DFF8B49075
:105F100001AA184647F0F0FD2F4604462E467CB9EC
:105F2000022DECD1A7F57A73B3F57A7F21D92649F2
:105F30004FF4FA634FF47A724046FFF72FFCE1E723
:105F40004DB1012D10D001AA4946002047F0D4FDE3
:105F500001350446E3E7012221464046FFF7EEF80B
:105F6000431C0646EFD1CDE72046FCF703FE07466B
:105F7000E9E7164DD5F8103AB8B25B689847FF2E9E
:105F8000BCEEC00A124B0BD195F89025F8EE407A82
:105F9000A24212DC10EE101A0E48FEF771F9B1E7BA
:105FA000F8EE407A03EB860310EE102A0A48C3EDA0
:105FB000007A3146FEF764F9A4E7E3EC017A013494
:105FC000E6E700BFC1900608649D0608840A001039
:105FD000B85D0020819C0608749C0608F8B5074649
:105FE0000846FFF7E7FBC8B11F4BDE6C01363046B1
:105FF0000EF088FD34460546F0B90134192CA8BFCF
:10600000002420460EF07EFD0546A8B9B442F4D126
:1060100038461649BDE8F840FEF729BE0846FCF7A9
:10602000A9FD04460EF06EFD054628B9214610482C
:10603000BDE8F840FEF724B90B4BDC6413F080FF99
:106040000C482A462146FEF71BF9182C09D80A48A5
:106050000C2101FB040090F87807BDE8F84013F02C
:10606000A5BF0020F9E700BF3C050020909C060872
:10607000A49C0608BA9C06084CE7050838B5124DE2
:1060800004460846FFF796FB60B1104B104893F9A1
:1060900000104B1C0ABF0F4BC9B2197ABDE838403B
:1060A000FEF7EEB80846FCF765FD032804D8C0B239
:1060B000FDF784FC2946E4E720460749BDE838405F
:1060C0000322FEF7D4BD00BF0E9B06083C0500204E
:1060D000D39C0608F8470020E39C060838B5124D0B
:1060E00004460846FFF766FB60B1104B104893F971
:1060F00001104B1C0ABF0F4BC9B2597ABDE838409A
:10610000FEF7BEB80846FCF735FD032804D8C0B238
:1061100016F074FE2946E4E720460749BDE83840FA
:106120000322FEF7A4BD00BF0E9B06083C0500201D
:10613000CF9C0608F8470020DE9C06082DE9F74FA3
:10614000424BDFF820A11A7A5B7A8AF800200546D4
:10615000012088468AF80130FFF72EFA00263C4CD1
:10616000B1460D233A4A7343414652F803B05846AC
:10617000FCF732FC002841D0B9F1000F01D0FDF747
:1061800099FF34485946FDF7F9FF00222146284679
:10619000FEF75EFDFDF78EFF237903F01803082B51
:1061A00046D0102B49D02046FEF779F8284A0D2317
:1061B00003FB0623B3F80900FBF7E0FD0746D8B15F
:1061C0002046FBF726FBD7E9022100900244014458
:1061D0002046FBF7D7FA78B9019059461E48FDF7DB
:1061E000CDFF019AB9681346009A28460A44214611
:1061F000FEF752FCFDF75EFF09F10109013640F29E
:106200003E239E4204F10D04ABD10020FFF7B1F90B
:10621000FF238AF800308AF80130B9F1000F11D15C
:106220000E494246284603B0BDE8F04FFEF71FBDB9
:106230000B492846FFF722FFB5E709492846FFF733
:106240004DFFB0E703B0BDE8F08F00BFF847002076
:106250008CFD0508FE990608FE9C0608B497060802
:106260000E9B06083C0500202DE9F74F80460846A6
:106270000F4645F0DDFA044620B1012826D13B78CF
:106280002A2B23D1A948AA4EDFF8C092FDF72AFF96
:106290000025B2464FF00D0B40F23E270BFB05F3F5
:1062A00048465AF80310FDF769FF221E18BF012265
:1062B000314640460135FEF7CBFCFDF7FBFEBD4203
:1062C00006F10D06EAD103B0BDE8F08F3D21384656
:1062D00047F056FC002800F0228103469A4613F846
:1062E000012D202AFAD0AAEB070A0130054610F842
:1062F000013B202BFAD0DFF838B24FF000090D2314
:106300005FFA8AFA03FB09F20BEB02045BF8021056
:106310000191084645F08CFA0199009002463846F2
:10632000FCF736FB0D230646002853D1009A524550
:1063300050D1277907F0E003402B00F0B9800ED848
:10634000002B55D0202B00F08B8040467949FEF77A
:106350008EFC204603B0BDE8F04FFDF7A0BF602BD8
:106360007FD0802BF1D1284645F062FAE379A779F6
:10637000DB0706460CD52046FBF716FD03780146E1
:1063800033B13246284647F010FC002840F0C18067
:10639000002E00F0BE80B742C0F0BB800D2303FB8F
:1063A00009B3204693F805A0FBF7FEFC3A4600210E
:1063B00047F0CFFBB2452CD85F493246284647F01C
:1063C000F4FB30B32046FBF7EFFC3246294647F09A
:1063D00000FC1EE009F1010940F23E22914591D1F5
:1063E00056493A46404603B0BDE8F04FFEF73FBC81
:1063F00007F00702042A1CD119460A222846FCF796
:1064000017FBD4F80530834201469ED32046FBF7A4
:10641000E3FC0D2303FB09F949485BF80910FDF77C
:10642000ADFE00222146404603B0BDE8F04FFEF726
:106430000FBC2846FCF79EFBB4F80550B4F80710D3
:1064400017F0050FAAB218BF2AB28BB218BF0BB251
:106450009042FFF67AAF98423FF777AF0146D5E713
:106460006679384A02EBC606002796F8F4230092B4
:10647000BA463B46009ABA4202D9BAF1000F03D09D
:10648000002B3FF462AFC4E7D6F8F01351F82700B1
:1064900060B129460193FCF757FA019B30B93946A0
:1064A00020464FF0010AFBF797FC53460137E1E71E
:1064B0006379009307F00707013F009BB342A8DD13
:1064C000AA4615F8013B202BFAD02046FBF76CFCBE
:1064D0000546032F03D8DFE807F0020D0D135046E1
:1064E000FCF748FBA8552C21504647F049FB0136E4
:1064F000451CE2E75046FCF73DFB25F81600F2E7A5
:1065000000230A2219465046FCF792FA45F8260065
:10651000E9E70D493A464046FEF7A9FB15E739463B
:10652000404603B0BDE8F04F08E600BF0E9D0608E8
:106530008CFD05085C9D060818CC0608B497060873
:10654000519D06084CE70508219D0608FE9906089E
:106550002DE9F04F914689B00C461A46002180463D
:10656000FEF7FCFFDFF8ECB006464D460027B9F118
:10657000000F6CD029460622204647F0C0FA0028BA
:10658000324614BF0121002140460CBF4FF0010AE2
:106590004FF0000AFEF7E2FF0646287815F05CF996
:1065A000079010B3687915F057F9079BEA785B7983
:1065B0000793AB7895F801E04FF461714FF0190C37
:1065C0001CFB03131CFB0212297900B14079CDF8A2
:1065D00004E0CDE90232079B0093CDE904103B466D
:1065E0005A4651464046FDF7B1FD207815F034F982
:1065F000079010B3607915F02FF9079BE2785B796B
:106600000793A37894F801E04FF461714FF0190CEF
:106610001CFB03131CFB0212217900B14079CDF859
:1066200004E0CDE90232079B0093CDE904103B461C
:106630005A4651464046FDF741FD0137142F04F1FB
:10664000060405F1060592D109B0BDE8F08FCA46EF
:10665000CBE700BF6A9D06082DE9F041064686B0EB
:106660000846FFF7A7F80F46054638B100235D49F5
:106670001A46012006B0BDE8F04169E70846FCF77C
:1066800079FA1328044600F3A38006264643781CB3
:106690008DF81750FBF730FA534D074670B1FCF7F1
:1066A00069FAC0B215F0EEF840B1AB19027983F87F
:1066B00060259DF8173001338DF817303846FBF709
:1066C0001BFA074668B1FCF755FA0D2809D80623CE
:1066D00003FB045383F861059DF8173001338DF8EF
:1066E0001730DFF80081B11C0DF117024144384624
:1066F000FCF744FAFBF700FA074668B1FCF73AFAF0
:10670000012809D8062303FB045383F864059DF888
:10671000173001338DF817303846FBF7EDF980B1AB
:10672000FCF728FAC0B215F0ADF850B1062303FB10
:106730000453027983F865259DF8173001338DF8ED
:1067400017309DF81720042A4FF006032FD103FBC2
:1067500004530022A3F8642521F044FC062303FB24
:1067600004554FF4617695F8600515F075F895F8C5
:10677000632595F862751923804695F8650513FB26
:10678000076713FB026615F067F8437998F8052050
:10679000039395F864350097CDE90163134895F8A4
:1067A00061352146FDF76CFD06B0BDE8F081052A94
:1067B00005D103FB0453002283F86525CCE7062AA4
:1067C000CAD008EB0602002348F806309380C3E7DE
:1067D000074913232A46304606B0BDE8F041FEF7CC
:1067E000DDBF00BF584D0020F84700206A9D060815
:1067F000839D06082DE9F04F174689B01A460C46CE
:1068000000218146FEF7AAFE3B4EDFF8F4B007F107
:106810006C0380463D46079394F90410374A0023E1
:1068200092F90800884263D00133092B02F10C026F
:10683000F6D1079B0C359D4204F10C04ECD109B054
:10684000BDE8F08F29460C22204647F058F9002871
:10685000424614BF0121002148460CBF4FF0010AF7
:106860004FF0000AFEF77AFEEA7995F9043006EB5C
:1068700082028046D2F8A42804922A7A06EB820289
:106880005146D2F8A4280392AA7906EB8202484620
:10689000D2F8A42802926A7906EB8202D2F8A428E0
:1068A00001922A6800925A46FDF750FCE27994F969
:1068B000043006EB82025146D2F8A4280492227AD0
:1068C00006EB82024846D2F8A4280392A27906EB8E
:1068D0008202D2F8A4280292627906EB8202D2F8F0
:1068E000A4280192226800925A46FDF7E7FBA0E730
:1068F000002FA7D1BA46D9E74CE70508904C0020F5
:10690000899D06082DE9F04707468AB00846FEF73C
:1069100051FF044638B1002354491A4601200AB0F9
:10692000BDE8F04766E70DF11C080790C8E90100D3
:1069300008464E1CFCF71EF94C4B40B21A4693F920
:106940000410814200F08B800134092C03F10C0308
:10695000F5D1002425463046FBF7CEF8064638B17F
:1069600000230A221946FCF763F801350790EDB2BF
:10697000DFF800A14FF000093046FBF7BDF80646EE
:1069800040B3FCF7F7F83A49002251F804CB6045D0
:10699000D3B203D00132102AF7D100230AEB8302CD
:1069A000D2F8A428904215D1B9F1020F1FD0B9F145
:1069B000030F21D05A1EB9F1010FD2B212D00B2A07
:1069C00003D88DF821300135EDB209F10109B9F193
:1069D000040FD1D1052D15D838460AB0BDE8F047CF
:1069E000FEF75CB9042AF0D88DF82230EBE7052BCE
:1069F000EBD88DF82430E6E79A1E0D2AE5D88DF8FD
:106A00002330E0E798E807001A4B84E807009DF878
:106A1000232003EB82020021D2F8A42804929DF8DF
:106A2000242003EB82020846D2F8A42803929DF8A2
:106A3000222003EB8202D2F8A42802929DF82120A2
:106A400003EB82030C4AD3F8A4380193079B00930D
:106A50009DF92030FDF732FB0AB0BDE8F0870C232A
:106A600003FB04248DF82000012574E7104C00205E
:106A7000F0EF05084CE70508899D06082DE9F04F61
:106A80008BB00C46089200211A460746FEF766FDB9
:106A9000DFF8B4B0089D099000264FF019094FF4B3
:106AA0006178089B002B4BD029460A22204647F0EC
:106AB00026F80028099A14BF0121002138460CBF8E
:106AC0004FF0010A4FF0000AFEF748FD2A890692AE
:106AD000EA8805922A790492EA780392AA780990C2
:106AE00019FB028202926A7819FB028201922A78CB
:106AF000009233465A4651463846FDF727FB228915
:106B00000692E288059222790492E2780392A278B2
:106B100019FB02820292627819FB0282019214F838
:106B20000A2B009233465A46514638460136FDF745
:106B3000C5FA1E2E05F10A05B3D10BB0BDE8F08FE2
:106B4000DDF820A0DBE700BFA69D06082DE9F04395
:106B500080468BB00846FEF72DFE0F46044638B13E
:106B6000002365491A4601200BB0BDE8F04385E7D4
:106B70000846FBF7FFFF1D28054600F3B3800A26F1
:106B80004643781C8DF82740FAF7B6FF044630B12B
:106B9000FBF7F0FF9DF8273001338DF827302046B2
:106BA000FAF7AAFF554C074668B1FBF7E3FF0D283B
:106BB00009D80A2303FB054383F8E8049DF827302E
:106BC00001338DF82730DFF83091711C0DF1270269
:106BD00049443846FBF7D2FFFAF78EFF074668B103
:106BE000FBF7C8FF222809D80A2303FB054383F8D3
:106BF000EB049DF8273001338DF827303846FAF73B
:106C00007BFF074668B1FBF7B5FF0D2809D80A23BB
:106C100003FB054383F8EC049DF8273001338DF81E
:106C200027309DF82730062B0CD009EB06020023F5
:106C300049F80630404653601381FEF72FF80BB039
:106C4000BDE8F0830A2606FB054600233846A6F871
:106C5000EE34A6F8F034FAF74FFF074640B1FBF7E1
:106C600089FF9DF82730A6F8EE0401338DF8273010
:106C70003846FAF741FF58B1FBF77CFF0A2303FBC4
:106C80000543A3F8F0049DF8273001338DF8273031
:106C90001B4B4FF0FF325A600A2202FB05424FF4B1
:106CA0006170B2F8F0340693B2F8EE34059392F8BE
:106CB000EC34049392F8EB34039392F8EA1419231A
:106CC00013FB0101029192F8E91413FB01030193F4
:106CD00092F8E834009300210A4A2B460846FDF753
:106CE000EDF9ACE708491D23224640460BB0BDE84C
:106CF000F043FEF753BD00BFD85D0020F0580020E0
:106D00003C050020A69D0608839D06082DE9F04F4E
:106D10002DED088BDFF82CA195B0804691461F46DB
:106D20000C4616464FF0000B94ED008AB5EE408AF3
:106D3000F1EE10FA7FD0D4ED019A94ED029AD4EDE1
:106D4000038AB9F1000F49D0D6ED00BA96ED01BA29
:106D5000D6ED02AA96ED03AAB4EE6B8AF1EE10FA14
:106D60006ED1F4EE4B9AF1EE10FA69D1B4EE6A9A54
:106D7000F1EE10FA64D1F4EE4A8AF1EE10FA0CBF8B
:106D8000012100213A460D46404681F00101FEF7FF
:106D9000E5FBB0EE6B0A074611A8FAF729FEB0EE44
:106DA0004B0A07900EA8FAF723FEB0EE6A0A069087
:106DB0000BA8FAF71DFEB0EE4A0A059008A8FAF7EC
:106DC00017FE0599069A079B039002910192009382
:106DD00052465B4629464046FDF7B8F9B0EE480AF0
:106DE00011A8FAF705FEB0EE690A05460EA8FAF7F3
:106DF000FFFDB0EE490A06900BA8FAF7F9FDB0EED8
:106E0000680A059008A8FAF7F3FD069B059A039017
:106E1000CDE9005302925B465246002140460BF1F9
:106E2000010BFDF74BF9BBF1080F04F1100406F15B
:106E300010067FF479AF15B0BDEC088BBDE8F08F7C
:106E400000219FE7C99D06082DE9F74FDFF898A1BB
:106E5000DFF898B107460D462846FEF7ABFC06461C
:106E600038B1002359491A46012003B0BDE8F04F5C
:106E70004CE7052251462846FBF78AFD60B9534B83
:106E800000221A601A611A621A631A641A651A6675
:106E90001A6703B0BDE8F08F4D4904222846FBF77E
:106EA00077FD04462846002C44D1FAF725FE80469B
:106EB0000028EED044F0BCFC464BC2B253F8049B11
:106EC000B9F1000F07D144492A46384603B0BDE85E
:106ED000F04FFDF7CCBE49464046CDE90023FBF715
:106EE00057FD0134DDE9002306460028E6D1374A84
:106EF0000346154600210133082B42F8101BFAD136
:106F00000BEBC404D4F8BCC0BCF1000F03D094F860
:106F1000B8E0764505DB3148314D4946FDF7B0F91B
:106F20009AE70CEB06130FCB05EB061484E80F0071
:106F30000136EEE7FBF71EFE072804463DD828463B
:106F4000FAF7DAFD064658B3FAF720FB1F4B03EBBE
:106F5000041383ED000A01253046FAF7CDFD0646FD
:106F600038B1FAF713FB194B03EB041383ED010A55
:106F700001353046FAF7C0FD064638B1FAF706FB90
:106F8000124B03EB041383ED020A01353046FAF786
:106F9000B3FD38B9384603B0BDE8F04FFDF77EBE0B
:106FA0000546D9E7FAF7F2FA0848032D00EB041476
:106FB00084ED030A3FF455AFECE70A490723324654
:106FC000384603B0BDE8F04FFEF7E8BB5450002050
:106FD000DD9D060850EE0508B4970608E29D0608F8
:106FE0000E9B0608839D0608709A06084CE7050864
:106FF0002DE9F74F92460C461A4600218146FEF7CE
:10700000ADFADFF870B0804656460025BAF1000FA1
:107010002ED031460422204646F071FD002842461B
:1070200014BF0121002148460CBF01270027FEF7AD
:1070300095FA738801933AF82530009380462B46E1
:107040005A4639464846FDF781F86388019334F87B
:10705000043B00935A462B46394648460135FDF716
:107060002DF8042D06F10406D0D103B0BDE8F08F51
:107070005746EAE7EC9D06082DE9F3410546084628
:10708000FEF798FB0C46074638B1002333491A46F1
:10709000012002B0BDE8F041AAE731492046FBF7E4
:1070A00053FC034670B92D4A4FF47A704FF4FA61DD
:1070B0000133042B1080518002F10402F8D102B098
:1070C000BDE8F0812046FBF755FD0328064641D870
:1070D0002046FAF711FD074670B1FBF74BFD4FF064
:1070E000010804463846FAF707FD48B9284602B0B9
:1070F000BDE8F041FDF7D2BD40F2EE248046F1E755
:10710000FBF738FDB8F1000FF0D0A4F2EE2240F208
:10711000DC539A4203D8A0F2EE229A420AD91149CE
:1071200040F6CA0340F2EE22284602B0BDE8F04124
:10713000FEF734BB0C4B0D4A03EB86030021A3F88A
:107140001446A3F81606CDE9004033460846FCF77E
:10715000B5FFB4E7064903233A46E5E7045F00209C
:10716000709A0608FD9D0608F0580020EC9D060860
:10717000509A06082DE9F04F89468FB01746002136
:107180001A460646FEF7EAF9DFF878A0054600241D
:107190000DF1240B59F824300293594602A83FF010
:1071A00003FA67B357F82430029A0393934218BF47
:1071B00001212A4608BF002130460CBF4FF00108CC
:1071C0004FF00008FEF7CAF904A9054603A83FF0EE
:1071D000EBF904A900912346524641463046FCF79C
:1071E000B5FF2346CDF800B0524641463046013443
:1071F000FCF764FF202CCDD10FB0BDE8F08FB8466E
:10720000EFE700BF0B9E0608F0B5074689B00846B9
:10721000FEF7D0FA0E46054638B1002319491A4642
:10722000012009B0BDE8F040A4E70846FBF7A2FC46
:107230001F2804461DD83046FAF75EFC014620465A
:1072400033F0E4FB78B10F4803AE314600EB840025
:107250003FF0AAF90C4A0096234629462846FCF737
:107260002DFF09B0F0BD384609B0BDE8F040FEF78B
:1072700033BA06491F232A46384609B0BDE8F04014
:10728000FEF78CBA145F00200B9E0608839D06084B
:107290002DE9F04F924685B00C461A4600218146F2
:1072A000FEF75CF9DFF874B0804655460026BAF167
:1072B000000F31D029460422204646F020FC002849
:1072C000424614BF0121002148460CBF0127002778
:1072D000FEF744F9EB780293AB7801932B88009387
:1072E000804633465A4639464846FCF72FFFE37836
:1072F0000293A378019334F8043B00935A46334633
:10730000394648460136FCF7D9FE102E05F1040532
:10731000CDD105B0BDE8F08F5746E8E7159E0608C9
:10732000F0B5074685B00846FEF744FA0E46054616
:1073300038B100231C491A46012005B0BDE8F040D1
:10734000A6E70846FBF716FC0F28044623DC304668
:10735000FAF7D2FB0146204632F0FEFFA8B1134BEC
:1073600004F1200203EB8203294693F827260292B8
:1073700093F826260192B3F8243600930C4A23464C
:107380002846FCF79BFE05B0F0BD384605B0BDE8C9
:10739000F040FEF7A1B907490F232A46384605B049
:1073A000BDE8F040FEF7FAB9945F0020F0580020E5
:1073B000159E0608839D06082DE9F04F87B01446F8
:1073C00003911A4600210546FEF7C8F8DFF830B1F0
:1073D00006464FF00008062303FB08F7C0374FF0BE
:1073E0000009039BDB5D0493002C00F08580E35DC6
:1073F000049A05939A4218BF0121324608BF002122
:1074000028460CBF4FF0010A4FF0000AFEF7A6F81D
:10741000059B0646CDE900935A4643465146284609
:10742000FCF794FE049B5A46CDE90093514643462F
:10743000284609F10109FCF741FEB9F1060F07F1F1
:107440000107CED108F10108B8F1060FC3D1DFF86A
:10745000B0B0E427039BA7F1E40913F807A0002CC0
:107460004CD0E35D04939A45324614BF01210021BC
:1074700028460CBF4FF001084FF00008FEF76EF8E9
:10748000049B0646CDE900935A460623414628460A
:10749000FCF75CFECDE9009A194A062341462846CE
:1074A0000137FCF70BFEEF2FD4D1039B93F8EF705D
:1074B000B4B194F8EF804745324614BF0121002152
:1074C00028460CBF01240024FEF748F8002300934F
:1074D0000B4ACDF80480072321462846FCF736FEE8
:1074E00000230093064A0197072321462846FCF70C
:1074F000E5FD07B0BDE8F08FA24693E7A046C9E7D7
:10750000279E0608F0B5054687B00846FEF752F9F3
:107510000B46044638B100231C491A46012007B027
:10752000BDE8F04048E71A49194F02AA184646F04C
:10753000E3FA03AEB8B1032C04D12846FDF7AEFB45
:1075400007B0F0BDFBF716FB02AA46F8040B39465C
:107550000020013446F0D0FAECE70E4832462146CE
:10756000FCF78EFEECE7032CE7D1DDE90346059B33
:1075700001931A463146E0B232F032FF019B0028F7
:10758000EBD12846FEF7A8F8DAE700BF145F002029
:10759000C1900608279E06082DE9F04F89B00C46D9
:1075A000079200211A460746FDF7D8FF0026079DDF
:1075B000DFF8A0B00690B2464FF019094FF4617899
:1075C000079B43B329460622204646F098FA002836
:1075D000069A14BF0121002138460CBF4FF0010A62
:1075E0004FF0000AFDF7BAFF6A79069019FB028294
:1075F00005922A7919FB02820492EA780392AA780A
:1076000002926A7801922A78009233465A4651468D
:107610003846FCF79BFD627919FB028205922279BC
:1076200019FB02820492E2780392A27802926278B5
:10763000019214F8062B009233465A4651463846BA
:107640000136FCF73BFD0A2E05F10605B8D109B05D
:10765000BDE8F08F3B9E06082DE9F04F80468BB0C9
:107660000846FEF7A7F88946074638B10023554972
:107670001A4601200BB0BDE8F04F8DE7524C08468A
:1076800094F86A3794F880B694F881A60793FBF7CC
:1076900071FA0928054600F38B800626464309F156
:1076A00001008DF82770FAF727FA074658B1FBF763
:1076B00061FA0D2807D8A31983F864099DF82730CB
:1076C00001338DF827303846FAF716FA074668B1C5
:1076D000FBF750FA834509D3062303FB054383F8E0
:1076E00065099DF8273001338DF827303846FAF7C1
:1076F00003FA074668B1FBF73DFA504509D806235F
:1077000003FB054383F866099DF8273001338DF8A4
:1077100027303846FAF7F0F9074670B1FBF72AFA36
:10772000079B834209D3062303FB054383F86709BC
:107730009DF8273001338DF82730DFF88890311D10
:107740000DF1270249443846FBF718FA9DF8273017
:10775000062B0BD009EB0602002349F80630404601
:107760009380FDF79BFA0BB0BDE8F08F03FB054457
:107770004FF4617194F86929192313FB02120592E1
:1077800094F8682913FB0213049394F86739039360
:1077900094F86639029394F86539019394F8643942
:1077A00000930021094A2B460846FCF787FCDAE7DC
:1077B000074909233A4640460BB0BDE8F04FFDF7B4
:1077C000EDBF00BF5C510020F84700203B9E06083B
:1077D000839D06082DE9F04F0F4689B0144600211D
:1077E0001A460646FDF7BAFE0546002C00F0DB807F
:1077F00022783B789A4218BF0121024608BF002137
:1078000030460CBF4FF001084FF00008FDF7A6FE10
:1078100023789B4A054641463046FCF797FC3B7867
:10782000974A41463046FCF749FC002C00F0BD80E9
:1078300062787B789A4218BF01212A4608BF00214E
:1078400030460CBF4FF001084FF00008FDF786FEF0
:1078500063788C4A054641463046FCF777FC7B78D6
:10786000884A41463046FCF729FC07F1CA030493D5
:10787000822304F1CA0B05934FF002094FF0000A6E
:107880003B78534500F39380002C00F0F38097F889
:10789000EA3094F8EA209A4218BF01212A4608BF2C
:1078A000002130460CBF4FF001084FF00008FDF7F3
:1078B00055FE94F8EA30744A054641463046FCF7D6
:1078C00045FC97F8EA30704A41463046FCF7F6FB33
:1078D00007F1EC09002C00F0CF8004F1EC034A46DC
:1078E00004F1FC014FF001089A4633F802CB32F85C
:1078F000020B844518BF4FF000088B42F5D188F089
:1079000001012A46C9B23046FDF728FE0821054686
:107910005046FAF769FF5D4A034641463046FCF798
:1079200015FC97F8EA104846FAF75EFF574A0346F7
:1079300041463046FCF7C2FB002C00F09F804FF020
:10794000FC094FF0010807EB090104EB0900FAF705
:10795000FBFF09F10409002818BF4FF00008B9F532
:107960008E7FF0D188F001012A46C9B23046FDF77A
:10797000F5FD082104F1FC00FAF7F0F8444A03464B
:1079800041463046FCF7E2FB97F8EA1007F1FC00AD
:10799000FAF7E4F83E4A03464146304609B0BDE8EE
:1079A000F04FFCF78BBBA04639E7A04657E7059B95
:1079B0003B440693002C5BD0059B06982344194654
:1079C0000793FAF7C1FF049B1A789BF800309A429C
:1079D00006BFB0FA80F84FEA58184FF000084B463F
:1079E00009F11002F85AE15A0233884218BF4FF0E9
:1079F00000089342F6D188F001012A46C9B2304608
:107A0000FDF7ACFD627804EB090105469BF8180010
:107A1000FAF7BCFE02909BF800300193079B00939D
:107A20001C4A0AF1010341463046FCF78FFB049BD8
:107A30007A78187E079307EB0901FAF7A7FE079BF0
:107A4000049A02901B7801930132069B04920AF17A
:107A5000010A00930F4A534641463046FCF72EFB7D
:107A6000059B09330BF1010B09F11009059307E799
:107A7000A046DCE7A04624E7A04652E7A04683E7FD
:107A8000549E0608669E0608949E0608AC9E06084C
:107A9000C39E06087B9E06082DE9F04F8FB0044672
:107AA00002AA0846AF4946F027F8064640B9034601
:107AB0000246AD494120FFF78DFE0FB0BDE8F08FC3
:107AC000AA49FAF741FF074620BBA64902AA46F099
:107AD00013F8FBF74FF80828054606D9A4490823F0
:107AE0003A462046FDF75AFEE7E7A24C94F8803666
:107AF000834202DC84F88056DFE7064604F5D0674F
:107B00003146384631F03CFD94F880360136B342B8
:107B1000F6DCEFE798493046FAF716FF0546E0B97C
:107B2000904902AA45F0E8FFFBF724F8082806462A
:107B300003D9924908232A46D3E78E4C94F881361C
:107B4000834202DC84F88166B7E728463146013576
:107B50003EF002FD082DF8D1F4E789493046FAF7E6
:107B6000F3FE074600BB7F4902AA45F0C5FF002887
:107B7000A3D0FAF7FFFF0828054603D98149082357
:107B80003A46AEE77B4C94F86A37834209DD0146FA
:107B900004F5D06031F03EFD294604F5D06031F0A7
:107BA00047FD84F86A5788E777493046FAF7CCFEF4
:107BB000054618BB6F4BDFF8AC9193F86A7706AEB9
:107BC00001461022304645F0C4FFB046BD4202AA2D
:107BD00080F20E814946002045F08EFF10B96B49B6
:107BE0003A460EE1FAF7C6FF013528F8020BEDE739
:107BF00096E80F00664C84E80F005EE76549304662
:107C0000FAF7A2FE054600283BD15A4B0DF11808A1
:107C100093F86A97464607464F45524902AA4FF0E5
:107C2000000080F2F28045F067FF014610B95A4922
:107C30004A46E6E00322304645F0CBFFB2464FF01D
:107C4000000B304643F0F4FD584502D801370436A6
:107C5000E2E79AF80000FAF771FE0BF1010B0AF85F
:107C6000010BEEE74D494A46CBE041462046032250
:107C700031F06EFC0135043408F10408AF42F4D150
:107C80001BE747493046FAF75FFE0546002840F0FB
:107C9000AC80384F334997F8808602AA45F02CFF14
:107CA00000283FF40AAFFAF765FF461E01D4B0453D
:107CB00003DC3C494346012213E72A4902AA00207B
:107CC00045F01AFF014600283FF4F7AE4FF00008D8
:107CD000082203A8CDE903888DF8148045F079FFC8
:107CE0000DF10C0903A843F0A3FD40451CD81D4924
:107CF00002AA002045F000FF00283FF4DEAE90F815
:107D000000A097F88196DFF8ACB04FF000084D4521
:107D1000144902AA4FF000007EDA45F0EDFE02465B
:107D200058B921494A466CE099F80000FAF706FE76
:107D300008F1010809F8010BD4E7002D40D11378B0
:107D4000303B092B3CD919490192FAF7FDFD019A04
:107D500090B310465946FAF7F7FD019A002838D03B
:107D600013494EE0C1900608784E0020DA9E0608BE
:107D7000E09E0608F8470020EB9E0608F49E0608E1
:107D8000029F06080E9F0608209F06080FA00608FF
:107D9000644F00204A9F06082FA00608569F060839
:107DA000749F0608799F06084FA006088F90060862
:107DB0008C9F0608859F06084FF001084FF0FF359D
:107DC00010460192FAF7D6FE0028019A03DA2149FB
:107DD00017E0A846F2E70EAB03EB4503013523F8A5
:107DE000200C94E71C494A460BE01C49324608E047
:107DF0001B49002045F080FE00283FF4F9AE1949E8
:107E00003A462046FCF733FF57E645F075FE00285A
:107E10007FF428AF144C31E745F06EFE0028E1D125
:107E2000124C06EBC6008230082203A9204431F030
:107E30008FFB5046FAF782FD37446A0087F84A07FD
:107E400004EB061006A9023045F020FE87F8628791
:107E500033E600BFC19F0608D69F0608F99F0608B3
:107E6000C19006082C9F0608744F0020784E002011
:107E700070B50A4C0A4E002594F8853013B120469F
:107E8000FBF7A0FF2046FCF779F801353046FCF7F8
:107E9000A7F8042D04F19604EED170BD68490020C6
:107EA0006C22002038B50C46054616492046FAF7E4
:107EB0004BFD30B9FFF7DCFF1348BDE83840FCF755
:107EC00011B912492046FAF73FFDA8B9104A82F8C5
:107ED000F50182F8FD0182F88B0282F8930282F8A4
:107EE000210382F8290382F8B70382F8BF03094A05
:107EF00082F821000848E0E72846BDE83840FDF751
:107F0000EBBB00BF74A006087AA0060895A006087F
:107F1000F84700206C2200209DA006082DE9F04FB4
:107F200089B00F4691460021139A98460646FDF700
:107F300015FB87EA09096FEA0903DFF884900693C5
:107F40000446002528460CF0CBFD129B184230D089
:107F5000069BDFF870B0034014BF4FF0010A4FF0EA
:107F6000000A049310EA070314BF4A465A462846FB
:107F7000059307920CF0C6FD079A039000904346C4
:107F800051463046FCF7E2F8049BB3FA83F12246EF
:107F900049093046FDF7E2FA059A039B009304462F
:107FA0004346002A14BF5A464A4651463046FCF71B
:107FB00085F80135182DC5D109B0BDE8F08F00BF97
:107FC000D79D0608B9A0060837B5044608460191B2
:107FD00043F02EFC0199054602462046FAF7D8FCEC
:107FE00070B9625D1046FAF799FC00B932B90135F3
:107FF0002C44204601340378202BFAD003B030BD46
:108000000020FBE7F0B5032985B005460C4616466F
:1080100014D80B4F3970FCF74DF80A492846FEF783
:108020002DF80949224601A8FAF754FB01AB324664
:1080300008212846FDF7DAFAFF233B7005B0F0BDB2
:108040003C0500200E9B0608D39C0608F0B50329CA
:1080500085B005460C46164614D80B4F7970FCF7D0
:1080600029F80A492846FEF739F8094922466846A0
:10807000FAF730FB6B46324610212846FDF7B6FA78
:10808000FF237B7005B0F0BD3C0500200E9B060869
:10809000CF9C0608F8B5114B93F88500D0B993F83A
:1080A0008C2012B193F88D20A2B90D4E96F89474DD
:1080B0008FB1187E70B90B4D0FCD06F214740FC43A
:1080C00095E80F0084E80F00012386F84F3709F088
:1080D0005FFC3846F8BD0120FCE700BFF8470020F0
:1080E000F05800201448002038B50546FFF7D2FFAD
:1080F000044660B907492846FCF7B9FD06492846F9
:10810000FCF7B5FD054B83F88C4083F88D40204685
:1081100038BD00BF77990608C0A00608F8470020C0
:1081200008B5FFF7E1FF50B1054B02229A75FBF746
:10813000F3FD0448FBF7DCFF0020FBF7A3FF08BDBD
:10814000F8470020DEA0060810B5094C94F8503717
:108150005BB9084B084918680C2245F026FD01233D
:1081600008B984F8513784F8503794F8510710BD96
:10817000F058002000280008E5A006082DE9F74F78
:10818000054601AA08464A49DFF850B145F0B4FC5B
:108190004FF00009012682464F464C46B046BAF1E0
:1081A000000F28D1B9F1000F2ED1424F002C7BD007
:1081B00041482146FCF764F897F884300BB903F086
:1081C0007FF9F9F76FFE002087F88D000EB103F0FC
:1081D00013F9FFF74DFE14B12046FDF7CAF9B8F1C7
:1081E000000F14D02846FFF77FFF80B1FBF794FD06
:1081F0000020FBF747FFB9F1000F0BD05046FAF70C
:10820000B9FC84B2002C3ED12846FDF765FA03B0D4
:10821000BDE8F08F29495046FAF7DEFB00283CD133
:1082200027495046FAF7D8FB002839D1594650461D
:10823000FAF7D2FB002835D122495046FAF7CCFB99
:108240000028E1D0002FDFD1FFF77EFFB0B11E4B39
:108250001E4D1C681E4E013C14F8011F4B1EDBB264
:10826000FD2BD4D82B689C42D1D20A2903D03046AA
:10827000FBF784FFF0E7FBF71DFFEDE71549284604
:10828000FCF7F0FBC3E74FF00009094901AA002001
:1082900045F032FC0137824681E74FF00109F4E7EF
:1082A000C846F2E74E46F0E70B48FBF721FF88E7A8
:1082B000C1900608F84700201EA10608F2A0060893
:1082C00033A5060800A106080028000804280008B5
:1082D0007297060805A1060841A10608FBA006083A
:1082E00030B587B0144B0493144B0393144B029393
:1082F000144B0193144B154A00930546144B154833
:108300000C461549FBF73AFFFBF7D4FEFFF71CFFBD
:1083100058B11248FBF7ECFE64B1114A11491248FA
:1083200007B0BDE83040FBF7ABBF10492846FCF76B
:1083300099FBF1E707B030BD8CA1060891A10608B2
:108340009BA10608A4A10608CB93060857A106081E
:108350000748002061A10608E7A00608B0A10608AA
:10836000284F0608204F0608CCA10608BCA1060825
:108370000121B5E72DE9F04F0A4687B000210646F6
:10838000FDF7ECF83B4C05903B4A2378608802EB04
:108390008303D3F8D4A9F9F7F1FC83680493374B2E
:1083A000C16893F88420002A4BD0DDF81080049136
:1083B000002721796279049B07FB012213F80290C0
:1083C000B8F1000F3FD018F80250059A4D4514BF80
:1083D0000121002130460CBF4FF0010B4FF0000B84
:1083E000FDF7BCF8013705907DB305F00F022D09AC
:1083F00040350292CDE90075214A53465946304630
:10840000FBF7A4FEB9F1000F2AD009F00F024FEAE2
:108410001919029209F14002CDE900725346184A37
:1084200059463046FBF74AFEA279012A38BF01229D
:10843000BA42BEDC134B0834A342A5D107B0BDE855
:10844000F08F9046B4E74546BFE7B8F1000FD9D0AA
:108450000D4A0097534659463046FBF777FED1E761
:108460007306E1D4084A0097534659463046FBF755
:1084700025FED9E730F005084CE70508F84700204D
:10848000F9A1060820F105080FA2060838B50C4B23
:1084900003EBC0050C4695F8E4280A4803EB820379
:1084A000D3F8D419FBF76AFE95F8EA3833B1611CAA
:1084B0000548BDE83840C9B2FBF760BE38BD00BF13
:1084C0004CE7050869A60608CB91060873B50E4669
:1084D00011490546FAF738FA18B93070012002B090
:1084E00070BD2C78602C8CBF613C413C072C10D8AF
:1084F000013501230A2201A92846FAF799FA019BBE
:108500009D4206D00F2804D8013440EA0414347088
:10851000E4E70020E3E700BFE78F06082DE9F04F0E
:108520002DED028B0A468BB000218246FDF716F82E
:108530006F4D814605F1800B00266E4B93F8844009
:10854000AB7AB34200F395801035AB45F4D140F2DD
:108550001620F9F713FCD0E902530CB12C461D4646
:108560000DF1100B15220021584645F0F2FA0027B4
:108570002E78002E44D069780391304608F03AFCFA
:1085800095F9023002935A1C534208EE100A5341E7
:10859000002C00F0A9800399002214F802C0B44511
:1085A00004EB020040F09C8090F90280029A424560
:1085B00040F0948042788A4208BF012301220BF8E0
:1085C000072003F001034A4683F00101504603935C
:1085D000FCF7C4FF039B81464CB1474A18EE101AC2
:1085E000CDE900A230464246F9F73AFB039B434AE5
:1085F00018EE101ACDE900A23046029AF9F730FBC6
:108600000137152F05F10305B2D16CB33A4FDFF8EE
:10861000EC8004F13F061BF8013B02930BBB207872
:10862000F8B194F9022001321BD0617808F0E2FB26
:108630004A46054601215046FCF790FF94F9022076
:10864000029B294681462078CDE900A7F9F708FB6F
:108650002078029BCDE900A84FF0FF322946F9F7B8
:10866000FFFA0334B442D6D10BB0BDEC028BBDE8A7
:10867000F08FE888F9F782FBD0E902230CB11446A9
:108680001A46297A6B7A06FB013312F9038014B378
:10869000E756B8450CBF012300234A4614BF012109
:1086A000002150460293FCF759FF029B814644B1DA
:1086B000114A3146CDE900A228463A46F9F784FA34
:1086C000029B0E4A3146CDE900A228464246F9F700
:1086D0007BFA013631E74FF0FF37DAE700236DE729
:1086E00003323F2A7FF459AF4FF0FF386BE700BFEA
:1086F0008C050020F84700204D410108BD400108CD
:108700002DE9F04F80468BB008460D4643F090F8B7
:10871000024678B3A8492846FAF73AF9044648BB16
:10872000FBF7C8FCA548A64DA64FA74EDFF8E4828C
:10873000FBF7D8FC14203DF023FFE11004F0070202
:1087400001313846FBF71AFD2B7F6A7F06EB830366
:10875000D3F8D41952B19D48FBF792FD0134102C87
:1087600005F12405E9D10BB0BDE8F08F4046FBF7D9
:1087700087FDF3E72846964905AA45F0BDF9054669
:1087800020B901464120FFF7C9FEECE79149FAF70D
:10879000DBF820B990494046FCF769FAE3E78F4ED1
:1087A0000827002431682846FAF7CEF8002808BFC9
:1087B0003446013F06F11006F4D154B988492846E1
:1087C000FAF7C2F828B187492A464046FCF74FFA23
:1087D000C9E700207E498DF8130005AA45F08CF901
:1087E0000646002C40D080B1FAF7C4F9451E09D4E2
:1087F000A37A9D4206DAE2684AB1012303FA00F047
:10880000104204D178493246DFE7784EFAE7E08833
:10881000F9F7B4FA764A92F884301BB192F88530B1
:1088200083F00103D0E90212002B08BF0A46217A27
:10883000637A05FB0133002712F903A0039702EBCB
:10884000030B634905AA002045F056F98146A0BBF9
:108850006849012344B39BF900202046CDE900314B
:108860002946F9F7B1F97EE768B10DF11301FFF779
:108870002DFE28B19DF81350284604F0DDFD20B9E7
:108880005D493246A1E7594EFAE7284603F02CFE2F
:108890008246284608F09AFA0390284608F0D2FA51
:1088A000A34607462546CCE7CDE900319DF81300E5
:1088B00052463946F9F7D4F955E74649FAF744F8EC
:1088C000064658BBACB14D4FEDB2207972B2294685
:1088D00003F0F8FA00283FF446AF028803780093CB
:1088E0003146C2F303233846120BFBF7C9FC0136AD
:1088F000EBE7424C7979386872B203F00BFE00283E
:108900003FF431AF0288037800933146C2F303236A
:108910002046120BFBF7B4FC0136EBE7384948461A
:10892000FAF712F810B34846FAF724F9064642B2AD
:108930006CB12079E9B203F0C5FAC8B9CDF800905E
:10894000226830496B1C4046FCF791F90BE77979B6
:10895000386803F0DFFD58B99DF813302A49CDF887
:1089600000901A09403203F00F03ECE74FF0FF3696
:1089700006AF39463046F9F76BFF08A95046F9F7BC
:1089800067FF564548D076B24CB18BF8006000972F
:1089900021681E4808AB6A1CFBF772FCE3E69DF8F1
:1089A0001320039B1A489E701109009708AB02F030
:1089B0000F024031F0E700BF00A1060823A206081D
:1089C000E001002039A206084CE70508ACA3060820
:1089D000C1900608F99406084AA206088C050020F2
:1089E0005EA2060862A2060871A206080E9B06088F
:1089F000F8470020BD40010881A2060893A206089E
:108A0000E2970608B4A20608D7A20608FFA2060845
:108A100022A30608E897060834B12168074808AB86
:108A20006A1CFBF72DFC9EE69DF8132004481109F3
:108A300008AB02F00F024031F3E700BF4AA306087B
:108A400065A306082DE9F04F8BB0074640F21620CB
:108A50000391F9F793F9039A044600213846FCF78D
:108A60007DFD414AD4E9025392F8844006460CB198
:108A70002C461D461522002104A845F06AF805F190
:108A80003F03039395F80090B9F1000F31D095F8AA
:108A900001A0002C65D0224600231178494558D109
:108AA00028336B4492F80180012203F8182CD0453A
:108AB000324614BF0121002138460CBF4FF0010B94
:108AC0004FF0000BFCF74AFD064654B1B8F1000F19
:108AD00007D0264B00935A463B4641464846F9F795
:108AE00003F9234B00935A463B4651464846F9F753
:108AF000FBF8039B03359D42C4D13CB3DFF86C9077
:108B0000DFF86CA0651C0DF11008403418F8013B2B
:108B1000CBB915F8013CB3B116B13046FBF7E8FA12
:108B2000297815F8010CCDF800903B460022F9F7A2
:108B3000DBF8002215F8010CCDF800A03B461146E9
:108B4000F9F7D2F800260335A542DFD10BB0BDE816
:108B5000F08F0133152B02F103029ED14FF0000874
:108B6000A5E7A046A3E700BFF84700204D41010854
:108B7000BD4001082DE9F04F80468DB008460D46F6
:108B800042F056FE024628B9014601200DB0BDE86C
:108B9000F04F57E70390B1492846F9F7F9FE039AD9
:108BA00030B9AF4940460DB0BDE8F04FFCF75FB8B3
:108BB000AC492846F9F7ECFE044600285BD1FBF7E8
:108BC00079FAA948A94FDFF8E4B2DFF8E482FBF7AD
:108BD00089FA17203DF0D4FC17F9015B002D3CD039
:108BE00029465846FBF7CAFADFF89C92DFF88CA2B8
:108BF00000231A46910089B228460593049208F092
:108C000057F9039008F0F4F9049A0178059B561C73
:108C1000C9B11BB90490FBF74DFA0498039B417846
:108C2000DA79037802F0020208EB8303C1B1009104
:108C3000D3F8D4398E48002A14BF4A4652463146EA
:108C4000FBF71EFB0123042E3246D3D113B989480A
:108C5000FBF748FA01340E2CBED10DB0BDE8F08F01
:108C6000D3F8D4398448002A14BF4A4652463146C4
:108C7000FBF706FBE6E7002480498DF81B4007AAB6
:108C8000284644F039FF18B94046FCF725FDE4E7D3
:108C90000DF11B01FFF71AFC05460028F4D09DF8E2
:108CA0001B60304604F0C8FB20B975494046FBF70D
:108CB000DEFFD2E7DFF8FC9123464FF0FF3403EBF1
:108CC000430212F8092096420BD0611C02D1002AFF
:108CD00008BF1C460133152BF1D1631C15D169491E
:108CE000E4E71C46654907AA002044F005FF064654
:108CF000002800F09E805949F9F726FE28BB624EF5
:108D0000624FDFF8B481044615E00025EAE7297ACE
:108D10002868039108F05AF90246E8796B790399BB
:108D200010F0020F14BF304638469B080090013304
:108D30004046FBF7A5FA01349DF81B00214608F0D8
:108D400059F805460028E2D187E75149022230460A
:108D5000F9F71EFE0746002849D1B01CF9F70AFFB3
:108D60009DF81BB00346BA4601373946584603936F
:108D700008F040F8039B38B94FEA1B1245490096AA
:108D80000BF00F0340323FE0027A9A42EBD1002D04
:108D900040D14FF0FF36BAF1FF3F9DF81B5008BF9E
:108DA000002504EB440409EB04030AF101025A70A4
:108DB00009F80450FF220AAC9A709DF81B00224665
:108DC0005146F9F755FD08AA31469DF81B00F9F701
:108DD0004FFD9DF81B20B2454FEA121120D12E48BD
:108DE00008AB02F00F024031FBF74AFA35E72B4996
:108DF0003046F9F7A9FD50B39DF81B30284900967D
:108E00001A09403203F00F034046FBF730FF24E716
:108E10004FF0FF3A04EB44034B445E78013EBAE75F
:108E20002048009408AB02F00F024031FBF728FA0B
:108E300013E704EB44041C4B0093A144024699F849
:108E400001109DF81B000123F8F74EFF05E7002DE8
:108E5000DED14FF0FF36B246A3E700BFF994060813
:108E60004AA2060800A1060881A30608104F0608BA
:108E7000A1A30608C2A30608B3A30608C19006086A
:108E8000C8A30608DFA30608219206080E9B060861
:108E900008A4060875A4060831A40608E297060887
:108EA0000BA406084FA40608BD4001089AA30608B3
:108EB0004CE70508A82E0020F3A3060800000000D8
:108EC000224BB0F5FA6F1A680346A8BF4FF4FA6355
:108ED000B3F57A7FB8BF4FF47A73D20416D540F257
:108EE000DC52904215D007EE903A40F2DB529042AD
:108EF000F8EE677A1FD8DFED166A9FED167A9FEDC0
:108F0000160A77EEE67AA7EE870A7047B0F57A7F01
:108F100002D89FED120A704707EE903ADFED106A13
:108F20009FED107A9FED100AF8EE677A77EEE67AF9
:108F3000A7EE870A7047DFED0D6A9FED0D7A9FED72
:108F40000D0A77EEE67AA7EE870A7047004D0020FB
:108F500000007A44D62000C000E0824400000000F7
:108F600000407A44661000400000404200A0BB442C
:108F7000D62000400000834410B584464FEA810E9D
:108F8000102312F4004F14BF0E2407245200013B9B
:108F9000CCF8004092B2F444F3D100EB81128C0182
:108FA000035142F82130122010BD00BF10B5844695
:108FB0004FEA810E0424130B03EB43031833120111
:108FC000013CCCF8003092B2F444F4D100EB011330
:108FD0000A01845043F82140062010BD704700BFAD
:108FE000704700BF034B00EB400003EBC000407C28
:108FF000704700BFA80900100023037043708370FE
:10900000C3707047704700BF00207047704700BFB3
:109010000020704701207047704700BF704700BFB5
:10902000704700BF704700BF9FED010A704700BF47
:10903000000000000020704703681B69184700BF4C
:1090400003682DE9F0415F6A1FB13B46BDE8F0417E
:109050001847002A164611DD04460D460E4400E06E
:1090600023689B68204698470028F9D0236815F8A4
:10907000011B1B6820469847AE42F1D1BDE8F08144
:1090800030B50A4B002193F900205D78092AC8BF4A
:10909000143A8418013125739D7885540829DA78AB
:1090A000227603F10403EED130BD00BFB41A0608E6
:1090B000C36B33B15B68426D9BB29A4205D3D01A41
:1090C0007047D0E907239A42F9D2C0681044C01A09
:1090D000704700BFD0E909120369914238BFC9182F
:1090E0008A1A016C39B14968013B12FA81F2934244
:1090F00004D9981A7047013B981A704700207047AE
:10910000036C13B190F864007047D0E90903181A92
:10911000B0FA80F040097047C26B10B4034662B1E8
:10912000426DC1685C69881A013A205C5DF8044BA5
:1091300008BF0A46C0B25A657047006A5C69411CA4
:10914000205CDC68A14238BF0A46C0B25DF8044B1F
:109150001A627047836E70B504460D460BB198478E
:10916000B8B1636AA269D554636A2169226C01337C
:109170008B4228BF0023636232B3EFF31183502286
:1091800082F31288226C1168C90703D5DBB283F31E
:10919000118870BD516889B271B9D4E9095085420E
:1091A00018D0A6690644D66018D9281A80B2506033
:1091B000A562002184F86410116841F00101DBB25E
:1091C000116083F3118870BD226ED36843F0800371
:1091D000D36070BD012284F86420D7E72569281A7E
:1091E00080B25060A162E4E770B5094C236873B1A6
:1091F0000546002606E099681A681E7321609047AC
:10920000236823B15A68AA1A002A1846F3DA70BDF7
:109210007CA50020A64B1A6812F0040140F0EA80F9
:10922000DFEDA46AA44B12F0200205D093F8D02001
:1092300012F0020240F0BC809FEDA04A93F80001BA
:1092400010F0010062D193F8011119B183F8020105
:1092500083F80101D3ED417A9FED997A9FED996AE8
:1092600067EE877A93ED437AE6EE867A36EEC77A32
:10927000C3ED417A83ED427A002A40F08B80DFED26
:109280008D7A002193ED497A93ED4A5A37EEC76AF9
:10929000D3ED487AA5EE067A37EE676A83ED497A10
:1092A000E5EE067AC3ED487AC3ED477A09B1C3ED1E
:1092B000427A93ED4B6A93ED4D7ADFED835A93ED4D
:1092C0004E5AC3ED4B7A37EEC66AF0EE474AD6EEF9
:1092D000254A7E4AF0EE477AE5EE247A127893ED3D
:1092E0004C6AC3ED4D7A37EEC67A0E2AA5EE076AB0
:1092F00083ED4C6A69D0242A27D1D3ED427A744B8E
:10930000FDEEE77A17EE902A5A80704793F8010134
:1093100028BB93ED417A012036EEC76A83ED437A8C
:1093200083F801010AB393F80221002A40F08780F4
:1093300051B3D3ED357A77EEE65A012275EE875AAE
:1093400083F80221C3ED445A7DE0372A40F0AE8015
:10935000FDEEE66A5E4B16EE902ADA80704793EDDA
:10936000437A36EEC76A002ADDD193F80221002A3B
:1093700045D093F814219FED4F4A002A6BD0022A62
:1093800002D009B1012A42D0D3ED477AF0EE466A05
:10939000012177E793F81411D3F8D420C3F81021F2
:1093A0000120814283F8020118BFC3F8082166E753
:1093B000D3ED387AB3F8E620F8EEE77AC3ED357AE4
:1093C0005ABB9FED3E4A012238E764EE255AD3EDA1
:1093D000357A3F4BFDEEE55AFDEEE66A15EE902A32
:1093E000FDEEE77A1A8016EE902A5A8017EE902A40
:1093F0009A807047304B0121D3ED316A13E7002981
:1094000051D093F814219FED2B4A002ABAD1F0EEE7
:10941000467A0121F0EE466A34E707EE902A9FED86
:109420002A6A9FED2C7AF8EEE77A86EE274AB4EEA8
:10943000C74AF1EE10FA88BFB0EE474AC3E7D3ED52
:10944000357AD3ED445A93F8142177EEE57AC3EDDB
:10945000477A002A93D1002996D093ED475A93F882
:10946000152175EE666A07EE902AF8EEE75A76EE59
:10947000877A9FED197AF0EEE77A67EEA57AF0EE3B
:10948000466AF4EEC77AF1EE10FAC4BF24EE077A0A
:1094900087EE274AF7EE007A77EEC47A67EE867A8F
:1094A000E5EE047AEEE69FED034A6DE7704700BFF4
:1094B00020560020000000007CA500209A99993ECB
:1094C000CDCC4C3FCDCC4C3E0000C8424D1E0020C0
:1094D000501E00206666663F00401C469C4B1B6881
:1094E000D90600D47047F0B59A4C2DED028BD4F814
:1094F0004C3187B013B104F59E709847D4F85031C1
:10950000002B75D0944894ED648A9847C21C054698
:109510007CD000287EDA431C00F00B816FF0010242
:10952000C4F858218D4E3368EB1A03FB03F34FF652
:1095300009218B42DCBF8A49A1FB031394F8AD11CA
:1095400004EB4100D4BF43F3CF034FF4C853A0F85A
:10955000B0314B1CDBB2052B84F8AD3100F09380A9
:1095600094F8BA313560002B00F09A80B4F8B2015B
:10957000B4F8B031B4F8B41194F864610344B4F8A9
:10958000B6010B44B4F8B81103440B441BB2B3F555
:10959000FA4F1946A8BF4FF4FA4121EAE171A4F845
:1095A0006C1146B9002A06DDB3F5167FC0F285803E
:1095B000012684F864616B4B18781B284DD01C2859
:1095C0003FD1D4F85C71684DD4F868312A80002FFF
:1095D0006E80AB8033DD002A31DDB1F5167F2EDAE7
:1095E000002E00F0B0809342D4BF0023012327E077
:1095F0005C494FF0FF330878C4F858311A461B28ED
:10960000C4F85C3102D1584D6A80AB8007B0BDEC24
:10961000028BF0BDD4F89431544904EB830201333A
:109620000968C4F86011052BC2F89801C4F8943198
:1096300053D094F8AC31002B55D1024670E700238B
:10964000EB80D4ED557AB4EEE78AF1EE10FA0DD541
:109650004FF0FF33C4F85C31D8E7D4ED557A424D72
:10966000B4EEE78AF1EE10FAE98014D4002A6CDB3C
:1096700007EE902AF8EEE77A67EE887AFDEEE77A51
:1096800017EE903ABBE7002384F8AD31012384F84C
:10969000BA3135606AE74FF0FF33C4F85C31B3E7A5
:1096A00094F864614FF6FF73A4F86C314FF0FF310A
:1096B000002E80D1002A7FF77EAFD4F86831934224
:1096C0003FDA2B4802EB8203C3EB0313A0FB030337
:1096D0005B09C4F8683100266DE700220123C4F855
:1096E000942184F8AC31234F0FCF01AE0FC6029AFC
:1096F0003B683360904202DC134602461846DDE9BF
:109700000413994202DC1E460B4631468142A8BF33
:1097100001469A42B8BF1A46039B8B4202DB0846B9
:10972000194603468A42A8BF0A469A42B8BF1A465B
:10973000F6E60E4BC4F858011B68C4F860310246C7
:10974000F0E6002637E701237AE74FF0FF3356E7CC
:10975000205600207CA50020B8A600200C06002082
:10976000CDCCCCCC4D1E0020501E0020881E0020E9
:109770001F85EB5114A70020038A2DE9F047B0F8AC
:109780000C901FFA89F919EA03092BD005460E46F9
:109790004FF000474FF00008B9FA89F327FA03F2B7
:1097A000D24391B21B3B298209EA0209042B16D845
:1097B000DFE803F0352C231A0300B36A002B37D0FF
:1097C00003F1FF3A1FFA8AFAC6F82880746A34B1A6
:1097D00023682046514698476468002CF8D1B9F1B7
:1097E000000FD9D1BDE8F0877068696B036889B252
:1097F0009847B9F1000FCFD1F4E7B068A96B0368BF
:1098000089B29847B9F1000FC6D1EBE7F068E96B70
:10981000036889B29847B9F1000FBDD1E2E730691A
:10982000296C036889B29847B9F1000FB4D1D9E720
:10983000E96A1FFA81FAC9E708B5254B1B68DB0402
:109840000AD5B5EE400AF1EE10FA12D19FED210AC9
:1098500043F0A4FC80B208BDDFED1F7AB4EEE70A46
:10986000F1EE10FA1CDA9FED1D0A43F097FC80B26E
:1098700008BDDFED197AB4EEE70AF1EE10FAE5D48F
:109880009FED177AB4EEC70AF1EE10FA14D870EE15
:10989000677A9FED147A9FED140AA7EE870AE4E732
:1098A00070EE677A9FED117A9FED110AA7EE870A95
:1098B00043F074FC80B208BDDFED0E7A9FED0E7AA6
:1098C00070EE677A9FED0D0AA7EE870ACDE700BF1D
:1098D000004D00200080BB440000404200007A445C
:1098E00000E0824466BEFFBE0060BB4438DFFF3E3E
:1098F00000407A440000834466BEFF3E00A0BB44A3
:109900002DE9F04F0C4695B03549054620461746DF
:10991000FEF75AFB0646002850D132492046FEF792
:1099200053FB064600284BD12F492046FEF74CFB3F
:109930000646002846D12D492046FEF745FB06463F
:10994000002841D120462A49FEF73EFB0028064662
:1099500012BF0824264601240FB144F01004254903
:109960003046FEF731FB88B344F0200414F48073D2
:109970000CBF012000200793FBF71EFE14F0090F17
:1099800000F01E831C48FAF7B3FB00212846FEF7BF
:10999000A7FC079B002B3BD11848FAF7A9FB1848F6
:1099A000FAF7A0FB04F01803182B05D11548FAF7B5
:1099B0009FFB1548FAF796FB01232AE00124CBE729
:1099C0000224C9E70424C7E78124C5E70F493046CC
:1099D000FEF7FAFA0028C9D044F48074C6E700BF45
:1099E000B4A40608BBA40608C3A40608C9A40608B4
:1099F000D2A4060838A10608D6A40608DEA40608E4
:109A0000F6A4060802A506082AA50608FBA0060873
:109A100000230693FAF74EFB04F01003B949BA4845
:109A20000593FAF72DFCB949B948FAF729FC04F473
:109A30008473082B07D1B7492846FAF79BFCB54930
:109A40002846FBF7B1F914F0800309930ED1B24B0D
:109A500093F8BC21002AB14A03F5DE7306BF012149
:109A600013460021AE4A2046FAF728FBAD492046AE
